:020000040000fa
:080000003001040000000000c3
:020000040000fa
:1002000068060400000000004a0704000000000027
:10021000fa18040000000000d21b040000000000d7
:10022000421f040000000000521b040000000000f8
:10023000321d040000000000d41f04000000000074
:10024000c81f040000000000fa1a040000000000ab
:10025000621c040000000000ca1c04000000000032
:100260008fdd20008079220000018800000000005e
:10027000050007000c000700260a0200000000002d
:100280000040da000000fe004440a9000000200009
:100290000000e0000300320000002000a001880000
:1002a0004440a8000000060020c8200011002000e3
:1002b0001600370062004000e0804800910188008d
:1002c0009001ba0062004000e0804800910188007f
:1002d0009002ba0062004000e08048000002eb009b
:1002e0006028e10005003a008301e90007003300bf
:1002f000038009000059eb00040037006128e10089
:10030000010032000082eb00050007009101880027
:100310001001ba000200e000e6ff3a00000005000c
:10032000910188008002780062004000e08048006f
:100330003559ba008301e900080032002559ba0096
:100340008301e900050032000400e000f4ff320000
:1003500015d9ba008301e900f1ff3a000000060058
:10036000889fbe00e30440000900a100808f540074
:1003700049003600e38f540001003e004900200090
:10038000704280000000e00002003200800078002f
:100390000c0037000185200003003700908f5400c7
:1003a000230036008080e800110078001100e00092
:1003b000faff3a000f003700928f54001c003600fd
:1003c0008280e800110178001100e000faff3a0095
:1003d000100178000185200003003700908f540041
:1003e000130036008080e80011007800820f500072
:1003f000faff3a0068428000890f54000100310082
:1004000009047800080078006b0007000000e00095
:1004100004003a00890f54001f0032000804d10084
:10042000f5ff37000818780030000700d4ff3700c8
:10043000110178009201780064805100890f50000a
:100440000300310012009000800878000700370098
:100450000900410080087800920190001300980084
:1004600011007800128814000909780091017800c1
:100470001100e00004003200130090008380e800c7
:100480000000e00001003a008000eb0071428800ab
:100490000280e800010037000000eb004f04be00be
:1004a00000000600000478000600370082004100ca
:1004b000a0428000e10078000200e800904288003d
:1004c0000100010092428000b0428000800f510084
:1004d000f6ff390000802000a042880020022000a2
:1004e000b0428800080078003a0007000000e000f1
:1004f000300032008080e90091027800e38f5200e2
:100500002c0036000508a3002a003a008242800031
:100510000200e00002003200828f5000040031002f
:100520000208780081428800160037000301780035
:10053000920190000300e00002003200818f510020
:10054000faff39001202780004004100808f500049
:1005500018003900810f500003003a0005094200dd
:1005600082007800070037000300e000030032003b
:1005700005804000808f51000e00390093009800e4
:1005800011019800110190000200e0000900320002
:1005900011804000820f500006003a004e28ef0004
:1005a00011009000110178009008410010009000a7
:1005b00090009800000006000000e00003003400f6
:1005c0000c000700e10f400001003a000000eb00c2
:1005d000000006000c02e20004003d000f42ab00e8
:1005e000020032000f02ab00feff32000040da00d2
:1005f000feff3700889fbe0080047800d042800054
:100600000000e00003003a00100007000000e000d6
:100610000a003500d04280000900e00002003a00e4
:10062000000478000600370000047800090040004c
:10063000060007000000e00001003d000084eb0020
:10064000080078004f04be0000000600800078001b
:100650000000e00004003a0000d12000d0428800f1
:1006600001017800060037000081eb0080dd2000ea
:10067000808f500002003e00d14288000001eb0054
:100680000200780000000600839f68000100e0007f
:1006900002003d0060001000e08018000300e00050
:1006a00002003d0060011100e081190025010700f2
:1006b0004f00e00002003b0060001000e0801800e6
:1006c00000000600889fbe008a9fbe0001057800da
:1006d0000100e0000400350008003c000000e000dc
:1006e000200032000500370060001000e080180094
:1006f00002003b0001f02c001a0037000004be008d
:100700006011b8006b0920000982cf000200390097
:100710000882cf000441b000694252000e0032004e
:1007200008003b0082817100610164008904d100ee
:100730000884d3008b05e8000442e800f9ff3a0082
:10074000050037000804440089844c008b05e9004b
:100750000442e900fbff3a000a0107000af0a70083
:1007600001f0a0004f05be004f04be0000000600cf
:10077000889fbe008a9fbe008c1f7800270107005b
:100780002e01330003866c006450e1002e0032001d
:100790006420e100330032006150e1002f0032009c
:1007a0006120e1003100320085855500eb07b00083
:1007b0000900200008042000050037000804440058
:1007c00089844c000a0031000603430087834b00f4
:1007d0000001530081815b00f8ff33000203be007b
:1007e0000800a0000804440089844c00f6ff39008a
:1007f000c639dd00830173000100320013002000c0
:100800008904d1000884d3000998a30005003200b0
:100810000800a7000300a0008904d1000884d300c9
:100820008b05e8008904d1000884d3000001eb00a7
:100830000281d200d300070001f0a1000cf0a70054
:1008400001f0a000060137006420e1000801320039
:100850000801be000200be00f7ff37006120e10082
:10086000030132006000b800f3ff370000002000f1
:1008700001f82700f0ff37000001be00ff0007006d
:100880000470a70003f0a1006509b1001600320052
:100890000d0035006828e10006003500f0ff2f004c
:1008a000f1ff27000300e00013003b0001002800d7
:1008b0000000050000004000818048008502e9003a
:1008c000fcff3a0008003700f88f420002003c00ad
:1008d0008000eb00000005008100d1000080d30003
:1008e0008502e800fcff3a000300e00002003b0044
:1008f00060001000e080180000000600889fbe0025
:100900008a9fbe008c1f7800c4000700cb00330014
:1009100003866c006450e100240032006420e10092
:10092000270032006150e100220032006120e10026
:10093000210032008b854200eb07b1000134b80082
:10094000003ab8000804420089844a00013ab8001d
:100950000030b8008880400009014a0004003300dc
:100960000000400081804800020149008b05e90039
:10097000c909dd008301700001003200130020006e
:10098000c814de004814dd004709de001200b20082
:10099000c808de00088470007a00070001f0a1009a
:1009a0000cf0a70001f0a000ad0037006120e100cd
:1009b000af0032000801be000200be00f7ff3700a2
:1009c0006150e100fcff3a00a900370003f0a200eb
:1009d000889fbe008a9fbe008c1f78008f00070092
:1009e000960033006450e1004f0032006420e100c3
:1009f0005200320003826c0007003b000905d00062
:100a00000306d000820f54000c065d00020039007e
:100a100002003200890178000306780085825500c3
:100a200004003d000003fd008103fd008502ea0093
:100a30008b854200840f720002003b0060001000b2
:100a4000e08018006011b8000005eb007a28e10092
:100a50000a00390006007800c75ddd00f707b20024
:100a6000878075002d003700828171000a017800af
:100a7000610560008180d1000080d3008502e9001b
:100a8000f9ff3b00060440008784480002003b0059
:100a900060041400e0841c000988a30007003200f1
:100aa0008a81710082817100610164008904d10032
:100ab0000884d3008b05e800170037000978a300ed
:100ac00013003a000b00e000130034008b05e9002e
:100ad0000804440089844c000a4474000978a30087
:100ae0000d003a000b00e000070034008b05e90020
:100af0000804440089844c0001003a000b002000e7
:100b00000978a300f7ff32000001eb000200370074
:100b1000828171000a0178001a0007000cf0a7001a
:100b200001f0a0004e0037006420e10002003a000e
:100b3000838f6c004e0033000801be000200be002f
:100b4000470037006022b800060220000000d000f5
:100b50008180d2000482d2008582d2000000a000f1
:100b60000202520083825a0003003b00020242004c
:100b700083824a000000a1000603e900f3ff3a0067
:100b80000000060081002000618055000b003d0040
:100b90000b00200061fe2f000100e1001d00340069
:100ba00082817100610164008904d1000884d3004e
:100bb0000000e800faff3a007100200061006400c4
:100bc000030070000200600009003200610444006c
:100bd000e0844c000988a500050032008b05e80080
:100be0006808e10002003a008904d1000884d300bb
:100bf000f20f20000258e10005003d00c75ddd0056
:100c0000f907b2008980750008007800000006002e
:100c10000bf827008b007800000005000004be00e0
:100c2000160007000003be000405be000200be005f
:100c300012000700844f7500000006000200be008d
:100c40006450e100050036006420e1000200360037
:100c50000968a30001003a000800be000160a0007e
:100c60004f0678004f05be004f04be00000006008e
:100c7000f0ff2f00f1ff2700f9ff3700c70ade0061
:100c8000f107b200f50fb20008003200e1cf4200d8
:100c9000020032000170a00024000500810f7000e6
:100ca000010032000408050044000500810f7000b7
:100cb00002003a00140005008502e900000040002f
:100cc00081c04800fcff3b000170a000240005002b
:100cd0000400fa00506780000000e0001e003200af
:100ce000f166800080da2f00808f50001a003500f6
:100cf000f166800080252000808f500016003c00a7
:100d0000d602a900d622a900d642a900d662a9001f
:100d10000000eb0050678800f2668000020f780048
:100d20001e0178000200e00003003d001e01780073
:100d30000201ea00020f7800007122001e01780013
:100d4000110009000200d800ef005000806620006a
:100d5000f90607004d003700f06680000000e00053
:100d60000c003400306780000000e8003067880025
:100d7000106780000000e90010678800106780009d
:100d80000000e0000e003d003000200010678800e9
:100d90000b003700306780000000e90030678800f2
:100da000106780000000e80010678800106780006e
:100db000e30f5000020034000000eb0010678800d1
:100dc00010678000100798001e019000e10f51008d
:100dd000130032001e009000e10f500004003c00a0
:100de0001e0190000200e000080032001a003700e7
:100df0001e009000e20f50000e0032001e01900015
:100e0000e30f51001000320013003700d602a90092
:100e1000d622a800d642a900d662a8000e0037004c
:100e2000d602a900d622a800d642a800d662a90000
:100e300009003700d602a800d622a900d642a80091
:100e4000d662a90004003700d602a800d622a90065
:100e5000d642a900d662a800f166800080da2f0091
:100e6000808f500009003500f16680008025200049
:100e7000808f500005003c00100020005067880063
:100e8000f100200080662000ab0607000080fa0019
:100e9000000006000400fa00606780000000e00027
:100ea0001e0032000167800080da2f00808f500022
:100eb0001a0035000167800080252000808f5000d7
:100ec00016003c00d682a900d6a2a900d6c2a9006d
:100ed000d6e2a9000000eb0060678800026780008e
:100ee000020f78001e0178000200e00003003d00c0
:100ef0001e0178000201ea00020f78000071220052
:100f00001e017800110009000200d800ef00500017
:100f1000a0742000880607004d003700006780009d
:100f20000000e0000c003d00406780000000e90088
:100f300040678800206780000000e9002067880083
:100f4000206780000000e0000e003d00300020001f
:100f5000206788000b003700406780000000e80031
:100f600040678800206780000000e8002067880054
:100f700020678000e30f5000020034000000eb0007
:100f80002067880020678000100798001e019000ed
:100f9000e10f5100130032001e009000e10f5000dd
:100fa00004003c001e0190000200e0000800320036
:100fb0001a0037001e009000e20f50000e003200b1
:100fc0001e019000e30f51001000320013003700a3
:100fd000d682a900d6a2a800d6c2a900d6e2a8004f
:100fe0000e003700d682a900d6a2a800d6c2a8005b
:100ff000d6e2a90009003700d682a800d6a2a9002f
:10100000d6c2a800d6e2a90004003700d682a80004
:10101000d6a2a900d6c2a900d6e2a8000167800026
:1010200080da2f00808f50000900350001678000b2
:1010300080252000808f500005003c00100020001b
:1010400060678800f1002000a07420003a060700c5
:101050000080fa00000006000000fa008000eb00ab
:1010600080662000db0507008000eb00a0742000f4
:10107000d80507000080fa00000006000200fa0010
:10108000000f78001e00e0000a003a000000eb00ac
:10109000f06688008000eb008066200026060700ce
:1010a000d602a900d622a900d642a900d662a9007c
:1010b0002d00370080c12f009e0f10000a003d0058
:1010c00080c12f00f0668800008f2d00f26680003e
:1010d000110009000200d8008000fd008066200099
:1010e0001506070020003700803e20009e0f1000ec
:1010f0000a003400803e2000f06688000071220063
:10110000f2668000110009000200d8008000fd0096
:101110008066200008060700130037001e007800d4
:10112000f06688001e00e00008003d00008f2d00e2
:101130001e017800110009000200d8008000fd00a7
:1011400080662000fc0507000700370000712200c0
:101150001e017800110009000200d8008000fd0087
:1011600080662000f40507000080fa0000000600f9
:101170000200fa00000f78001e00e0000a003a00aa
:101180000000eb00006788008000eb00a0742000e6
:10119000e9050700d682a900d6a2a900d6c2a900f7
:1011a000d6e2a9002d00370080c12f009e0f10004d
:1011b0000a003d0080c12f0000678800008f2d00cd
:1011c00002678000110009000200d8008000fd00c5
:1011d000a0742000d805070020003700803e2000c2
:1011e0009e0f10000a003400803e20000067880037
:1011f0000071220002678000110009000200d8007f
:101200008000fd00a0742000cb050700130037000c
:101210001e007800006788001e00e00008003d0006
:10122000008f2d001e017800110009000200d80077
:101230008000fd00a0742000bf05070007003700f4
:10124000007122001e017800110009000200d80080
:101250008000fd00a0742000b70507000080fa00a0
:10126000000006000800fa00000f7800110798003f
:101270001e007800200798002e0190000200e00078
:1012800003003d002e0090000000ea0020079800b7
:101290001e019000320798003e0090000000e00020
:1012a00003003d003e0190000201ea003207980071
:1012b0002e0090003e01900082004000803e200001
:1012c000808f500006003c001e0090001e001000a1
:1012d0006aff07001e0090001e004000a4ff0700e8
:1012e0000080fa00000006000000fa00306780006d
:1012f0000080fa00000006000200fa00000f7800eb
:101300001e007800306788000080fa0000000600a8
:101310000000fa00406780000080fa00000006002c
:101320000200fa00000f78001e0078004067880075
:101330000080fa00000006000000fa00c4c2a90004
:10134000c4e2a900c522a900c582a900c542a9001e
:10135000c5a2a900c5c2a900c5e2a900c0c2a900d2
:10136000c0e2a900c122a900c182a900c142a9000e
:10137000c1a2a900c1c2a900c1e2a900d022a9004e
:10138000cc22a900d042a900cc42a900e2e2a900e7
:10139000e302a900e802a900e822a900dee2a90010
:1013a000df02a900e402a900e422a900e202a900e8
:1013b000de02a900d602a900d622a900d642a900c1
:1013c000d662a900d682a900d6a2a900d6c2a900d9
:1013d000d6e2a900d202a900d222a900d242a900d5
:1013e000d262a900d282a900d2a2a900d2c2a900c9
:1013f000d2e2a900d1a2a900cda2a900e842a90089
:10140000e862a900e442a900e462a900de22a80083
:10141000dec2a800e4c2a800e4e2a800e502a80039
:10142000e522a800d302a800d322a800d342a80036
:10143000d362a800d382a800d3a2a800d3c2a80078
:10144000d3e2a8000080fa00000006000200fa00c3
:10145000b9ff0700ca040700fffe07000040eb00c9
:101460004100070040c7bf00614060000004e00089
:10147000020032004007a9000000fe001e00070025
:10148000000f7800f00020009e0f100002003a00cc
:10149000b10a070006003700e00020009e0f100090
:1014a00002003a009e0a070001003700d30a070035
:1014b000ffff37000800fa00200798003107980066
:1014c0006000b800008fbe0004003700100020004c
:1014d000010020001e0f40005e9748002e00900083
:1014e000be009000be0f1000ae8f1800f7ff350051
:1014f0000080fa00000006000000fa00e6c2bf000b
:101500000080fb004600de00614060000081fb00bf
:10151000e7c2bf000080fb000000d1006140600016
:101520000080fb000000400080007800e7c2bf00a0
:10153000614060000080fb0000804000000040002f
:1015400080007800e6c2bf000080fb004700de009c
:101550000080fb00008040000000400000004100cf
:101560000080fa00000006000200fa00004f780038
:1015700010c0b3009e4f100004003a00e185200027
:1015800010c0b3008048780003003700e1852000d8
:101590000040eb00804878000000eb000015880058
:1015a0000000eb00101588000000eb0020158800fb
:1015b0000000eb0030158800a802a800a822a800af
:1015c000a842a900a862a900a882a900a8a2a9000f
:1015d000a8c2a900a8e2a900a902a900a922a900fd
:1015e000a942a900a962a900a982a900a9a2a900eb
:1015f000a9c2a900a9e2a900aa02a900aa22a900d9
:10160000aa42a800aa62a800aa82a800aaa2a900c9
:10161000aac2a900aae2a900ab02a900ab22a900b4
:10162000ab42a900ab62a900ab82a900aba2a900a2
:10163000abc2a900abe2a900112a200091407800ba
:10164000c0cfb30000c06000a1e2b700a042a80074
:10165000012a20009140780000ceb30000c0700045
:10166000a0e2b700212a20009140780030ccb300de
:1016700000c060000034a000a2e2b700a342a800ae
:10168000512a20009140780000ceb30000c06000d5
:101690000004a000a5e2b700e08520001004e000ef
:1016a00007003200412a20009140780000ccb300ae
:1016b00000c060003041b300a4e2b700070037006b
:1016c000412a20009140780000ccb30000c06000a7
:1016d00071c2b30001407000a4e2b7008560a900a8
:1016e0008d60a800a1e2a800e08520001004e000c1
:1016f00005003a000000000031688000000320006f
:10170000808f5000fbff36000080fa0000000600ca
:10171000809fbe000a00fa00c18520000040eb0057
:1017200080487800d18520000040eb008048780098
:101730008560a900e08520001004e0002800320048
:1017400000282000000f78002186200020688000fb
:101750000000d000810040001e0078009008780052
:101760001e8fe80021862000206880000000d00045
:1017700001004000810c2000808040001e007800a5
:10178000900878001e8fe8002186200020688000e5
:101790000000d000010040000119200080804000be
:1017a0001e007800900878001e8fe80020688000f6
:1017b0000000e800800078002168880030062000e2
:1017c000808f50006b0136000000eb00206888001d
:1017d000d185200010c0b300804878006501370033
:1017e000c001200050158800212a20009140780077
:1017f00030ccb30000c060000034a000a2e2b7000b
:10180000412a20009140780000ccb30000c0600065
:1018100071c2b30001407000a4e2b700f18520005e
:10182000d0c3b300914f10000f003a00c00f20004a
:1018300050158800212a20009140780030ccb30058
:1018400000c060004041b300a2e2b700412a20007e
:101850009140780000ccb30000c060003041b3007c
:10186000a4e2b7005f003700f1852000e0c3b300b9
:10187000914f10002c003a00212a2000914078005e
:1018800030ccb30000c060000044a000a2e2b7006a
:10189000412a20009140780000ccb30000c06000d5
:1018a0007041b300a4e2b700008620001080fb0066
:1018b000100798001e009000e10f50001100320048
:1018c0009e009000e18f500004003c001e0090003c
:1018d0000000e00008003200420037009e00900047
:1018e000e28f50000a0032001e009000e30f50000b
:1018f0000a0032003b003700c0112100501588005b
:1019000038003700c021220050158800350037000c
:10191000c04124005015880032003700c0812800e3
:10192000501588002f003700f085200021c0b3003b
:1019300090cf10002b003a00212a2000914078001f
:1019400030ccb30000c060000044a000a2e2b700a9
:10195000412a20009140780000ccb30000c0600014
:101960007041b300a4e2b700008620001080fb00a5
:10197000200798002e009000e10f50001100320067
:10198000ae009000e18f500004003c002e0090005b
:101990000000e0000800320012003700ae009000a6
:1019a000e28f50000a0032002e009000e30f50003a
:1019b0000a0032000b003700c011210050158800ca
:1019c00008003700c02122005015880005003700ac
:1019d000c04124005015880002003700c081280053
:1019e0005015880000282000000f78002186200074
:1019f000206880000000d000810040001e007800b8
:101a0000900878001e8fe800218620002068800062
:101a10000000d00001004000810c200080804000c8
:101a20001e007800900878001e8fe80021862000b4
:101a3000206880000000d000010040000119200053
:101a4000808040001e007800900878001e8fe8001b
:101a5000206880000000e80080007800216888008d
:101a600030062000808f5000020036000000eb009e
:101a700020688800f1852000e0c3b300914f10007a
:101a800022003a00306880000000e8008000780002
:101a90003168880010032000808f5000020036005b
:101aa0000000eb0030688800a1ab200030688000a7
:101ab0000000d000810040001e00780090087800ef
:101ac0001e8fe800a1ab2000306880000000d0002d
:101ad0000100400041062000808040001e00780088
:101ae000900878001e8fe800a1ab200030688000cd
:101af0000000d00001004000810c200080804000e8
:101b00001e0078009008780091003700f1852000d1
:101b1000f0c3b300914f10003f003a000086200050
:101b20001080fb0030079800be009000e18f50004d
:101b3000180032003e009000e10f500004003c000d
:101b4000be0090000100e000080032008000370075
:101b50003e009000e20f500019003200be009000dd
:101b6000e38f5000210032007900370061be200071
:101b70001e007800900878001e8fe80061be2000eb
:101b80001e00780010007800c0009800e2e2a80073
:101b90006f00370061be20001e0078001000780042
:101ba000900098001e8fe80061be20001e007800a3
:101bb00010007800d0009800e302a800640037000d
:101bc00061be20001e00780010007800a000980080
:101bd0001e8fe80061be20001e0078001000780013
:101be000e0009800e802a8005900370061be20001c
:101bf0001e00780010007800b00098001e8fe800ea
:101c000061be20001e00780010007800f0009800ef
:101c1000e822a8004e003700f085200031c0b30054
:101c200090cf10004a003a00008620001080fb0090
:101c3000400798004e009000e10f50001b0032005a
:101c4000ce009000e18f500004003c004e00900058
:101c50000000e000080032003d003700ce00900098
:101c6000e28f50001f0032004e009000e30f500042
:101c70002a0032003600370061bf20001e007800c5
:101c8000900878001e8fe80061bf20001e007800d9
:101c900010007800c0009800e2e2a9000186200050
:101ca00010c0b300804878002900370061bf2000d1
:101cb0001e00780010007800900098001e8fe80049
:101cc00061bf20001e00780010007800d00098004e
:101cd000e302a9000186200020c0b30080487800fc
:101ce0001b00370061bf20001e0078001000780044
:101cf000a00098001e8fe80061bf20001e00780041
:101d000010007800e0009800e802a9000186200099
:101d100030c0b300804878000d00370061bf20005c
:101d20001e00780010007800b00098001e8fe800b8
:101d300061bf20001e00780010007800f0009800bd
:101d4000e822a900018620000040eb0080487800ce
:101d5000f0852000904078001048e800f0c3b30000
:101d600080cf500003003600f18520000040eb00da
:101d700080487800c185200010c0b30080487800fa
:101d80000080fa004f00be00004006000000fa008c
:101d9000c08520001080fb000080fa0000000600d3
:101da0000000fa00d08520001080fb000080fa00bf
:101db000000006000000fa00a1e2a8000080fa007e
:101dc000000006000000fa00a1e2a9000080fa006d
:101dd000000006000200fa00000f780023862000b1
:101de0009e007800400620000008b80022688000ad
:101df000020040000000d000030040001000780006
:101e00000080fa00000006000c00fa00000f7800c5
:101e1000110798006000b80020079800310798006b
:101e2000200020009e0f100031003e001e00900098
:101e30000000e0002e0032009e00900040062000ce
:101e4000808f50002a003e000000eb004007980001
:101e5000216880001e009000008050005006b000f5
:101e600042062000110009000280d8008000fd0019
:101e700050079800ce0090001e009000808f500008
:101e80001b003100238620009e00780040062000c1
:101e90000008b8005e019000020040000000d00081
:101ea00003004000100078006101b9002e0090008e
:101eb000be0090000000410081804900200798008a
:101ec000310798004e0090000000e800400798009d
:101ed0005e0090000000e8004206200011000900aa
:101ee0000200d8008000fd0050079800e1ff370095
:101ef0001e0090006101b8002e009000be0090000e
:101f0000e1f907000080fa00000006000800fa006e
:101f1000000f78000000eb002007980070382100c7
:101f2000300798000000eb00100798009e0090001a
:101f300030062000808f50002f003c0023862000b8
:101f40009e007800400620000008b8001e019000a6
:101f5000020040000000d000830040002e009000ee
:101f6000910f10000b003400238620009e007800a3
:101f7000400620000008b8001e019000020040004a
:101f80000000d000030040001000780020079800f7
:101f900015003700238620009e00780040062000b0
:101fa0000008b8001e019000020040000000d000b0
:101fb000830040003e009000910f10000a003d0099
:101fc000238620009e007800400620000008b8000c
:101fd0001e019000020040000000d00003004000fd
:101fe00010007800300798001e0090000000e80004
:101ff00010079800cdff3700ae0090003e00900023
:10200000008050000080fa00000006000800fa007e
:10201000000f780011079800220798002e0090000a
:102020000000e00024003200ae00900040062000d6
:10203000808f500020003e000000eb003007980029
:10204000be0090002e009000808f50001a003100da
:10205000ae0090003e009000008050008000d00054
:102060001e009000008040000082e90025862000cc
:102070009e017800216880003e00900000804000b2
:1020800042062000110009000280d80001017800fa
:10209000400620000018b800000041000000d000f9
:1020a00005004000100a78003e0090000000e800a3
:1020b00030079800e2ff37000080fa0000000600b9
:1020c0002800fa00889fbe008a1f78000000eb00fd
:1020d000000f78000000eb0010079800700020004f
:1020e0009e0f10000f003c00e1ce20001e00780083
:1020f0000000d000810040000000eb008008780064
:10210000680147009e007800400020000008b800e9
:10211000000141006000b8000089be001e0fe80009
:10212000eeff3700000000009e0090003006200007
:10213000808f50002b003c000000eb00000f780067
:10214000700020009e0f100022003c006801470034
:102150009e007800400020000008b8008004410084
:10216000680147009e007800400020000008b80089
:10217000000441001e00780039000700cf80de0017
:10218000b81c4000a89448006000b80020079800e0
:10219000310798002e019000be019000703e200093
:1021a00001002000800f5100818f590007003c0082
:1021b0002e009000be00900061004000e0804800ca
:1021c0002007980031079800f2ff37001e0fe80043
:1021d000dbff37001e0090000000e80010079800a9
:1021e000d1ff37000000eb00000f780070002000e6
:1021f0009e0f100016003c00e1ce20001e0078006b
:102200000000d00001054000680147009e007800f2
:10221000400020000008b800000041001000be008f
:1022200028f907000004be001e009000cf80de00e9
:1022300024f907000001be000800be004cf90700a9
:102240008df90700000d78001e0fe800e7ff37004a
:102250004f0578004f04be000080fa000000060021
:102260000400fa00000f7800700020009e0f10009c
:10227000030036000000eb00100798000b00370049
:1022800061be20001e0078000000d0000101400067
:1022900061bf20001e0078000000d0000100400057
:1022a0001201780010005100100798001e009000e5
:1022b0000080fa00000006000600fa00000f780017
:1022c000700020009e0f1000030036000000eb009d
:1022d000200798001800370061be20001e0078001b
:1022e0000000d0000101400061bf20001e00780006
:1022f0000000d000010040001201780010015100e0
:10230000e1ce20001e0078000000d0000100400057
:1023100010005100100798001e0090000000e0001f
:10232000030034001e0090002007980002003700d0
:102330000000eb00200798002e0090000080fa00bb
:10234000000006000400fa00000f78007000200072
:102350009e0f1000030036000000eb0010079800ed
:102360000600370061be20001e0078000000d0008b
:102370000100400010007800100798001e00900037
:102380000080fa0000000600811f7800801f78009e
:10239000f0ff2700c0128800003020000000b300ca
:1023a000d0128800de02a90000000000e002a900af
:1023b0009001090000000000e002a80041e2a8002e
:1023c0004602ae00feff3700f0ff2700c012880073
:1023d000004020003001b300d01288004602ae0059
:1023e000feff3700f0ff2700c01288000010200019
:1023f0000030a0000040a000d01288004602ae00cd
:10240000feff3700f0ff2700c012880000202000e8
:10241000d01288004602ae00feff3700f0ff270012
:10242000c0128800006020000010a000d0128800b8
:102430004602ae00feff3700f0ff2700c012880002
:1024400000702000f005b300d01288004602ae00f4
:10245000feff370001f02000301280000100600014
:102460000000e000fcff3a00301280000100600034
:102470000000e000fcff320030128000010060002c
:102480000000e000fcff3a00301280000100600014
:102490000000e000fcff32004662ae0002003700a0
:1024a000801280009012800041e2a900f01e2000fe
:1024b000101288004362a8004342a8008920a900a6
:1024c000a8c0a800a8a0a900a880a9009120a800e1
:1024d00041e2a8004f007800cf007800000006001d
:1024e000801f78004022ef004222ef004422ef00dc
:1024f0004822ef004c22ef00c6e2a800e5a2a900a6
:10250000e582a800e5e2a900e5c2a9004002a90011
:102510004022a90040a2a9004122a90040c2a8006f
:102520004102a9004142a900f00e200010128800cb
:102530004362a9004342a800300020002012880016
:102540004c02a8004802a8008920a9009120a900f7
:1025500041e2a9004f007800000006008920a90090
:10256000809fbe00829fbe0080128000901280007b
:10257000a0128000b01280004408e20022003a005d
:102580004808e200200032003400f8004400f8005f
:102590004440a80050428000a0018800c142800051
:1025a0001e000700110078000000a100c012880082
:1025b0001a000700110078000000a100d012880066
:1025c00016000700110078000000a100e01288004a
:1025d00012000700110078000000a100f01288002e
:1025e00048a8ed0048a8ed00c1428800a101800084
:1025f000514288004400f9003400f9004f01be0048
:102600004f00be00004006004628ef0044a8ef003f
:102610004f01be004f00be0000400600e2804000b7
:1026200004003900a1018000e1804000a101880080
:1026300001002800000006000200fa00e202a800e3
:102640000000eb00000f7800f07022009e0f1000d9
:1026500002003c001e0fe800fbff3700a0ff070050
:1026600049ff07000080fa00000006000400fa009d
:10267000000f78001107980046a8ef004428ef00eb
:102680009e0090001e007800060007000080fa00ff
:10269000000006000000fa00e202a9000080fa0033
:1026a00000000600811f7800821f78004100dd00d5
:1026b000030037004f017800cf00780000000600cb
:1026c000414288000001eb00a1152a008100400072
:1026d0000300390002002800828040001200200020
:1026e0004400f8003400f8004440a8000000200036
:1026f00002004000a001880000000000190007004f
:10270000110078000000a100c01288001500070029
:10271000110078000000a100d0128800110007000d
:10272000110078000000a100e01288000d000700f1
:10273000110078000000a100f012880048a8ed0008
:1027400048a8ed00c1428800a101800051428800e4
:102750003400f900000000004400f9008920a900bd
:10276000d4ff3700e280400004003900a10180005e
:10277000e1804000a101880001002800000006005f
:102780000000fa000000eb00800888000111200022
:1027900091407800f0ccb30000c0600010e1b700b9
:1027a0000000eb0030088800205c200060088800f2
:1027b00084c0a9008cc0a80011e1a8000080fa0024
:1027c000000006000000fa0011e1a9000080fa00f4
:1027d000000006000800fa00000f780011079800ba
:1027e00040688000200798002e0090000000e00064
:1027f0000b0032002e009000300090009e0f500021
:1028000003003a0011002000310798001f00370034
:102810002e0090004000900020079800f2ff370043
:10282000a0002000cef60700200798002e009000a0
:102830000000e00002003a001000200019f7070035
:102840002e0090009e00900001087800ae009000dd
:102850000000eb0090009800ae00900010c0b300a4
:10286000c04098002e0090009e0078003100980033
:102870002e00900041688000410098002e009000da
:102880004068880011002000310798003e00900049
:102890000080fa00000006000800fa00000f78002f
:1028a0000000eb00100798004068800020079800a7
:1028b0002e0090000000e0001a0032002e00900070
:1028c000300090009e0f500010003a001e00900053
:1028d0000000e000050032009e0090002e009000f5
:1028e00040009000c0009800030037002e009000c8
:1028f00040009000406888002e009000fbf6070022
:102900001000200030079800080037002e009000cb
:10291000100798002e0090004000900020079800bb
:10292000e3ff370020002000300798003e009000b1
:102930000080fa00000006000800fa00000f78008e
:102940001107980040688000200798002e00900032
:102950000000e0000e0032002e00900030009000d9
:102960009e0f500006003a002e0090009e0090003e
:10297000010878001000200030079800060037009a
:102980002e0090004000900020079800efff3700d5
:1029900021002000310798003e0090000080fa00de
:1029a000000006000600fa00000f78004068800072
:1029b000100798001e0090000000e0000e0032009a
:1029c0001e009000300090009e0f500006003a005c
:1029d0009e0090000000eb00900098001000200086
:1029e00020079800060037001e009000400090006d
:1029f00010079800efff3700200020002007980004
:102a00002e0090000080fa00000006000600fa0088
:102a1000000f780040688000100798001e009000aa
:102a20000000e0000e0032001e0090003000900018
:102a30009e0f500006003a009e0090000040eb0000
:102a4000c0409800100020002007980006003700c2
:102a50001e0090004000900010079800efff370024
:102a600020002000200798002e0090000080fa002f
:102a7000000006000600fa00000f780040688000a1
:102a8000100798001e0090000000e0000e003200c9
:102a90001e009000300090009e0f500006003a008b
:102aa0009e00900010c0b300c040980010002000ad
:102ab00020079800060037001e009000400090009c
:102ac00010079800efff3700200020002007980033
:102ad0002e0090000080fa00000006003600f8008a
:102ae000809fbe00829fbe00849fbe00869fbe0066
:102af0000200fa0040688000000f780084c0a9003e
:102b00001e00e0001c0032001e00780040409000d3
:102b1000e14f500014003a001e0078001000e00061
:102b2000110032009e0078001e0078001000900016
:102b30000000e800900098001e0178001e00780058
:102b40009000e90012009000810f5000060036004e
:102b50001e00780030009000000001009e00780008
:102b60000000eb00900098001e00780040009000ec
:102b7000000f7800e2ff37000080fa004f03be002c
:102b80004f02be004f01be004f00be003600f900ec
:102b9000004006000600fa00000f780011079800b8
:102ba0001e007800200798002e009000e30f5000d0
:102bb000640032002e009000e30f500007003e003a
:102bc0002e009000e10f50002d0032002e009000ea
:102bd000e10f50003f003e000d0037002e00900036
:102be000e50f50008f0032002e009000e40f5000df
:102bf000700036002e009000e60f5000a500320055
:102c00002e009000e70f5000be003200d2003700c7
:102c10001e009000e10f50000f003600c4c2bf003c
:102c20000080fb004600de000080fb0061006000c9
:102c30000000a200614060004601dd00412c200040
:102c400091407800f0cbb30000c0600002407000fb
:102c5000c4e2b7001c0137002e40900061406000c4
:102c60004601dd00412c200091407800f0cbb300fc
:102c700000c0600002407000c4e2b70012013700db
:102c80001e009000e10f50000b003600c4c2bf00d0
:102c90000080fb004700de000080fb000000a20077
:102ca000c700dd00c4c2bf000074a1000140700075
:102cb000c4e2b700040137002e409000c700dd00d9
:102cc000c4c2bf000074a10001407000c4e2b7009c
:102cd000fd0037001e009000e10f50000f0036008d
:102ce000c5c2bf000080fb000000d1000080fb00d7
:102cf000610060000000a200614060000041d0005f
:102d0000512c200091407800d0cfb30000c060006b
:102d100002407000c5e2b700eb0037002e40900083
:102d2000614060000041d000512c200091407800ab
:102d3000d0cfb30000c0600002407000c5e2b70011
:102d4000e10037001e009000e10f50000f00360038
:102d5000c5c2bf000080fb004400de000080fb0015
:102d6000610060000000a200614060004401dd00dd
:102d7000512c200091407800f0ceb30000c06000dc
:102d800002407000c5e2b700cf0037002e4090002f
:102d9000614060004401dd00512c2000914078002a
:102da000f0ceb30000c0600002407000c5e2b70082
:102db000c50037001e009000e10f50000f003600e4
:102dc000c5c2bf000080fb004200de000080fb00a7
:102dd000610060000000a200614060004201dd006f
:102de000512c200091407800b0cfb30000c06000ab
:102df00002407000c5e2b700b30037002e409000db
:102e0000614060004201dd00512c200091407800bb
:102e1000b0cfb30000c0600002407000c5e2b70050
:102e2000a90037001e009000e10f50000f0036008f
:102e3000c5c2bf000080fb004500de000080fb0033
:102e4000610060000000a200614060004501dd00fb
:102e5000512c200091407800f0cdb30000c06000fc
:102e600002407000c5e2b700970037002e40900086
:102e7000614060004501dd00512c20009140780048
:102e8000f0cdb30000c0600002407000c5e2b700a2
:102e90008d0037001e009000e10f50000f0036003b
:102ea000c5c2bf000080fb004600de000080fb00c2
:102eb000610060000000a200614060004601dd008a
:102ec000512c200091407800f0cbb30000c060008e
:102ed00002407000c5e2b7007b0037002e40900032
:102ee000614060004601dd00512c200091407800d7
:102ef000f0cbb30000c0600002407000c5e2b70034
:102f0000710037001e009000e10f50000b003600ea
:102f1000c5c2bf000080fb004700de000080fb0050
:102f20000000a200c700dd00c5c2bf000074a10000
:102f300001407000c5e2b700630037002e409000ea
:102f4000c700dd00c5c2bf000074a10001407000d1
:102f5000c5e2b7005c0037002e409000c700dd00de
:102f6000c5c2bf000074a10001407000c5e2b700f7
:102f7000c5c2bf000080fb004700de000080fb00f0
:102f8000614060004601dd00512c20009140780036
:102f9000f0cbb30000c0600002407000c5e2b70093
:102fa000c5c2bf000080fb004600de000080fb00c1
:102fb00061006000614060004501dd00512c20008f
:102fc00091407800f0cdb30000c060000240700076
:102fd000c5e2b700c5c2bf000080fb004500de00af
:102fe0000080fb0061006000614060004201dd0084
:102ff000512c200091407800b0cfb30000c0600099
:1030000002407000c5e2b700c5c2bf000080fb00ef
:103010004200de000080fb00610060006140600053
:103020004401dd00512c200091407800f0ceb30027
:1030300000c0600002407000c5e2b700c5c2bf001a
:103040000080fb004400de000080fb0061006000a7
:10305000614060000041d000512c20009140780078
:10306000d0cfb30000c0600002407000c5e2b700de
:10307000c5c2bf000080fb000000d1000080fb0043
:1030800061006000c700dd00c4c2bf000074a10081
:1030900001407000c4e2b700c4c2bf000080fb0062
:1030a0004700de000080fb00614060004601dd005b
:1030b000412c200091407800f0cbb30000c06000ac
:1030c00002407000c4e2b7000080fa000000060071
:1030d0000000fa00c4c2a900c4e2a900c522a900e8
:1030e000c582a900c542a900c5a2a900c5c2a90000
:1030f000c5e2a9000080fa00000006000200fa0004
:10310000000f7800100020009e0f10000f00360006
:10311000d0c2bf000080fb004200de000080fb0048
:10312000610060000000a200614060004201dd001b
:10313000012d200091407800b0cfb30000c06000a6
:1031400002407000d0e2b700090037009e407800ce
:1031500061c060004201dd00012d20009140780037
:10316000b0cfb30000c0600002407000d0e2b700f2
:103170000080fa00000006000200fa00000f78004c
:10318000100020009e0f10000f003600d0c2bf00bc
:103190000080fb000000d1000080fb0061006000a7
:1031a0000000a200614060000041d000012d20001d
:1031b00091407800d0cfb30000c0600002407000a2
:1031c000d0e2b700090037009e40780061c060007f
:1031d0000041d000012d200091407800d0cfb300f5
:1031e00000c0600002407000d0e2b7000080fa002a
:1031f000000006000000fa00c4c2bf000080fb000f
:103200004600de000080fb00610060000080ea00f4
:10321000614060004601dd00412c200091407800b3
:10322000f0cbb30000c0600002407000c4e2b70001
:10323000c4c2bf000080fb004700de000080fb002e
:103240000080ea00c700dd00c4c2bf000074a10016
:1032500001407000c4e2b700c5c2bf000080fb009f
:103260000000d1000080fb00610060000080ea00e7
:10327000614060000041d000512c20009140780056
:10328000d0cfb30000c0600002407000c5e2b700bc
:10329000c5c2bf000080fb004400de000080fb00d0
:1032a000610060000080ea00614060004401dd00d0
:1032b000512c200091407800f0ceb30000c0600097
:1032c00002407000c5e2b700c5c2bf000080fb002d
:1032d0004200de000080fb00610060000080ea0028
:1032e000614060004201dd00512c200091407800d7
:1032f000b0cfb30000c0600002407000c5e2b7006c
:10330000c5c2bf000080fb004500de000080fb005e
:10331000610060000080ea00614060004501dd005e
:10332000512c200091407800f0cdb30000c0600027
:1033300002407000c5e2b700c5c2bf000080fb00bc
:103340004600de000080fb00610060000080ea00b3
:10335000614060004601dd00512c20009140780062
:10336000f0cbb30000c0600002407000c5e2b700bf
:10337000c5c2bf000080fb004700de000080fb00ec
:103380000080ea00c700dd00c5c2bf000074a100d4
:1033900001407000c5e2b7000080fa00000006009e
:1033a0000000fa00c4c2bf000080fb004600de003f
:1033b0000080fb00610060000080ea006140600066
:1033c0004601dd00412c200091407800f0cbb30095
:1033d00000c0600002407000c4e2b7000080fa0044
:1033e000000006000000fa00c4c2bf000080fb001d
:1033f0004700de000080fb000080ea00c700dd001f
:10340000c4c2bf000074a10001407000c4e2b70054
:103410000080fa00000006000000fa00c5c2bf00ec
:103420000080fb000000d1000080fb006100600014
:103430000080ea00614060000041d000512c200073
:1034400091407800d0cfb30000c06000024070000f
:10345000c5e2b7000080fa00000006000000fa0094
:10346000c5c2bf000080fb004400de000080fb00fe
:10347000610060000080ea00614060004401dd00fe
:10348000512c200091407800f0ceb30000c06000c5
:1034900002407000c5e2b7000080fa00000006009c
:1034a0000000fa00c5c2bf000080fb004200de0041
:1034b0000080fb00610060000080ea006140600065
:1034c0004201dd00512c200091407800b0cfb300c4
:1034d00000c0600002407000c5e2b7000080fa0042
:1034e000000006000000fa00c5c2bf000080fb001b
:1034f0004500de000080fb00610060000080ea0003
:10350000614060004501dd00512c200091407800b1
:10351000f0cdb30000c0600002407000c5e2b7000b
:103520000080fa00000006000000fa00c5c2bf00db
:103530000080fb004600de000080fb0061006000b0
:103540000080ea00614060004601dd00512c20004f
:1035500091407800f0cbb30000c0600002407000e2
:10356000c5e2b7000080fa00000006000000fa0083
:10357000c5c2bf000080fb004700de000080fb00ea
:103580000080ea00c700dd00c5c2bf000074a100d2
:1035900001407000c5e2b7000080fa00000006009c
:1035a0000200fa00000f78009e007800a08f210032
:1035b00088fc07000080fa00000006000000fa0006
:1035c000a08f2100b4fc07000080fa000000060074
:1035d0000200fa00000f78001e00e0000300350032
:1035e0009e007800a08f2100d3fc07000080fa0025
:1035f000000006000000fa00e0cf20001004e00008
:103600000a003a008000eb007000200061fd070016
:10361000e0cf20001080fb00110020005dfd0700be
:10362000e0cf20001048e8001c003700e0cf200069
:1036300071c0b30090cf10000d003a00e0cf200021
:103640001080fb000000e9008000eb0051fd070046
:10365000e0cf20001080fb00110020004dfd07008e
:10366000e1cf20000040eb00804878000b003700dd
:10367000e0cf20001080fb000000e9008000eb009c
:1036800044fd0700e0cf20001080fb001100200067
:1036900040fd0700e0cf20001048e8000080fa005d
:1036a000000006000200fa00f0cf20001080fb00ae
:1036b000000f78001e007800e20f50001c0032005e
:1036c0009e007800e28f500007003c001e0078004a
:1036d0000000e0000b0032009e007800e18f5000f7
:1036e0000c003200230037001e007800e30f50006a
:1036f000160032009e007800e48f50001a0032005d
:103700001c003700210020000000eb0021fd070015
:103710001800370021002000100020001dfd0700c8
:1037200021002000700020001afd07001100370062
:10373000210020002000200016fd070021002000ad
:103740006000200013fd07000a0037002100200060
:10375000300020000ffd0700210020005000200055
:103760000cfd07000300370021002000400020006e
:1037700008fd0700f0cf200031c0b30090cf10004b
:1037800003003e00f0cf20001048e800030037009f
:10379000f1cf20000040eb00804878000080fa0064
:1037a000000006000000fa0000d020001004e00035
:1037b00011003a00a0d020001004e0000e003200fa
:1037c00001d0200010c0b300804878008000eb00da
:1037d0000000eb00effc070000d020001080fb0091
:1037e00011002000ebfc0700a1d020000040eb00fe
:1037f000804878003100370000d020001004e0003d
:1038000011003a00a0d020001004e0000e003a00a1
:1038100001d0200070c0b300804878008000eb0029
:103820000000eb00dbfc070000d020001080fb0054
:1038300011002000d7fc0700a1d0200010c0b30069
:10384000804878001d00370000d0200071c0b30010
:1038500090cf10000b003a0001d020000040eb0098
:10386000804878008000eb0070002000c9fc070051
:1038700000d020001080fb0011002000c5fc0700d4
:103880000e00370000d0200011c0b30090cf100010
:103890000a003a0001d020000040eb008048780088
:1038a0008000eb0010002000bafc070000d02000d0
:1038b0001080fb0011002000b6fc07000080fa0019
:1038c000000006000200fa0010d020001080fb006b
:1038d000000f78001e007800e10f50001500320044
:1038e0009e007800e18f500004003c001e0078002c
:1038f0000000e000080032001a0037009e00780047
:10390000e28f5000120032001e007800e30f5000da
:103910001300320013003700210020000000eb00ec
:103920009cfc0700210020004000200099fc0700bb
:103930000c003700210020001000200095fc07003b
:10394000210020003000200092fc07000500370015
:1039500021002000200020008efc0700010037001d
:10396000dbfd070010d0200021c0b30090cf100075
:1039700003003e0010d020001048e800030037008c
:1039800011d020000040eb00804878000080fa0051
:10399000000006000200fa0020d020001080fb008a
:1039a000000f78001e007800e10f50001500320073
:1039b0009e007800e18f500004003c001e0078005b
:1039c0000000e000080032001a0037009e00780076
:1039d000e28f5000120032001e007800e30f50000a
:1039e0001300320013003700210020000000eb001c
:1039f00068fc0700210020004000200065fc070053
:103a00000c003700210020007000200061fc07003e
:103a100021002000500020005efc07000500370058
:103a200021002000600020005afc07000100370040
:103a3000a7fd070020d0200021c0b30090cf1000c8
:103a400003003e0020d020001048e80003003700ab
:103a500021d020000040eb00804878000080fa0070
:103a6000000006000600fa00889fbe008a9fbe0084
:103a70000000eb0080658800510037008065800001
:103a800021cb200000004000000040000101400068
:103a90006000b8000089be000000eb00706588007f
:103aa0001e0037008b6580008065800021cb2000e0
:103ab0000000400000004000010040001004be0073
:103ac0008065800071658000c2c820000000400051
:103ad00000004000000040000100400000004000e5
:103ae0006005790070658000f3f9070000d0b90027
:103af000cf80de00080140008981480021cb2000f2
:103b00000b80450000004000010040000288be001c
:103b1000706580000000e8007065880070658000b6
:103b2000e70f5000dfff340080658000000f780051
:103b30008065800021cb2000000040000000400094
:103b4000010040001000be001007980021079800f7
:103b50001e019000ae019000e00f5100e08f59006f
:103b600006003d001e009000ae0090006300400083
:103b7000e080480010079800210798001e0190007f
:103b8000ae0190004e1add004210de00000072000f
:103b9000c298de0062222000000141001e00780071
:103ba0001e00780080004000a0cb20000080400074
:103bb00002087800806580000000e80080658800c9
:103bc00080658000e10f5000acff3400e1658000ab
:103bd00010032000808f500012003c00e16580003f
:103be000e0fc2f00808f50000e003400d165800073
:103bf00010032000808f50000a003c00d165800037
:103c0000e0fc2f00808f500006003400e06580004b
:103c10007400b900e0658800d06580007400b900c8
:103c2000d0658800e1658000803e2000808f5000d4
:103c300003003400803e2000e06588000600370065
:103c4000e165800080c12f00808f500002003d00a0
:103c500080c12f00e0658800d1658000803e200093
:103c6000808f500003003400803e2000d065880023
:103c700006003700d165800080c12f00808f500082
:103c800002003d0080c12f00d0658800e065800003
:103c9000faf40700d065800035f507004f05be0037
:103ca0004f04be000080fa00000006001000fa0079
:103cb000889fbe008a9fbe00600798007107980029
:103cc0004006200050079800d0cc2c00c1d423001f
:103cd0003007980041079800300020002007980026
:103ce000de0090006e0090000080500010079800e9
:103cf00050638000cf80de0072f207000005be0036
:103d00001e009000cf80de006ef207003e019000a2
:103d1000ce019000f9f207000004be002e009000d2
:103d2000cf80de0067f207000001be000800be0081
:103d30008ff207000001be000a00be0024f3070056
:103d4000cdf2070050638800516380001e00900090
:103d5000808040007e0090000088b900000f78004d
:103d6000703e20009e0f100011003400703e2000b5
:103d70007e019000110009000200d8008000780048
:103d80001e00900000805000506388005163800046
:103d9000c0032000808f500002003400c0032000c8
:103da00050638800703e2000000f7800120037003a
:103db00080c12f009e0f10000f003c0090c12f000b
:103dc0007e019000110009000200d80080007800f8
:103dd0001e00900000804000506388005063800007
:103de000ea0f400002003d0060ff2f005063880092
:103df00090c12f00000f78001e0078004f05be0014
:103e00004f04be000080fa00000006000a00fa001d
:103e100030079800410798000000eb002007980049
:103e20000000eb0010079800ae0090003e009000ec
:103e3000008f50009e0078004e0090000088b9006e
:103e4000100798009e009000703e2000808f500068
:103e500003003400703e2000100798000600370071
:103e60009e00900080c12f00808f500002003c0017
:103e700090c12f00100798001e0090000080fa00eb
:103e8000000006000400fa00889fbe0070002000b9
:103e900009f90700000478000000eb0006f90700ac
:103ea000800044004f08de00010040000080d10087
:103eb000610020007dff0700100798000000eb0064
:103ec000fdf807000004780010002000faf8070051
:103ed0008004440070002000f7f807000004780018
:103ee00060002000f4f80700000044000080540047
:103ef00041002000c5ff0700000f78001e00900061
:103f00001e0050005df407001e0090001e004000df
:103f100097f407004f04be000080fa00000006007e
:103f20000000fa0004f507004bf407000040eb0026
:103f30008df5070062f80700419c200020bd21009c
:103f400024fa0700a128200020f4210021fa07000c
:103f50000bfa0700ffff37000000fa00f6f4070035
:103f60003df407000040eb007ff5070054f8070020
:103f70004138200020b5210016fa0700a1282000b2
:103f800020d3210013fa0700fdf90700ffff3700d7
:103f90000000fa00d1d0200010c0b30080487800a3
:103fa0000080fa00000006000000fa00e0d02000c7
:103fb000104078008040e800e0d020000148780000
:103fc000e0d0200010407800e14f5000090036009a
:103fd000e1d020000040eb0080487800adf90700f8
:103fe00040fd21002cfa0700c1d020000040eb006a
:103ff000804878000080fa00000006000600fa0001
:104000000040eb00004f780013f4070040c7bf00ea
:10401000614060000004e000020032004007a90097
:104020000000fe000153270080fc2100e9f9070091
:10403000000037000000eb0030fc07000000eb0040
:104040004dfc07000000eb00b0f70700fe0f50002a
:1040500008003c0010002000acf70700fe0f5000e5
:1040600004003c0020002000a8f70700fe0f5000cd
:10407000040034001000200020fc07001000200085
:104080003dfc07000000eb0075f807008000780099
:1040900000192000808f50000100340055fc0700fb
:1040a000100020006ef80700800078000032200029
:1040b000808f50000c0034002000200068f80700ba
:1040c0008000780000322000808f5000060034000d
:1040d0003000200062f807008000780000322000e5
:1040e000808f500006003c000000eb0087f70700bf
:1040f00080007800e0152000808f50000e00340012
:10410000c0d02000104078000004e0000a003a000f
:1041100049f90700c1d0200010c0b30080487800e2
:10412000415927000000eb0050f907000153270018
:1041300040fd2100a7f90700d0d0200010407800f2
:104140000004e000bbff3200d1d020000040eb00b3
:10415000804878001e80fb006101b90012079800ba
:104160002307980090002000010020001e0190000d
:10417000ae019000800f5100818f590045003e0034
:104180001e009000ae0090000060010009003700a2
:104190000d00370012003700170037001c003700f1
:1041a00021003700270037002b0037002f00370091
:1041b0003300370001fd07004138200020b5210001
:1041c00084f907003300370020b52100b2f9070059
:1041d00001322000a0af21007ef907002d0037003a
:1041e000a0af2100acf90700017d200020c621000e
:1041f00078f907002700370020c62100a6f907003c
:10420000419c200020bd210072f9070021003700e9
:1042100020bd2100a0f90700017d2000a0cc2100d5
:104220006cf907001b003700a0cc21009af90700a9
:10423000800c200091f3070080f32f00ccf30700df
:104240001400370080f32f008cf30700800c20004f
:10425000c7f307000f00370080f32f0087f3070034
:10426000800c2000c2f307000a003700800c2000f9
:1042700082f3070080f32f00bdf30700050037002d
:104280008000eb000000eb00f6f30700a00f200019
:10429000c3fc070081c0b3009ecf100002003e00a7
:1042a0001e4fe80063ff37000040eb00004f78002e
:0442b00060ff370074
:020000040000fa
:0200000401f009
:04000000e6ff000017
:020000040000fa
:0200000401f009
:04000400ff7f00007a
:020000040000fa
:0200000401f009
:040008007fff000076
:020000040000fa
:0200000401f009
:04001400ffff0000ea
:020000040000fa
:10000800320d0100320d0100320d0100320d0100e8
:10001800320d0100320d0100320d0100320d0100d8
:10002800320d0100320d0100320d0100320d0100c8
:10003800320d0100320d01006e150000320d010075
:10004800320d0100320d0100320d0100880b000055
:10005800320d0100320d0100320d0100320d010098
:10006800320d0100320d0100320d0100320d010088
:10007800320d0100320d0100320d0100320d010078
:10008800320d0100320d0100320d0100320d010068
:10009800320d0100320d0100320d0100320d010058
:1000a800320d0100320d0100320d0100320d010048
:1000b800320d0100320d0100320d0100320d010038
:1000c800320d0100ae120000320d0100320d0100a8
:1000d800320d0100320d0100320d0100320d010018
:1000e800320d0100320d0100320d0100320d010008
:0800f800320d0100320d010080
:020000040000fa
:10010800320d0100320d0100320d0100320d0100e7
:10011800320d0100320d0100320d0100320d0100d7
:10012800320d0100320d0100320d0100320d0100c7
:10013800320d0100320d01006e150000320d010074
:10014800320d0100320d0100320d0100880b000054
:10015800320d0100320d0100320d0100320d010097
:10016800320d0100320d0100320d0100320d010087
:10017800320d0100320d0100320d0100320d010077
:10018800320d0100320d0100320d0100320d010067
:10019800320d0100320d0100320d0100320d010057
:1001a800320d0100320d0100320d0100320d010047
:1001b800320d0100320d0100320d0100320d010037
:1001c800320d0100ae120000320d0100320d0100a7
:1001d800320d0100320d0100320d0100320d010017
:1001e800320d0100320d0100320d0100320d010007
:0801f800320d0100320d01007f
:020000040000fa
:1042b40020fb0000abf2000008fd0000b01000007d
:1042c400050a0000befb000007fa00009702000088
:1042d400e60a0000a308000062110000bd0500000a
:1042e40057f800000b020000a9ee000081f900005d
:1042f4009405000094f60000d2ff0000bef900000f
:10430400df03000044fe00004fed000008f0000051
:10431400e2e000009cf30000ebf8000060f700000e
:1043240093090000dcf7000083fb0000c3110000c8
:10433400e319000069210000431b0000e818000095
:104344000c100000210c0000b21a0000400e000006
:10435400240f0000a50600008bf5000016040000e1
:10436400a3f800009dfd00001cfc0000b5ee000059
:10437400eeee000063e900007cf2000003e40000bc
:104384004eed0000d0e8000015d70000aded0000b0
:104394007fea000028f0000088f30000aef6000079
:1043a400cff10000ecfd00001f16000043010000e7
:1043b40049110000b71700003d120000541300001b
:1043c4009d1700008a1e0000aa1200005921000057
:1043d4007f080000a90200001e1800009f0e0000c4
:1043e400291c0000f21b0000e10b000003ff000089
:1043f400560500006e090000dbfa00006aff0000a9
:10440400a7f40000c8e00000a1e300007fde000084
:104414000ee3000082ea00004ded0000bded000057
:1044240048e90000eef100002df0000012fe00004b
:10443400c5f000007cdf0000e6ef000089f4000016
:1044440087fb0000fdfb00008b05000076f50000f3
:1044540080fd000074140000bf1c000068280000e8
:104464000616000096180000680e0000a31c000049
:104474004f1e0000e1160000d22a00001d090000b2
:10448400d70e0000a21a000067140000161a0000dc
:1044940079080000b2fc000075ef0000f6f200009d
:1044a400f4f300007ce1000049e60000b3dd000005
:1044b40093d900003be60000f7dc0000c1e50000f2
:1044c400d7e30000f9d6000088de000094f0000075
:1044d400b7f800001bf400006d08000002020000a1
:1044e40078f3000013080000461600006a1a000062
:1044f400071e0000ab180000b219000040230000a2
:10450400d82400009e290000cb240000dc220000f7
:10451400920c0000c2060000c5130000f000000069
:10452400ff05000040f80000e8ec000068ec000023
:1045340081ea0000e6f00000c0ec00001dfd000070
:10454400cbeb0000e1e60000e2ef0000e0e4000055
:1045540017ea000034de000093db0000bce3000037
:1045640082eb000022f10000cefc0000f80c0000f9
:10457400fb0c0000fb100000d61200000b20000012
:1045840085280000eb1e0000661500005410000092
:104594004d1600005f060000d40900004417000017
:1045a40060000000dffd000096010000ac06000082
:1045b400f20e00006f05000023fb000093f10000e1
:1045c400dced0000e6ea0000cfe50000c8eb0000e7
:1045d40078ea00002de2000015ef0000b0ee0000c4
:1045e4005cf80000630500005df5000016fb0000a8
:1045f400ebf9000022050000ea0e00000b0a00009f
:10460400b40e0000edf80000d8060000f810000019
:104614002b0d0000551d0000900300001a07000038
:10462400ef100000dd0c0000fc1a0000720f000007
:10463400ce140000c0fd0000c1f100003d020000e6
:1046440077f600002809000060f70000eeeb000098
:1046540074f50000e7e800007df50000ccf90000e7
:104664006ffe0000ebf1000071ee0000f2fc0000b0
:1046740051ec0000e0ee00003af3000012df00000d
:1046840001e9000013f3000003fc000063060000ce
:10469400f50200005d160000b80a00002e110000ab
:1046a40034180000981000000f200000520500008c
:1046b400a20d0000a90f00008d0a0000461800009a
:1046c400851600000b170000dc0300002d1300000a
:1046d4003d140000dd090000280d0000d8fc000096
:1046e4006ef3000003ea0000ade8000079e7000083
:1046f40089eb000024ed00006ae30000a8e100005b
:10470400c0e5000016e8000056f30000f7f60000cc
:1047140023eb0000f0f10000efef000041ef000098
:10472400cdf9000035fb000080f90000b6fd000063
:10473400970c0000c00f000004210000c7260000f1
:10474400561a0000471f0000ee1d00004e23000013
:10475400d8220000f71b0000ef100000a1030000a6
:104764003005000005050000d3080000f103000037
:1047740071ee0000e7e60000b3e900008ee90000f6
:1047840048f900002cfc000096f3000007ef00003d
:104794007fe700005be80000e3e70000caf20000e6
:1047a40094e800001ae3000086f200003af90000e1
:1047b400e2050000c0080000fb0c0000ed0a000048
:1047c400a7150000be180000f5140000021d00002b
:1047d4007d0c0000b0070000db0a0000af0b0000f6
:1047e400f80a0000920b0000daff000021f8000034
:1047f40027010000ddfe0000e3040000db020000ee
:1048040058fa0000a8e2000007e60000feee0000ef
:104814006fe600003e01000014f7000021f40000e0
:10482400e5fd00008ffd0000bb060000480200000b
:104834000b0600000ef80000bcfc0000630400003e
:10484400ceff0000e80e000083090000050400000c
:10485400cc0a00000d09000010090000a90c00009a
:10486400390a0000950a00002a040000f70d000030
:104874003d0f00004afd000004030000d2ec0000dc
:104884008ced000012010000a6f900008909000067
:10489400f4fe00009bf300000cfa00008eee000012
:1048a400c1fd00008afa00003efd0000bf080000c0
:1048b40045e6000034f400009af000003ee60000f3
:1048c400f201000039eb0000e7f1000084fa000077
:1048d40035000000fb160000de070000461900004a
:1048e400791a0000f80b0000c61800004a0a0000fc
:1048f40070160000a20a000074f60000eb09000024
:10490400c7f80000db0400000b0b0000960c00004d
:104914004e11000043fe0000df1500006305000097
:10492400abfb0000f0fd00004ae5000037f2000098
:104934003cea0000d4ed000047fa0000ddeb000083
:104944008ceb0000d3ec000050ef0000a5f7000052
:1049540048fd0000c4fa00000cf4000076ea0000f0
:1049640073f100007dfa0000daf80000940a0000f8
:104974001e070000af08000077150000aa0c000015
:104984000d1c000058190000bd0a0000321200007e
:10499400d41300009e150000f6110000b9120000a7
:1049a400f0080000a2f70000400500005c040000cd
:1049b40017ff0000a603000070ee00000df10000d8
:1049c400a7f40000cef40000fbff0000dafb0000b7
:1049d400c1fe000007e9000073e80000fff40000d6
:1049e40044e900007ffa0000e3f300003fe900001f
:1049f40058fd00001afe0000d60b0000461000000f
:104a04000b06000072110000a7fe00009b0a0000c4
:104a1400f70a0000d2ff0000c31a00009df900004d
:104a2400de080000b50f000046fe0000100d000077
:104a3400edfd0000eb02000055f30000bf01000093
:104a44004d00000076f5000047fa00006ce100001c
:104a54007ef60000c1f10000fefa00002a01000009
:104a64007c010000f00900005ff60000b00f0000b8
:104a74002e05000076030000be0b000029f600009e
:104a8400e4fa0000cdfb0000ac050000280600009d
:104a9400830800004b0a00008f0300000a05000091
:104aa400210300007105000022060000310500000a
:104ab40043fc0000f40000009e02000064fb0000c0
:104ac4000fff0000d1f9000021fc0000d1fe00001e
:104ad4008bff0000a7020000000600006ef9000032
:104ae4003ff200009dfe0000a2f500007cfa0000e9
:104af400acf8000024f90000aff80000b1ea0000af
:104b0400b901000075fa00002bfb00003cfd000019
:104b1400b2ee0000640100008cff0000110d0000e3
:104b2400d61000002e0f00000213000065050000df
:104b3400211300007e0300004d050000b81600009c
:104b440026fe0000ad080000170e0000540300000c
:104b5400040e0000610600004008000020fe000072
:104b64004cf10000c805000066f4000066f7000080
:104b740016f200001be200000c0300003bee0000f4
:104b8400ebf900003c010000a8ed0000410000002a
:104b940005ea00001cf7000024f20000eaf200001d
:104ba40064fd000030e300008902000071ff000092
:104bb40036050000eb0d000048070000800f0000e0
:104bc4001e0600006b130000ea0800000411000038
:104bd400340a0000600100001c100000320a0000ca
:104be400d1120000020a0000a71100008e07000085
:104bf400c30600007006000055f50000c906000059
:104c040095f4000031f40000a2f30000fbf300006f
:104c140076fc0000adf200005e0400003af20000f1
:104c2400e1ee000014fb00007ced000037fb000007
:104c3400b1f9000003f60000e2f500004bf90000b2
:104c44003c0a000026040000290a00006f07000047
:104c54002a0000007b08000024030000310a000041
:104c640089130000c4080000d7ff0000540a0000a4
:104c74003100000063f9000016010000cbfc0000c5
:104c840007f80000edf60000010700002bfb000010
:104c940093fb000063fd000053ef0000c7fc00001d
:104ca40014fa0000bb00000088050000890300001e
:104cb40021fe0000e6ff0000d40600008dfb00008a
:104cc40009080000ba060000b5fb0000b4fc0000af
:104cd4000c0600004a0700000d01000052130000fa
:104ce400770100003dfd000000090000dcf8000031
:104cf40019010000eef80000faff00005003000064
:104d040072fa0000c007000096fd00004f0b00007f
:104d140096030000e4f400005a0100007df700004f
:104d24008cf5000076fb0000f4f7000017ed00009e
:104d340073f700006dfb0000bc030000c204000018
:104d4400c90000002306000083f600006903000088
:104d5400b7f6000030f90000e300000004eb0000a7
:104d6400fbfe0000de0000000a0a00009a140000a6
:104d74008612000090130000440800005b0d000040
:104d840009090000680c000048160000e602000053
:104d9400a6020000ca04000023fb0000a5fc0000da
:104da40000fb0000cbf8000045f00000ebf700002a
:104db400ebf40000b3f700006c01000002f2000005
:104dc40010f6000045f500000bfa00009bf9000006
:104dd400deff0000c0020000d7f700007efe0000e6
:104de4007cf5000072fe00008a060000f901000054
:104df400acf900008ffc0000a10500009a0200003d
:104e0400e00700006d010000db000000f10000007d
:104e140052050000e004000029070000a00c000077
:104e2400ad020000d5070000d2040000080600000f
:104e34003909000026050000ecff00008bfa000091
:104e4400760400001bfc0000f6f90000c204000018
:104e5400c9f40000c6f80000de040000530100009d
:104e64009c0700003d0500002f060000a2f9000089
:104e740032f600004bff000025f5000030fd000075
:104e8400c5f40000b6f20000e60100005401000081
:104e9400b90500003909000062090000b1020000f0
:104ea400270000003bfe00006afd0000d8fe000061
:104eb4002afc000080f5000084f500008701000052
:104ec400ccfb00007a01000081000000f0f3000038
:104ed40091ff000061f900004a000000fc0100009d
:104ee400bcf300006a000000c5fa000005060000db
:104ef400ce0b00003eff000044150000720c0000c1
:104f0400e9070000680e0000cd0400005014000002
:104f1400630700004efe00000507000027fb0000a9
:104f24000c050000b102000062fb00001afd000045
:104f34003df000006bfc000089fd00000ff500004f
:104f440068ff00007df900006cf90000cbf8000058
:104f5400f4f9000008ff00007ef800006cfc00007b
:104f6400f3f600004ef70000bff60000f9fa000067
:104f7400920a0000d9fa0000ccfb00004f060000a2
:104f8400f20700009708000029050000e30800006c
:104f9400f7000000e8fb000037000000f203000007
:104fa4008a000000cbfc000093fb00003c050000dd
:104fb400cc0800001b05000017120000d8070000f1
:104fc40042030000d3070000dc020000f2020000ec
:104fd400d50200003407000006fe000005f90000b9
:104fe4000bfe0000c1fb00001cfb0000e1fc000004
:104ff40009f6000034fc00004efc000016f400002a
:10500400b8fd00004af50000d7f30000a7fa00003d
:10501400b0050000af010000f1fc0000da0c000054
:105024001ffd00000cfd0000f2fc00003efe00002d
:105034008506000077fe0000d7000000e3fb0000b7
:105044006604000023030000fa010000fb0a0000cc
:105054007dfd0000f1f8000069020000d2000000ac
:105064007dfc0000f104000066fe0000dafe000092
:105074009e0300001c0100002bff00001dfe000029
:105084009a0800001ef9000062fc000045050000bb
:10509400e7fa000058050000eeff000021fb0000c5
:1050a400a9030000d70a0000540600007a04000097
:1050b4007d09000037ff00002f060000650700008f
:1050c400dcfc00009bfe00004bfd0000d6fa000053
:1050d400a4f70000840400005e0400002f01000017
:1050e400de0a000096fd000073fd000078fb00005e
:1050f4000efb000056f600006ff5000037fa0000c2
:105104007aec00002f01000080f30000a2f20000fe
:1051140056010000c9f500001400000001fb000066
:10512400b1030000f8f8000009fe000008020000c6
:1051340059fb0000c90a0000ff0800000a0e000025
:10514400dc0900007d11000015040000ae0f000012
:105154000c1400005a03000056120000e400000082
:105164001604000030fa0000660200004c02000041
:10517400f1f10000f305000091f3000085f7000051
:10518400a5fc0000ebf9000037fb00004af4000026
:1051940029fe000098f800003600000090fd000091
:1051a40044f70000400300007af400000ef8000009
:1051b4003b010000d8fc000078fe00000c03000056
:1051c400c1050000bfff0000690800003e070000a1
:1051d4009603000018fb0000a8ff000016fd000065
:1051e40070f800004b0a0000b6f1000066030000ee
:1051f400bd000000b3fe000081130000a504000000
:105204001518000066010000cf0a0000c303000067
:105214005af50000b60f000005f800002205000052
:10522400c0fd0000e8fe0000d30500006ff600009a
:105234002400000093f100004cff0000c4fd0000b6
:10524400f0f40000f301000071f300002bf80000fb
:105254009af2000000f6000011f80000f5f60000d4
:10526400a30c0000f9fa00000f090000ea02000094
:10527400170300005a110000dcf700008c11000035
:105284009afc0000d2000000ee04000094f7000035
:10529400f41000009bf90000e0060000f702000093
:1052a40021ff0000e10200006cfc0000110100007d
:1052b4008df60000e7fd000044f80000c002000085
:1052c400e2fb0000e3fa0000ccf900005cf6000009
:1052d400430500003dfd00004d0c0000ad02000040
:1052e4001e060000f80a000063ff00002d05000000
:1052f4007e070000101000000f0400005d0700008e
:1053040085050000bf0100007004000024fc0000bb
:105314003bfe0000b8f6000047fa00007afd0000ea
:10532400dbf900007903000069fd00003df3000093
:105334005af800008ef3000051f5000073f80000e5
:105344001cf80000aef60000bdf10000f6fc000001
:1053540097f900002ffe00006d030000aaf9000079
:10536400e6030000390400008d030000eb0900008f
:10537400c002000053080000b50a00008d0b0000b5
:10538400300f000073060000851100008206000043
:105394004e0600007a0e000055060000300c000096
:1053a400dafc0000520a000068fd0000e8f3000087
:1053b40066010000bff100000c00000018f50000b9
:1053c40017f4000087f8000075f00000e9fa000007
:1053d40013f80000def6000082f40000c8fb0000b1
:1053e400950100001bfb0000e9f900001803000010
:1053f400b9fe000044fa000069070000c20400007e
:105404008c010000610800001304000089fd000005
:105414005e0400008d040000040d0000400b000039
:10542400950100000f060000abfd0000bbfe00006c
:10543400daf90000a0fd000058030000cdfc0000d4
:10544400c1ff0000460400004d01000004ff0000fd
:105454008f0c00008cfa0000ecfe000084020000b7
:10546400f5f600001c050000d5f800006d000000f2
:10547400fdf6000036f400000ffe0000b1fb000052
:105484008a0800001b0100002a020000ef0000004f
:10549400d50400008afa0000a00200006d06000096
:1054a400c5f900008a0f000090fe0000d307000039
:1054b400790a0000b5030000060b0000c3fc0000dd
:1054c4004405000057f800001bfb000051fc0000dd
:1054d400b1f30000d3fc00005cfb00005cf70000ab
:1054e400b3f40000aafe00002ef60000d3f800007a
:1054f400bbfa0000aff20000dbf9000031f5000058
:10550400ef0000001b030000840400006cfe000098
:10551400a5fa0000ab0d00005bfb00006206000072
:10552400b10c0000c7090000ed1100002a000000c2
:1055340020140000a20600009b0e0000dc190000ed
:1055440032fb0000e610000091020000dd010000c3
:1055540047090000dff6000057f90000b5f6000027
:1055640045f80000fcf800000eff000020fa0000df
:10557400f0ff0000d7f5000037fc00004ff80000f2
:10558400b8e400004f04000026ed000055fc0000c4
:10559400dffe0000bcf300008f050000bdf000003a
:1055a400af030000bbef00007f050000f103000023
:1055b400baf100002c0f00003bf20000ea0c0000de
:1055c40096020000a604000095130000b00000003d
:1055d400341a000021020000611200008913000047
:1055e4004d00000047140000e10000001403000017
:1055f400a7ff00004efa000076fa0000b4f10000a4
:1056040097fa00002af30000daf500000a0100000e
:1056140057fd000097fa0000b8f80000e1f9000017
:105624009ef7000087fc00000b00000084fb0000d4
:105634000b07000024fd0000e3fc0000d10900007a
:10564400d3fa00009b0400008f000000a8040000af
:10565400b80800007bfd0000780e0000ad050000d6
:10566400800b0000cd040000b9f70000ae0000007c
:10567400bbfb00009afc000075fd000067fc000005
:1056840077f80000d7fd00002cf80000dd010000d1
:10569400840000005e030000a2000000ccf60000bd
:1056a400150700005af20000fe0a000013f700007c
:1056b400620100006f0a00004bea0000db140000e6
:1056c4005fef0000410f00006e000000a4f3000033
:1056d400ad1b0000bcea00002c11000091f9000091
:1056e40098f900007608000073f20000041200002c
:1056f4004d040000550b0000c307000072010000b8
:1057040021040000e901000049020000dbfd000063
:1057140089ff000020f700008704000079fc0000e6
:10572400e1f800004b04000039f800003ff90000e4
:1057340006f4000071f9000013f90000ebed00001d
:10574400a0f400002df3000077fd000069f80000cc
:10575400c3fd00009102000072fb0000140300006e
:105764002bfa00006e0f0000de080000db0f0000c3
:105774007a1200003402000085120000c00200000a
:1057840014130000780600009e0800007d0f00003e
:10579400c4010000180d000093fb0000380b00004a
:1057a4000cfc00006cfd0000a5ff0000e0f300000d
:1057b4005d0400006bf0000010040000a6f7000078
:1057c400a9ea0000e0f800004ce7000084fe0000b5
:1057d400dbf4000073f50000e502000009e70000b7
:1057e400edfe000047f800009cf60000c306000030
:1057f40067f300004a060000ebfa0000b3ff000064
:10580400250f00003f020000a40a0000320200003d
:10581400b909000044130000890c0000a91100001c
:105824003817000049090000620700004a0f000011
:10583400c20300009102000015fe00003afe0000c1
:105844000ef90000f0f2000053010000d9fa000044
:10585400cbf50000eaf700007ff30000a1f8000098
:10586400eaee00004df00000dff600007ef90000d3
:1058740093fc000086f60000d4060000ccf600007d
:10588400060400008d0a0000b0f70000350d00008a
:10589400f4030000f7160000d0060000fb09000026
:1058a400b111000075fe0000e91000005ff900006e
:1058b400680a0000baf8000047fd000053ff00002a
:1058c40070f10000180d000035e50000ff04000031
:1058d4000ef6000041f30000ad09000056ed000093
:1058e400f50f00001eec0000a9fe0000a9ff000057
:1058f40065ed0000a41200007af10000250b000001
:10590400b3fd0000effc0000b80e00002bf4000013
:10591400cc110000ff010000100c00006604000020
:10592400d5000000dd0e00003cf90000990a0000db
:105934006ef600004a0c000017040000bd010000d0
:10594400d90d0000e5f900002f1700003bf300001b
:10595400850a00006bf70000a2f100007d0a000038
:105964000ae30000251000005de5000082fe00004f
:10597400a5fe0000dbe30000351300006be100002e
:105984006d060000b9eb00000bef000008090000f1
:1059940061e40000690b000011f2000079060000c8
:1059a400d10200006701000061150000ab05000092
:1059b40084150000a4020000e11400005308000054
:1059c400060e0000f60d000070fe000062140000d8
:1059d40067fd0000670c000004fe00000b060000d9
:1059e4004005000024f800005602000027ec0000e7
:1059f40097090000e4f100001cf90000f0fe00002b
:105a040020f20000a9030000aae30000a9fc0000a2
:105a14004ff70000d4f8000018fe00008bf40000db
:105a2400dc06000086fa0000770100006ef7000033
:105a3400bb03000087f9000068fe0000d6070000e1
:105a4400e4f400005410000056f500005b08000068
:105a5400dc010000b2fe0000b51b0000e7fd000001
:105a640022180000990000001c0a000061060000d2
:105a740062fe0000c21a00002bf50000861100002f
:105a84008ef6000077ff0000f9ff000028e6000012
:105a9400e70f00007fe8000045070000e2f4000083
:105aa4001eef000053080000f4e300003905000075
:105ab4007eef00003fff000014fe000029f9000003
:105ac400a70b000078f20000e90a000007010000bb
:105ad400480a0000c80100008e050000610b0000a8
:105ae400290000009c15000017f600008811000032
:105af400f0ff00001ffc00004a0c000024ef00002f
:105b0400df0f00008cf1000077050000a4f900000d
:105b14009de50000ff0800004aec00009903000026
:105b2400e7f40000fffa0000f2060000bef60000f1
:105b3400550f000054040000b102000047fc0000af
:105b440033ff000032080000c601000076f90000af
:105b5400ca0800001a030000bff40000b30a0000e2
:105b6400c0f80000c009000041000000d602000097
:105b7400ba13000037f40000dc0d0000fbff000046
:105b84003a070000d10400006bf90000d7120000ae
:105b9400d9f900003c00000080fc000094ff0000e4
:105ba400eef90000a2f6000023070000e6f1000071
:105bb400c4f90000c1f600005bfd0000eef6000031
:105bc40036f10000adfa000012ef000021010000e0
:105bd400d6ed0000a5f800008c000000f6f20000ed
:105be400d60a00009ef70000f7030000320500000b
:105bf4007c060000f11200002dff000034140000a8
:105c04008c0b00002e0d0000021100006f03000039
:105c140021110000d60c0000d50c0000610b00001f
:105c2400d30a000055010000b3000000d8ff0000b3
:105c3400c0fd0000fefc00006bf50000b601000092
:105c4400c6f2000086f30000aaeb000030ef00006b
:105c54009df700005bee00007602000043f00000b8
:105c640083fd0000c9f70000b1ef000069040000e3
:105c740018f300009404000015fe0000300000003a
:105c84007e0300000ff800000d0c000084000000eb
:105c9400e507000095100000e1000000ae0c0000d4
:105ca400bc0d0000bb030000df0e00007b050000fc
:105cb4007f040000ef15000099020000de040000dc
:105cc40024040000d9fc00001f010000fdf50000c1
:105cd4001b040000adfa0000a1f5000075000000ef
:105ce4007df6000060f8000008f300006fef00008c
:105cf400fefa0000c5fa00004dee0000b2fd0000ff
:105d0400910300005c030000490400002e00000021
:105d1400820a000094fd0000ba090000e1040000ba
:105d2400b2f90000ef0200004dff0000a40a0000d9
:105d340049030000f90300006dff00009f0200000a
:105d4400d1050000a5020000b400000081f60000a7
:105d54009a040000e100000063fe0000f9f2000074
:105d640069fb0000e4fd0000fef5000090f5000072
:105d740064f40000471300002ffb0000730d0000c3
:105d8400630a0000b5f60000a60a0000e5f2000070
:105d9400e2100000660400002efd00000305000070
:105da4003dff0000e70700002aee00007406000033
:105db4002e040000700400004c0b000008ff0000db
:105dc4008d0a00003cff00006a0900000afd000083
:105dd40034fb0000e302000079f90000ef01000049
:105de40048f00000c2f7000050fa000064f8000018
:105df40047f30000bff800004e060000c6eb0000a9
:105e040044030000ea010000b5f9000040f8000076
:105e1400c8f300007513000020f6000017f400001a
:105e2400bafc000077f900005a050000a0fd00004c
:105e3400c70e0000c10b0000cc0800008213000054
:105e4400bb0f00003909000024040000220f0000e9
:105e54005b1000002d05000007090000720e000011
:105e64003b02000042020000e604000042f400008d
:105e74004ef400009700000042ff0000c0f500004f
:105e8400eff6000055f6000097f2000076f80000e7
:105e94009fe900002cec0000b902000079f8000032
:105ea400b3fb0000650000003bf60000a9f9000008
:105eb400b4ff0000090100005af700008efe000044
:105ec400e8fd00004b010000d10a000051fc000075
:105ed4007d080000a3100000e7100000a8070000e0
:105ee400a10d00000d0d00007afa0000ad070000be
:105ef40001fe0000b407000028fe000017070000a0
:105f040011060000bde80000c609000068f80000a2
:105f1400c60b0000f80c0000b1fe00005910000090
:105f240083f30000acfd00006af3000045f60000b6
:105f340009f000000ef100002c0d000010f4000028
:105f4400d8f90000c6fd0000d5f9000034f40000c3
:105f540026ff00001f0d00000d000000f3100000dc
:105f6400010700007404000039fe000085f60000fb
:105f7400670c000019000000f60100001ffb000080
:105f84006400000008fe000053f80000cf0c00007d
:105f9400a9f40000e4f900000ff900005b07000019
:105fa400d707000061f000000f050000ffef0000bc
:105fb40085f80000d1f4000032ff0000e711000072
:105fc400d0f90000100b0000180200002c0600009d
:105fd40016040000f00f0000601b000063fb0000cb
:105fe400ca0200000e020000330800009bfd0000fe
:105ff40075fa000032020000fefa0000530a0000a5
:1060040070000000b3090000d20200006ded000032
:10601400c90100008b03000050f80000a700000035
:10602400f00900005bfd0000bdeb000026e7000066
:1060340084f50000a1f20000ebf600001208000055
:106044006eff000055f900009cf50000e20400001a
:10605400930600003bfc00008b04000019090000bb
:106064000c010000f6f8000000010000dbf2000063
:10607400b1ee00004cf700007c050000160900009a
:1060840063020000fe1c0000591000004c0e0000ca
:10609400341000001e1100009e2400007905000049
:1060a400550900009204000076ee0000d5f40000cb
:1060b4003df9000059060000cef100003af100005d
:1060c40042050000b0ff00009dfb0000c5f5000084
:1060d4006ff800000af300002fec00000bfe000034
:1060e40007fd00000df7000091f900009df300008a
:1060f4003dfd000007f80000e7050000e718000078
:10610400f7fb000004f300001cfe0000080100007f
:10611400ba000000feff0000e0050000f4090000e2
:10612400fff90000c4070000d8180000920700001f
:106134005201000012f90000e41000007402000093
:1061440076f6000012240000d50d0000d8f80000f7
:106154006bf80000cef9000032fd00009af8000050
:10616400370a00004d0a000092fa000060f50000b2
:1061740076000000ce040000a8f5000060ed0000e9
:106184002906000093fd000043e6000071ff0000b3
:106194001af300005aeb0000d5f3000034ff0000ae
:1061a400970c00000ffe0000220c0000a70b00005b
:1061b400bd05000034f80000e6f900009b1d000056
:1061c400a9040000f1000000eb050000adf7000099
:1061d400a7fb0000b5f90000a9120000aa080000fe
:1061e400f7fc0000c30d0000c7ff000066fc0000c0
:1061f40001ec000017e40000330000002fef000062
:10620400d0ee0000870d000034fd0000460a0000b7
:106214004808000011090000f11d000027050000d6
:10622400e01e00003f14000088f9000051fa00004d
:10623400d0ef00004a0400007ef10000f9f70000ee
:10624400ef080000bdf40000fd050000b40e0000de
:106254009b060000b608000006f90000e3f9000000
:10626400e302000089ed000097f500002805000016
:106274000fee0000b1e50000a5f300002df30000cf
:10628400a3f900005b020000ab070000c205000098
:106294001cfb0000650300007501000006030000fc
:1062a400abf80000fcf800007f12000055f8000075
:1062b40019f60000a50c000010f10000c7fd000055
:1062c40018160000a4030000d11400008a12000074
:1062d400800c00002e0f00000bfe00008202000064
:1062e400b905000049180000e1000000c5fe0000e7
:1062f400fe0a000050ec0000af0500000ffa000099
:1063040008fc00006e0700000df400008407000084
:10631400a8ee00003ced00000eea000077e7000064
:10632400c9020000d6e600001c0500007901000047
:10633400b1ea00001c0d0000c3f30000b309000023
:10634400220e0000c9fc00007f100000260000009f
:10635400a6030000daff0000cd080000120d0000c3
:1063640023fa0000e201000079fe0000f3f70000c8
:106374002f0400004a010000c4f60000b5ff00002d
:1063840076f5000035040000ff09000070060000e7
:1063940088140000ee080000960e0000c8020000f9
:1063a400720a0000f2fc0000c3fc0000220e000090
:1063b4003cee00008405000076f40000bbee000013
:1063c400abfe00002bf10000e8020000cc09000045
:1063d4002a0900002ffc0000b9f800005be9000066
:1063e400adf40000e4fe0000b1fa00000c06000069
:1063f4001dff000037070000fef6000053040000f4
:10640400fbfd000009030000d11900004afd000053
:106414005f0f00002afa00008bf20000b1fc0000bc
:1064240090fc0000d5f80000f0f30000250c0000fb
:10643400d9f000003e020000c5f60000b7ed0000f0
:10644400e7040000a9f50000bc05000002f8000004
:10645400e30800004afc0000fc0100007413000083
:10646400ce010000df240000950a00001a1a000083
:10647400d21900004505000081170000b50c00008a
:10648400930f000062f4000007fe00000df200000c
:106494000cf60000bcff00008aee0000f3000000d0
:1064a400c0e9000079f9000008f00000ecf10000f8
:1064b40001ef0000beee00007a070000dfd7000005
:1064c40077fa000040e80000f6e8000084110000bc
:1064d4003ff300009710000040050000820d00000b
:1064e400c70f00002c0d0000be0c0000b5f9000021
:1064f400581d0000fffa000051f800005cfd000088
:10650400c5ea00002b020000b8050000b912000023
:106514002d0c0000af1c0000350d000076050000b6
:10652400f1120000bbf9000062190000800d0000a8
:10653400fff6000006ee0000d8e80000dbf40000df
:1065440097f3000048000000c3ee00009c0a00001e
:10655400ac06000034f70000d3120000b8f00000cd
:106564009cf40000fcff0000dbf9000030ec0000ac
:1065740004eb000078ff0000e3f200007ffd000060
:10658400e3fe0000520100006d140000ec0d000059
:106594007605000028090000c6f5000020fc000074
:1065a400881500009fee0000a2f80000d5f8000056
:1065b400a1f10000560c000049fc00004e09000047
:1065c400890c000097120000bd0200006b06000059
:1065d400da150000aaf1000004100000020b00000c
:1065e40071ec00002ff900006e0700009e09000006
:1065f4007d0e0000580c000018f90000400f000048
:1066040091ff0000f3fb0000b104000096ea0000d3
:1066140091ed000005000000f5f8000034d60000fc
:10662400f5f90000c9f20000fce90000ed060000e5
:106634000ee90000480c0000150f000041fd0000a9
:1066440012020000b7fd0000a10200005502000084
:10665400a62a0000d7fe00002eed00004a1100001b
:10666400bcfc0000081200005d0b000058fe000096
:1066740062fe0000fffd00002eee0000a3f2000009
:106684005afd0000c8df0000f508000047f50000cf
:1066940022e40000c9010000f10f000038180000d6
:1066a400450300001f100000bffb00005828000035
:1066b400fe1d00001cfc0000661c000003f100002d
:1066c400bf010000f10b000040090000bff400000e
:1066d400640000008f11000014f00000100c000092
:1066e40056f2000034ff0000260b0000afe4000067
:1066f400e5e80000fbf1000015f20000d6ef000011
:1067040099050000b3d8000063e00000a106000072
:10671400bff5000084130000d2fa00006bf70000fc
:10672400ab0a0000a40500007f010000340500004e
:106734003222000052f200004e0900009b110000ba
:10674400fde800005a120000260c00005e0a00005a
:1067540047fd000053fe0000b1fc0000040d0000e2
:106764003f0b000031e80000fb0e00007ef5000046
:106774007e0a0000d6100000acfe0000bdf8000048
:106784001bef0000e3100000dbee0000b21300007a
:1067940064fe0000c3f7000095130000ccd800008d
:1067a40080fa0000f6060000d9050000c3fb0000d3
:1067b400a5fc0000b4f300004de40000b611000095
:1067c40009000000ff0500009e0900004af60000d1
:1067d400cd1100007a0f0000e0040000a7020000c1
:1067e4003a0800001ff9000028ec0000040500002e
:1067f40013eb0000dff500008d04000068e60000e4
:1068040095fc0000ebf40000e402000034160000e4
:1068140049fd0000a9f10000960e00006415000077
:1068240091fc00002a1f00002c05000010f8000055
:10683400ba0d000015050000e30b00000309000079
:10684400f504000005f80000ea070000a3fa0000c0
:10685400d8fd000013160000b7fe0000dbee0000b8
:106864005ff5000033f20000dfec00008d0f000044
:10687400cbf00000e7ea0000adfa0000c9e1000037
:10688400b7ff00008801000037ef000074ff00002c
:10689400e70f0000e4f7000054fd0000251300009a
:1068a400e8010000aefc00009f0b000071ff000037
:1068b4003f020000ae1e000086f500001ffe00002f
:1068c40055fb000008e300009a0900000c040000d6
:1068d40003fc0000c3f0000079fc00003bf9000059
:1068e40057f80000dc1a0000ad060000f5170000a0
:1068f40047150000ac000000e6220000140a000066
:106904004e0c00004d210000ec0000002cf90000aa
:10691400a7040000f4070000def3000017fc0000e9
:1069240030f70000cdef000026010000f9f8000068
:10693400b3f2000009ef0000f5ec0000a9de00004e
:1069440046000000fbe8000043e800005205000098
:10695400b3dc0000e608000043f20000c2040000bb
:106964003a16000021fd0000d9110000e0f70000f4
:106974009815000028fd0000c213000096130000c3
:106984007be90000e90a0000840100009509000089
:1069940095080000211000005aff0000c80c0000f8
:1069a400fc020000c3f40000bb180000affa0000b2
:1069b4009d01000014f900000a030000baec000075
:1069c40017f200007d0a0000a4e30000850d00001a
:1069d400bdf200006e0d00001c18000007ec000062
:1069e400040d00001ff20000c6ff0000e7030000d2
:1069f400c8040000f601000068e80000f905000082
:106a0400bbf20000a6f30000030b000053020000d9
:106a14000c0b0000b5090000f8ff0000e9040000b9
:106a2400a50b000076fe000017ff0000c7fc000065
:106a34003ff10000e9f80000dcfa0000e4f6000091
:106a4400fbeb000031fe000087040000930300000c
:106a5400430400006eef0000340900009bfc0000ba
:106a6400a3fb00003d0e00009d0200006d1100001c
:106a7400170b00009e1000000d030000c804000066
:106a840028160000660d0000f0110000cf0200007f
:106a9400b1fe000073050000010b000089f4000042
:106aa40097f1000073f400003de700001aff0000b6
:106ab4000df1000095f1000003f7000028f5000037
:106ac4000afc0000eaea000035f90000c8f90000f9
:106ad4000bf6000033ff00007e00000026000000db
:106ae400aa010000ed0900000b030000960000005d
:106af40023fd0000a00d0000bb1400007a09000073
:106b040070070000f2f100004b00000034030000a5
:106b1400d3fd000032fe000068f200002e010000e8
:106b24005bf40000f8fb0000b3070000ad0a0000ae
:106b3400e50f0000ca0a00009f100000c1fe00001b
:106b4400280a00000712000087080000d709000087
:106b54008c030000800000001f0b00004b090000a4
:106b64005ef6000064f70000d6f500009e03000006
:106b7400900200003304000083ef00005be6000095
:106b84007ffc00001cde0000adf100009ff8000057
:106b9400a7f8000043fa000065f100007efd000044
:106ba400eef60000e310000060080000f4fe0000b0
:106bb400e10000008ff90000e20a00004913000020
:106bc4009e060000a8fe0000c003000051fb000068
:106bd400ee060000cc030000620300008500000004
:106be400c6fd00005107000083fb00005f080000a1
:106bf400d800000025ff0000090400008df4000007
:106c04005dfc0000f00400001f070000e401000028
:106c1400ecf700003c010000f3030000040e000048
:106c2400bd14000031f200009a000000a6fa000032
:106c3400c7f00000b10800006b0100002d05000042
:106c440070ef0000fdfb000012f7000063f4000089
:106c54008d130000f7f8000009070000c0040000cd
:106c640028f300003b030000b1020000950500007a
:106c74007af800008ef1000047fd0000b9fc000026
:106c8400a6060000ddfc0000f6f1000039ff00005c
:106c940077f40000e6060000180a0000b5fe0000c4
:106ca400be070000a0f4000006fe00001508000066
:106cb400520a0000270f000061060000d40a0000f9
:106cc400230800004e060000ae0d0000e61400008c
:106cd4000e0f000038ff0000feff0000bf0400009c
:106ce400db03000028fe0000fef800007af100003b
:106cf40068ec000039f4000085f10000e1fb0000bd
:106d040039f70000c8e9000015fb00005ef200003e
:106d1400b1f20000a101000000ff0000dbf600005a
:106d24004afb000067010000bdfc00005c07000096
:106d340040060000bffe00001efc000039030000f6
:106d4400ed0900003b130000580a000023f700007f
:106d5400fc06000079f7000064ff00004809000009
:106d64004c0000002e050000acf200000c060000f0
:106d740055fe00002d0400004b130000b800000075
:106d84001c1600002cfc0000bc0300004719000086
:106d940058fb0000500900003c07000050ff0000b1
:106da4002d020000ab030000b2020000baf500009f
:106db40077f400001af10000cbfd0000d2ff0000c0
:106dc4000af80000fcfa000014f10000d7ee0000fd
:106dd400a1f1000034fc000013fd00001dfc0000c4
:106de4006c02000053f6000029fd000040ff000083
:106df400cf01000019140000e7010000e8000000c2
:106e0400160e0000ea00000016050000650b0000e5
:106e14007d06000047fd000099fb0000ac05000062
:106e2400aef8000089fb000077fa000066f300006a
:106e3400f80900001df50000c5f80000df07000098
:106e440031f6000054fb00000cfd0000d4040000e7
:106e54007ffd0000890500006a0c0000e5000000c9
:106e6400d9090000a60a00009e0f00001b110000b3
:106e74001dff000037fb00003708000030f700005a
:106e840026070000b9020000f2f400000803000025
:106e940075eb0000b1030000e4f7000070fc000093
:106ea4003c0c0000eefb0000ec040000e7ea0000ec
:106eb400ac0000007efd000076ef000072030000cd
:106ec400fcf6000032f700005bfa0000b8f700009f
:106ed40027fa00007cf5000019f700003a080000ca
:106ee400750b00002e070000f8f90000890d000062
:106ef400930600008bf80000181800004d030000f2
:106f0400430d000087130000ce0000003c0e00007b
:106f1400040b00002b090000f11000007c0d0000a0
:106f24006103000083ff000058040000daff000042
:106f340070ef00005afd00006bf10000d9ed000075
:106f440001fb000089e900007df100006bf3000003
:106f5400f1f2000040fd0000b1ff0000cbf00000a2
:106f6400e6fe00002bff0000ddf50000d802000063
:106f74003efd00008f01000063fa0000d00900000c
:106f84001ffd000051060000920c000071ff00007c
:106f9400e11b0000aefa0000dd00000076020000f4
:106fa4001c0100009f020000d9f400008e060000be
:106fb400b4f600006b000000b4f80000e7f800002d
:106fc4008808000054030000810b0000b90b000086
:106fd4006203000027010000d1120000f508000040
:106fe4005709000069130000fbfe0000b50500000e
:106ff4003903000012f30000650000003df40000b6
:107004008ef90000b9000000f0f5000014f900004a
:10701400eeee000053010000fbf10000dbf800007d
:10702400d30300001ff500008b02000039f40000b8
:1070340048fe000049f90000330100007a05000011
:10704400bf070000520900009ef50000db0b0000a2
:107054009000000018060000e3040000f5fe0000a4
:107064005a010000abf90000daff000097f60000b7
:107074002a09000011fd000068010000120400004c
:107084007cf10000f80100004afb00006f000000e2
:107094000c000000a9040000410600006503000084
:1070a40088070000eafd00000d080000400700000a
:1070b4001c0b0000030e00000609000032fc000057
:1070c400d7fe0000f408000008f00000ba03000036
:1070d400c1fc00009af300001a04000027ed000030
:1070e40062ff0000fcfc00009dfc0000a9fb000006
:1070f40063f200000006000060ec0000e003000002
:10710400ec03000003f00000e40a000011f00000aa
:107114006cfc00009f020000c6f600002a0100007b
:107124003cfb0000fa07000081fd00006500000040
:107134003b0a0000c6030000b10b00003405000048
:10714400240000000a0f0000530a0000d5000000cc
:10715400df0f000014010000c10f0000db1000006d
:10716400cf0300004213000042fd0000190c000090
:1071740094fa0000a8fe0000bc0700009aec00008e
:10718400f100000059e60000baf40000ccf200005f
:107194004de90000a60400002af5000021fc0000cf
:1071a40044f4000083fd0000670000006bf9000058
:1071b4001afd00009af5000058050000e4fe0000e6
:1071c40002fb000059030000e0fe00009e000000e6
:1071d400da0a0000e500000089030000200b00002b
:1071e400c1fc00008f030000a5fb0000e9030000c0
:1071f400da010000e4fa0000e705000050f00000a6
:107204005d00000099fa000082fd0000e014000017
:1072140055fc0000f807000082090000e2050000a8
:10722400480c00005d0d0000520c00003104000009
:10723400300b000016fa0000ef010000f703000015
:10724400e1f60000ef0100001cfb000003f5000064
:1072540041f700008a02000017f80000befa00009f
:107264002efd000041f20000fffb00001afa0000ae
:1072740071f9000061f6000067ff000084fc000063
:107284002a050000310b000060f80000200b00000c
:107294001a060000ddfe0000950a00005d030000f0
:1072a4005c000000bbfe0000abfa0000d3f9000054
:1072b40077fe00004501000052ff00006d0200004f
:1072c400d7f90000fff400001f0400005003000081
:1072d40057fd00001bfd0000e100000038fc000029
:1072e400f203000089050000c9fd000081100000c0
:1072f40024030000770b0000a40d0000e901000046
:10730400be0e00008afe00003b030000ebfe0000fe
:1073140074fe00008601000097fc00009dfe000042
:10732400a2ed0000dff60000a0f9000052fd00000d
:107334009a03000071f7000007f70000c6fb000085
:1073440038f90000cbf50000a9fc00005dfa00004c
:107354003ff900004df7000066fa0000b5fa00009e
:10736400d201000032080000bff80000d50600007a
:10737400b702000026060000811500009e000000f0
:10738400d108000073050000ecfd0000e70c0000cc
:107394000c050000910c000046090000b206000034
:1073a40089100000e2020000eb0f0000aa040000b4
:1073b400fb000000b406000023f10000f800000008
:1073c40040ff0000c4f90000c9f700002cf00000e1
:1073d40050f2000092f6000021fd00007efc000047
:1073e400aff8000013f500008ffc00009df80000ca
:1073f4000304000090ff00007afa00000b01000073
:1074040043f00000f6fe000046fe000034030000d6
:1074140028090000f800000014090000b3ff000070
:10742400bd030000f30700005cfc000081fc0000c9
:1074340003fc000054fc0000fa0400008bfe000072
:107444003a01000082fa000024f500006e030000f7
:10745400dbfe00009d0a0000d40400005e02000070
:10746400e70700009afc0000da0b0000110d000091
:10747400270500001908000049030000a8fe0000c9
:10748400bffe00008c040000070a0000d0fd0000cd
:10749400320000008ff900003df70000c60500002f
:1074a400b1f400009c000000b3f7000097f4000062
:1074b4000f00000009f40000f1040000f9f60000d8
:1074c4009e010000dc020000b4f30000e4090000a7
:1074d40041fc000086060000d90500006bf60000a0
:1074e400de060000e4fb00008e0100004203000001
:1074f4005cf800009f0300005bfc000074030000c4
:10750400cf060000c5f90000d800000079f900009a
:107514009af80000dcff0000b5fd000075080000cb
:10752400dbfd000058fc00004805000067fe000079
:10753400cc0f000017090000540a0000510c000091
:107544009ffc0000380d0000e1040000b3070000b8
:107554009003000096fd000084070000def20000a6
:107564009dfe00005dfc0000bef50000c2fe0000b0
:107574000ff0000013fc000085ff0000d2f60000ad
:10758400dffa00005af40000caf1000089f4000098
:1075940049fe000063fe00002cf50000a0fc000082
:1075a40051f60000e2fa0000690400007bff0000cd
:1075b4006d0a000006000000850400006f0400004e
:1075c40075020000800c0000040100000717000091
:1075d400a8ff0000230300005412000005fd000072
:1075e40048170000df010000a80d0000ff0b000099
:1075f4008afc0000880f0000b4ff0000f4050000be
:1076040055f500000fff0000cd000000c5f3000099
:10761400d4fe0000fcf40000ecfd0000ccf70000f8
:1076240081f70000b2fa0000fcf800008efc0000b4
:10763400f9f7000075f900006ff4000048fc000041
:107644003204000084f8000057f9000006ff00002f
:1076540030fa000082030000370700000602000031
:107664008005000027010000d9ff00003c0600004f
:10767400f8fd0000affd0000180600000103000043
:1076840082010000e8f500008e02000027030000dc
:107694002efd00006f06000096f800007d08000033
:1076a400dd0300008b0100006209000029fd0000d9
:1076b4005d070000360700007205000038fe000078
:1076c400bbfe0000b001000086ff00006301000063
:1076d400cffe00003cff0000b2fc00008ffe000063
:1076e4002efa0000a9fc00007df90000adfd0000a9
:1076f4002a020000e9f3000059fc00005af90000d6
:107704007e000000c706000070fb00006105000059
:1077140055ff000049010000c805000025020000d3
:1077240054000000edfe0000da080000d3ff000062
:107734004f01000016fe0000570300002b0200005a
:10774400d6fc00005e080000aef30000e00a000072
:107754005bfb00008df600001807000041ec000000
:10776400510d0000d7fc0000d0010000ab04000064
:1077740026f400001310000069fc0000d00900008a
:107784007d01000034fe0000b80e00000efd000074
:10779400fe07000046fe000034020000c1040000a1
:1077a400dbfe000075fd0000eff50000f2030000b1
:1077b40031f6000089fd0000cef7000092f70000ca
:1077c4004c050000aef100001800000000f20000bb
:1077d40049fa0000ccfd00002ffb0000610400000a
:1077e4003ef300007a03000063f5000093070000f5
:1077f400c9000000bffc0000830e0000e9f7000090
:10780400640c0000eafa0000a80800009e040000ce
:107814003f000000840e00007ff4000050120000be
:1078240045000000d1090000140c000085fa000096
:107834000f0d0000e6fc0000970f000080fe000022
:10784400b604000044030000c6f40000140c000059
:107854002ff600000c020000b6fb0000c0f9000087
:107864003aff000071f700001bfd00009dfa0000c4
:1078740070050000ccf600009af9000090fd0000ad
:10788400eff9000006fd00002b030000b3fc00002c
:1078940050fa00000101000057fa0000090c000032
:1078a400e1f600001a05000098fd0000b5fb000099
:1078b400961000005eed00001b110000c0f20000f5
:1078c40073fb0000f107000016ea00007a160000be
:1078d40073f10000fe06000081050000ecee0000dc
:1078e400b311000046fb0000010c00007200000010
:1078f400b1fd00000b050000cffa00001c0d0000d4
:107904007efe0000e30300002f01000045fd00009f
:10791400eb01000044050000220000004bfe0000c3
:10792400bb0b00008af4000072080000d2f80000cb
:1079340087fc0000900b000090eb0000ae060000f6
:10794400d0f00000c201000042030000c1f90000b1
:107954008d0a0000cdee00003e0d00000ffd00007a
:10796400d7fc0000c8070000b7fa00001c020000a2
:10797400a3fe0000db030000a5f90000620a00007a
:107984006afb00005efc00008101000099f6000023
:10799400ff05000099fe00008703000077f800004f
:1079a4000303000077fa000057060000a508000052
:1079b400e8f70000890f000084f40000e6100000de
:1079c400390200004701000078100000b3f4000001
:1079d400ed1100001df30000030600004204000046
:1079e40081f300003b0a000054f50000d0000000c1
:1079f40042fb00007bff00005ffa00007dfb0000fb
:107a040074f900003bf100003f08000085f4000019
:107a1400a00200007efd000001f100006b040000e4
:107a2400fff40000ac0100006bfa0000c5fe00008a
:107a3400c804000012fa00005e0e0000eef8000018
:107a4400540500000d0700005df800006708000001
:107a540010fe000077050000150400001b0c000058
:107a6400aafd0000f5030000be0b000054fa00005c
:107a7400d60d000048f80000270600002001000091
:107a84008b010000ed08000076f90000330c0000c3
:107a94007df20000ac0a000038030000a0f70000eb
:107aa400da0d000096f300007202000044000000aa
:107ab40043f60000910100006ffb000072f7000024
:107ac40070fb000004f800009700000093fb000026
:107ad40016000000c30200002ff00000ae0a0000f0
:107ae400d2f9000025ff0000280a00003af3000044
:107af400e00a0000adfb0000e700000037030000cf
:107b04004bfa00003603000062f60000f80b000098
:107b140079f90000d5ff0000a90e0000fdf3000074
:107b2400330b000090f8000022010000d30900008c
:107b340037f800008906000017ff0000b4040000b5
:107b440032fc0000a2060000b2040000ccfb0000de
:107b5400a802000025fd000070fe00001bff0000cd
:107b640029010000b2fa0000c307000081f30000fd
:107b74007b04000035050000cbf500008d0a0000f1
:107b84005af40000c50300001bf60000e9020000df
:107b9400d6fc0000f1f80000ae0d000023f1000057
:107ba400310f0000ed00000000030000380a00005f
:107bb40099fb0000510100003dfd00009f0a0000f8
:107bc40009fc000001020000ebff00001df80000aa
:107bd4009d01000007fd00003dfc0000d4fb0000f7
:107be40039fc00008bf70000a30300005f000000d5
:107bf40093fb00000406000080fb0000aeff0000c1
:107c0400dffd0000f50300002f08000070070000ee
:107c1400140b0000db0000003c1300004bfc0000d0
:107c2400f6080000ef040000e0f20000af0d0000d1
:107c340084ed0000450d00000cf7000011fd00006c
:107c44006b030000aee60000c70d0000b7e70000bc
:107c54007e090000cdf900001ef500009c0800001c
:107c640051ed000018090000f6f600007607000048
:107c74006cf600006efa0000ac000000ddf60000b7
:107c8400280900003cf7000099050000c6fe00002a
:107c9400acfc0000db0100002b0d0000c00700005d
:107ca400e0010000e207000047fd00004d0700006e
:107cb40026ff0000c9060000ff01000006000000c6
:107cc400ed0300000a000000dc0c00009500000039
:107cd4006f030000ad030000b7f4000010030000c0
:107ce4005700000036f9000057080000f2fa0000bf
:107cf40055010000c20400004cfd0000d405000042
:107d0400dcfe0000e6fc000000f800009600000025
:107d1400ebfa0000eaf600003afe000081fb0000e6
:107d2400b2fa0000fff800005f000000b900000094
:107d3400640100006bff0000020200007cff0000f1
:107d4400480000003cfe000034020000b0ff0000c8
:107d5400bbf40000200500005dfa00008f01000064
:107d640086020000790200004f05000005fe0000b5
:107d7400a6060000b4fe00001b10000068fe000010
:107d8400c00300004307000033f300006b08000049
:107d9400c7f90000670600008dfc00003dfb0000f1
:107da400360b0000a2f400006f0a0000c4fa0000c1
:107db4001ffd0000480900003bf10000460d0000d3
:107dc40082fa00001afe0000d3050000d8ec00007f
:107dd4002d0900003cf4000016010000840400009a
:107de40087f300004e070000e9f7000014070000c5
:107df400a70200003aff0000a3060000f4f600000a
:107e0400aff90000de09000028fd000004010000b5
:107e14009909000098f10000ba1000008df90000e3
:107e240075fb00002e0c000087f40000880500009c
:107e340071f8000069090000d3fb0000d7000000be
:107e4400c00200008df50000000c000061fe00007f
:107e5400b0090000be020000640b0000fffa00003d
:107e640056ff00006b0a00004ef400006c0f000087
:107e74002bf300009afc000069ff00007cfd000069
:107e8400d60700001af70000d10700001ff5000014
:107e94007efd000047f70000aa010000d90400009d
:107ea40012f80000460700009eea000037070000b1
:107eb400c8f7000086fc00009d090000a2ed000048
:107ec400570d00008cf300000508000002040000b8
:107ed400e1f50000e50d00001df5000004060000ba
:107ee400eaff0000e5000000b000000018020000f6
:107ef4003b090000d2fb000068050000d1fc000033
:107f040063050000dd0200001efa000020040000ea
:107f14007f050000990000005c020000a904000035
:107f2400bbfa000069030000a20200002d05000056
:107f3400db050000c70600002f05000048fb000019
:107f44004c0a000031fb00007d02000081050000a6
:107f5400edec00003e03000032f80000a1f7000041
:107f64009b02000002f90000adff0000a0f5000034
:107f74006afd00000b010000eafe0000bdf80000ed
:107f8400bcfa000007010000ccfa00004f0000001a
:107f94007ff8000009000000fbf5000081000000ec
:107fa400d800000046fb0000c8100000b6fc00002a
:107fb4003b0c000051010000530200002c0a000099
:107fc4005afb0000e80b00009bf80000d5060000f7
:107fd40080000000fd020000b315000019f000004d
:107fe40085080000c00100009cf900004e0b000051
:107ff4006df30000320a000010ff000004fe0000d0
:108004006305000036f80000d40100008ff9000079
:108014001505000034f6000076fa00001700000091
:10802400f4fc000032ff000092f50000050300009c
:10803400c7f20000c80300004d01000078fb0000f7
:1080440037030000f4ed0000f8060000800600008d
:10805400c6fb0000b10400009d0100004b030000ba
:108064000b04000001000000920300007c030000e8
:1080740083010000210000005efd0000bf0100003c
:1080840054fe0000e90500009f060000d5fe000034
:10809400860700000505000057fe0000300d0000b3
:1080a400a1ff000070f60000c206000041fd0000c0
:1080b400b100000049fa0000c1f70000ebf800002d
:1080c400dc02000047050000acf300004a07000092
:1080d4007dfe00000b000000af020000f7f5000079
:1080e40094ff00005afc00003fff00002efe000039
:1080f400d0fc0000fbf9000071fa0000ca03000084
:108104004a00000050f70000a1000000d601000062
:108114001d04000069080000defa0000fe040000ef
:1081240006ff00007e020000eafe0000d6fd00000b
:10813400e706000050f900003210000048ff00007c
:10814400d602000034080000a0fc0000730a0000fe
:10815400f2f500009e04000050030000cd02000070
:1081640056fd0000e5f20000b100000093f90000a4
:108174005f0300001001000009050000260500004f
:108184004b000000ff020000de01000074fe00004e
:10819400b9fd000002000000a6f500000ffb00007e
:1081a40067fd0000a0fd00001dfb0000f2040000bc
:1081b40023000000970300000e0c000071fc000077
:1081c400e805000016fa0000c7fc0000b6fa00003b
:1081d400410200001dff0000b1eb0000a4030000f9
:1081e4006df30000daf7000096050000ccfd0000f6
:1081f400bb0f0000360a000001fe00009f0a0000c9
:108204001c030000abfb000021fb0000da000000af
:108214001c0800009df7000030020000ae030000bf
:108224004bfe000021030000ce030000de0300002b
:10823400ac0e00008e0300000cfd0000250a0000b7
:10824400daf00000f10500006ff90000e3f7000028
:108254004d020000d1f4000098090000c5f50000ab
:10826400e90300003cff000085ff00006fff0000f1
:108274002cf90000abff0000a5f00000640600002c
:10828400fdf7000017fe000073ff0000a2f10000dc
:10829400ea040000adff000031020000e108000024
:1082a4002f0800005e0f0000640600005600000066
:1082b400bc040000f3f500007c0300003efd000058
:1082c4002af600008a04000096f40000fffd000076
:1082d40011090000d0060000500d00004205000006
:1082e40057070000c90400007afa000043020000a6
:1082f400bdf30000c208000072f800006cf5000035
:10830400c40c000007e70000cc02000051f9000093
:108314006c030000190c0000d4fd0000120a0000d8
:10832400f3f900009d080000d5f10000dff800001b
:108334003e01000047f6000024fc00001302000088
:108344002dfd00008cfc0000860b00005cf4000096
:108354004a0c0000c506000039fb0000810800003b
:10836400cbf60000b3f900005406000013ff000030
:10837400e7f600004c09000064f90000fafb000075
:108384007504000066080000d404000065030000c2
:10839400c506000021fb0000b807000034eb000014
:1083a40061020000290000009bf100001c0a00008b
:1083b40001fc0000d00800001eff00005b0c000060
:1083c4001304000089060000a3130000c3fb00008f
:1083d4002d08000024fb000002fa000058050000ec
:1083e400f7f80000f5f10000a6050000ebf5000029
:1083f400fbf1000057150000b507000095ff0000d1
:1084040046000000df01000059f50000b6f6000048
:1084140041f80000fcf000002802000014f0000005
:10842400ebf700007807000018f0000015f80000d2
:10843400a4080000200100003d000000310a0000f3
:10844400aa0d00008d040000e6070000f1fb000007
:1084540012ff00004c11000027f80000410c00003e
:10846400650400005cf10000ff08000087090000bb
:1084740055040000940100005d130000e2020000b6
:10848400cdfd00007ffd0000e1f70000fe000000cc
:108494006af50000f2f5000082ff0000c50100004b
:1084a400f4ef000008080000b7070000b0f6000071
:1084b4005eff00005dff0000ee01000031f20000ed
:1084c4002cf80000c4f4000020fe0000cef30000ed
:1084d400dbf80000230d0000e4f60000b3090000ff
:1084e400b90900002f0900005f0d00006b0c0000ab
:1084f400090c0000bdff000039fc0000bff80000bb
:108504007bfc00008dfa000057fa00008500000093
:10851400910400009afb000057090000c10d0000ff
:10852400fe030000600800006e050000e00100008a
:10853400f9fa00007efc0000e0fc000003ff0000ec
:1085440040ea000082ed0000bf0000002ffc0000a4
:10855400d4fc00007c060000b609000043f90000ca
:10856400530a00006b060000660a000007030000bf
:10857400dff000001300000000f200003e030000e2
:108584004a0100007cfe0000f2fd0000e1eb000067
:10859400ff0600002102000096fd0000d711000034
:1085a40042070000f1fe0000a9f9000023020000c8
:1085b40062fe00007df400002b000000def70000e6
:1085c400500800007bff0000fe09000004140000b6
:1085d4007df60000a4040000e00400000b0e00007f
:1085e400d5f5000038f80000c7ff000015ed0000c5
:1085f400aafb000000fa0000af0d00003d080000d7
:1086040005040000e70200009b0300002e080000a0
:10861400f70d0000e30e000006f500005cf6000014
:1086240046f8000020fd00002ef50000fef80000d2
:10863400fcf8000083fe0000deff00008100000063
:108644006610000034fd00005a09000041fd0000de
:1086540094fe0000a5f7000045f60000cb060000dc
:108664005cec00007ff7000079ea0000720600006d
:10867400580500006bf3000027110000f0fa000019
:1086840084040000570a0000bf140000bb1200005d
:10869400e1fb0000ceff000043fa0000c3fe00002f
:1086a400b3fd0000fe080000ba0b000070f80000e3
:1086b400b1fc0000f8000000cffd000097000000ae
:1086c400f6070000310800000ff90000f3f5000080
:1086d400d700000077fd00000dfc0000cefc000078
:1086e400650200009f0300008af40000620a000093
:1086f4001206000068f10000760a00001b05000065
:108704007a0000009df40000daf400000a01000081
:108714007aee000026fa000034fb00002905000070
:108724008c07000039000000ac0700005dfd00006c
:10873400260500008c0c0000350900009afb00009f
:10874400deff000022f7000097f800006f0600002b
:10875400a7fa0000430b0000140500007401000098
:10876400920500008b080000290200005106000059
:1087740075100000e0f2000070ff000098f900009e
:1087840064fa000097ff000087e9000038f7000052
:1087940007fd000021fa000043f80000570600001e
:1087a4005ffc00009cf800000809000016070000a8
:1087b400420e0000f4020000d7fa00004b01000052
:1087c400e4000000bdff0000d70a00004c080000d0
:1087d400f1fb00001e010000d5f9000055f2000075
:1087e400ce070000810a000074fa00005f03000055
:1087f400b2f30000aef800004c07000037f40000ac
:108804008c040000d10200007def00008203000010
:10881400e00c0000ddfa0000d8fd0000f1060000c5
:108824009d01000015fb00006cfa000035fc0000ff
:10883400cd030000250a0000bcf60000470200003a
:108844002e0a0000e0fd00000e13000018070000cf
:1088540035f90000cd0f00005f0500005cff00004b
:108864009d0800007ef50000f8f8000060fd00009f
:1088740026f6000085010000220200008ef30000ad
:1088840016fc0000ed06000040f4000019ff000093
:108894001106000038030000740000002af50000ef
:1088a4007efa0000eefb00009b00000032f60000a0
:1088b4008c0800006d0100005ee900000d07000057
:1088c40082fc00004f0000000d090000b60000000b
:1088d400be0b0000b2060000cffe0000bf0800007f
:1088e4001a09000017f80000f90a00005b040000f0
:1088f40062f700008701000076fe000009fc00001a
:1089040071f200008403000041fc00009f0300009a
:108914004a060000d8f40000fb0e000091f90000a4
:10892400bffc00000b10000064fe00006afc0000a5
:10893400cb090000c007000032f700006a080000fd
:10894400350100006501000025fc000003ea000079
:10895400c7ff000093fc00005bfc00002300000044
:10896400fbfd000019f400002ff70000360800009a
:10897400c9fb000067ff0000f2000000a6ff000032
:10898400e0020000cdfc000039fc0000b906000044
:10899400280a0000c90000007b0b0000d50300007a
:1089a400a7000000500f00007305000073030000cf
:1089b400370600006aff00004009000021020000a1
:1089c400fbef0000afff000020fa000000f80000f9
:1089d4006dfc00001fff000014f6000028eb0000ef
:1089e400df020000d6ec000066fa00007b070000fe
:1089f400090000000911000021fa000082fe0000b5
:108a0400e606000050090000c9020000fb0a00004d
:108a1400e106000002fa0000380800004af90000ec
:108a24007b0700006cfe000019f700009eff0000a9
:108a3400aefb000051fb000066f90000a80800002e
:108a44001af60000fefd0000df0100003ef7000002
:108a5400f90100008206000026010000aefa0000c1
:108a6400be05000089ff00005d0c000092fe0000be
:108a740006f6000059020000d5fc0000d30c0000eb
:108a8400b5030000c00900007106000081fe00006b
:108a940078030000c3010000b40700001bf90000c4
:108aa40049010000c8fe000013ef000077fc00003d
:108ab4008804000063020000c40400003ffd0000bd
:108ac40087f100000cfd0000df060000a901000092
:108ad4000efe0000daff000024f80000d1ff0000c1
:108ae4000ffb00007ef00000d900000037fa000000
:108af4002e000000aeff00007a020000a40800006f
:108b0400b7fb0000ef000000b2f700009e05000074
:108b1400030a0000050800002910000052f50000b7
:108b2400bd000000bb0800002bfe0000da0a0000b4
:108b3400b2070000d0fd0000fdf90000e8fe0000cf
:108b4400c000000099fa0000fafc000011fe0000c9
:108b540040f90000d9f9000003f900001efd0000ef
:108b6400ba080000760000009600000089070000a3
:108b740030020000f0020000e6020000ce04000013
:108b8400daff0000ec0100003600000015020000ce
:108b9400f1fe00001bf5000020040000aaf800000c
:108ba400e9ff0000100500004cfe000078fc000006
:108bb400c6f3000064030000f2ed000001f60000bb
:108bc4006007000035fb0000fc000000e6f3000035
:108bd40093fa0000c8100000c40900007d080000da
:108be4004b110000a4040000720600001f0a0000dc
:108bf400970e00005a0900001c00000087020000c4
:108c040038f3000060f80000b8f4000029fe00000a
:108c1400e7010000b6f600005dfc00008bf90000df
:108c2400e7f50000cef40000ed07000029f1000094
:108c340020fa0000230d0000c7fb0000e60b000033
:108c44009cf5000085fb0000c80a0000b403000086
:108c5400b1080000aa090000860c000058fd0000bd
:108c640046040000c300000026f600007ffe00005a
:108c74001e02000069f900008cf50000e9fb000009
:108c840062f60000b40d000012fd000078f600004a
:108c9400fe0c000089f10000a2040000650500003c
:108ca4009ef8000069020000a6030000be07000051
:108cb400a6fa0000820600007ffd00005f060000a7
:108cc400ed100000b4f70000ea0a00006808000094
:108cd40047fd000027010000b00100009cfb0000dc
:108ce40050f10000fbff0000bbf80000adf80000ed
:108cf4006b03000012f70000770b0000a4010000d2
:108d0400a6f600009c1200005af7000041fe000085
:108d1400480c0000b3fa00002b030000fffb000026
:108d2400cc000000aef800000bee0000cdf5000012
:108d3400f7fa0000e40b0000ebff000017fc000052
:108d4400db09000027f20000a0ff00007e100000f5
:108d54003bfd0000bf0b0000950500005afe00001b
:108d64006cff0000dcfc0000b4070000b20b000044
:108d7400650600005af500008f060000e1010000be
:108d84000df700000c03000064f20000c8f40000ba
:108d94001f010000520000005efc0000fefb00000a
:108da4005dfb00009cff00000f080000ba010000fa
:108db400dfff0000200e0000a9010000eff6000014
:108dc400cf07000043040000110a000090070000d0
:108dd4007afc00000efe0000fff900008c03000086
:108de400460a0000c6020000e9f90000c0fd0000c8
:108df40033f8000062f10000dbfa0000f6fc00002a
:108e040076f700005df40000dcfb00007afa000055
:108e1400e0f70000f2fc000053010000b508000078
:108e2400ab0300004f070000e6100000120d000025
:108e3400900b000056070000ff0900001605000013
:108e4400760100005004000064fa000096f500006a
:108e5400a8f7000074060000defd000028f80000fa
:108e6400cbfb000082f200009df7000003fb000032
:108e7400810300005b0200004a0800002d0400008a
:108e8400e5f900005bfa000048f80000f80800006b
:108e9400e20a00001e02000057fc0000470a00001e
:108ea400ff05000017fa000064ff000011fc000039
:108eb400aa02000043f70000f5000000b300000020
:108ec400caf20000430300000dfe00004bf900004d
:108ed40023f9000075ff0000ed06000070fb0000a0
:108ee400caf900000a01000016060000ba080000d2
:108ef400180600001f01000038fc000030fb0000d1
:108f0400aa0800007c1300003c060000850600004f
:108f1400320b00003cfe00008afc000021fb000034
:108f2400ab020000d103000058f4000017fb00005e
:108f340089f90000f2f100008c03000063ff0000d7
:108f4400a5fb0000b5ff00009af60000e50c000048
:108f5400220400007bfd0000ff06000096f70000dd
:108f6400bb050000d5f900009af700000dfc0000d5
:108f740021f20000a60200002c0200009704000069
:108f8400c70200001b0100000b000000ecfc000005
:108f940048020000010a00003f0f0000cafd000063
:108fa40077040000d1fe0000dcf200008005000020
:108fb400c6040000eb080000fcfe0000a9f9000054
:108fc40086060000eefa0000defa0000eafd00006a
:108fd4003afa0000c4fc0000c7f9000048fd000094
:108fe40049fd000089f60000ac02000006060000fe
:108ff40007030000b407000058050000740b0000cc
:10900400b8fe0000f3010000f90800002afd00008a
:10901400c9080000a1fd000034fc0000f8f60000bf
:10902400dafc0000ba0a0000effb00002301000094
:10903400f3f50000e30100004ef8000049f30000de
:10904400ca0500006ef5000003030000bdf7000030
:109054000ef80000b4fa00001ffa00001207000026
:10906400c7020000770b0000abff0000730d000087
:10907400df0a0000ab040000670b00001d030000c2
:10908400fc0b0000e1fe000062040000e0f70000b9
:109094005ffa00001a01000042f70000a00300007c
:1090a4002af100000e0100007cfa000084f50000a3
:1090b400b3fe00003bfc00005d070000f9f900006e
:1090c40043070000d5f60000e1fd00006e03000038
:1090d400b2fc0000ea150000f70200004b09000092
:1090e400310400008b020000dcfe00002cf80000bc
:1090f4004509000005f6000009fa000042fd0000e1
:1091040076f20000d8f8000087fb000030fb000076
:109114002f02000022fe00002bfc000020040000af
:10912400e8fe0000aafe00007a000000ce0700005e
:1091340072000000f40300002106000021fb00007f
:109144005a0b00005e05000054090000710b00007a
:1091540085fb0000f90700006f00000024fa0000fe
:1091640003020000330000003707000041fb000049
:1091740029fc00006cfb0000a7f500001b060000a2
:1091840049f60000780200004afd000080f4000067
:10919400790900006af40000b30000003402000002
:1091a400fffe000014040000c0fa000002fe0000ec
:1091b40033fa00009304000047fc0000080100009b
:1091c4002b090000f8f9000089fe0000e702000006
:1091d4006dfb000073010000d20b0000faff0000d9
:1091e400e4060000a8fe000098fa000080020000d7
:1091f4008ffc0000800400003d00000064090000b2
:10920400baf80000c7fd000053060000faf00000a1
:1092140091060000f3fb0000fefc0000c801000002
:1092240052fa0000effd00004ffc0000980400001b
:10923400a1ff0000b00c0000e90300004702000099
:109244003e090000c0fa00005c0200002c0500008a
:10925400fb040000e5ff00006c0500003df8000081
:10926400cdfc000068040000d7f300007404000083
:1092740039f70000ddf90000d1f90000f6f600002e
:10928400defe0000bff700003606000088f500008f
:1092940096fd0000500000001cf900003409000095
:1092a4009b020000220300006c0800006407000019
:1092b40027fd0000080d0000100200007a010000e4
:1092c40071110000ee0100003e0b000022fe0000c0
:1092d40030ff000090fb000051fa0000f6fb000094
:1092e400fef300003806000021f500009efa00009d
:1092f40029ff0000ccf70000d8000000fb010000ab
:109304002b00000021fc000094030000d7fa0000a9
:10931400b4040000240700004afe0000fa0b000019
:109324009d02000071fb0000db0100005e010000f3
:10933400fefa00004701000065020000b7f70000d4
:10934400ebfe0000f6fa00006cf50000e5fe0000fc
:109354004efb0000aeff000026050000f0fd0000fb
:10936400fefe0000ab0400008e01000043fd00007f
:109374004506000006020000ab010000ce05000017
:1093840050020000f80500002302000094030000ce
:1093940024070000ca07000096f80000c4fc00007f
:1093a4001a070000f2f80000a3030000ca0100003d
:1093b4008cfc000015fc0000faf70000a7fb00007d
:1093c400d7f9000013fd000029fd0000b7040000d8
:1093d40030fd00001cf70000b50500008900000006
:1093e400940100000d050000ee010000ef020000f2
:1093f400b1fe0000af000000aafe00008afd0000dc
:10940400f7fc000018ff00003706000084f7000096
:109414001cfb00006809000030ff0000420100004e
:1094240091080000a4fe0000c7000000ec0000004a
:1094340000fa0000320500004dfd0000fdfd0000b3
:109444004b0800005601000064fa000036fb0000df
:10945400ec02000099f90000f2fe000049fe000051
:1094640042f90000560000006afc0000b901000047
:10947400a30200008e010000d4040000970d000038
:10948400bb04000003fc0000be08000074030000dd
:10949400b5ff00008c04000062fc000041fd0000e8
:1094a40047000000d9f8000002050000c6fc0000d7
:1094b4006dfa00001e06000084f90000ddf80000cb
:1094c400a9f4000003000000f4ff000003fa000008
:1094d4002300000092fb0000b7010000cbfa00005b
:1094e40020ff0000af0400002dff0000e700000093
:1094f400260a00000c050000d1f90000bf0b000093
:10950400a20300000f030000bd0a00004fff00008b
:109514008b070000950100006afe0000ef030000c5
:1095240042fe000056f9000044fb0000f5ff000075
:109534009af6000046f70000e40200005f02000013
:1095440098fb000092010000680200007cfa000011
:10955400da000000e9fc00006f0400005d04000074
:1095640028fd0000d8080000bb00000085fc0000b6
:1095740070fd00003301000076fd000042fc000095
:10958400d0fd00009cf90000a60000007bf900005b
:10959400c701000084fe0000a5fb00005103000089
:1095a400f6fe00005505000057fb00008f07000081
:1095b4001d0900008cfb0000bb04000012ff00002a
:1095c400a5000000e3010000fcfe00005c090000af
:1095d400c90700003ffd0000000700001605000059
:1095e40055f7000010ff000006030000dffe000036
:1095f40011fe000022ff00002cfd00007fff000090
:1096040069fc000055fb0000e8010000b4fa00000a
:10961400e9f900001ffe000020fe0000edf7000045
:10962400490300006a0b000086f90000d50400001d
:10963400f1020000cff90000c70300007efd000026
:1096440005ff0000c2010000fffb0000f2fd000066
:109654002f07000037fa0000b8f9000038090000ad
:10966400b900000034040000be0500003207000009
:109674002401000058fd0000170300004bfc00000b
:109684004b020000a7fb000003000000de03000003
:1096940093f80000b2000000180400003ffd000031
:1096a40040f70000abff00008cfa00006ffb0000e5
:1096b400a6030000bcfe00002f080000cdfd000042
:1096c4005a000000030a0000d0fc00001002000051
:1096d40060050000e20500004f010000a2ff000049
:1096e4003903000023fc0000c6fd000078fe0000e2
:1096f400e0000000a5fd0000cbfa0000bfff000061
:10970400e7fc0000adf60000d7f700005b050000a1
:1097140099fd0000f5f700004d01000016fd000062
:109724006dfb0000fb000000e4000000620200008a
:10973400f3030000a9fd00008d090000af0500003f
:1097440000000000d80a000091090000c3090000cd
:109754002d02000019090000ffff000047fa000075
:10976400a8030000c7f70000b6fe00003df80000a3
:1097740069f90000d00100008bf600003efe0000f5
:10978400640200009600000078ff000075ff0000ee
:109794002402000058f8000092f80000f8000000cd
:1097a400f5010000c8020000d5fb00002f040000f2
:1097b4001c0400000cfb000094030000c5ff000023
:1097c40081010000d4fc0000cdfd0000bcff0000be
:1097d40000fa00008f010000cbfe0000d20400005c
:1097e400f9fc000061fc0000cc070000fefe000054
:1097f4006202000020050000e9000000d5fd000021
:1098040017020000310000006efe00000700000097
:10981400a8010000d7080000060200002400000090
:109824008f010000d902000077fc0000edfb00006e
:109834003c07000012ff0000f1fd000030ff0000b3
:1098440013fb000047fd000070fd00000cfe00004b
:10985400170300006cfd000043fd0000e20300005c
:10986400dffc00005901000034030000160500006d
:10987400a7fd000008fd00007303000056f7000078
:10988400b2fc0000dafa0000e8ff0000d6ff000096
:10989400e9fd000071020000e3fd00004bff000041
:1098a40022fd0000f00a0000d2000000d7010000f1
:1098b400dd040000fbfe00000f03000052f900006d
:1098c40025090000b5000000e9010000c200000005
:1098d400befd000001060000b5f8000020040000f1
:1098e4006dfd000016fd000008fa00009bfa000060
:1098f400cdfb0000e4f80000690600007ffe0000d4
:10990400ac0800006dfe0000f5020000590a0000da
:10991400e4fd000097040000200000002005000082
:1099240085fd0000ce020000d6fc0000e5fa000030
:109934004e03000075fb0000f7080000fafb00006e
:109944008bfe0000d6000000a8fa00006afc0000ac
:10995400b7f80000ec0300006cf70000f3f8000017
:109964000bfc000097f90000affe0000e2000000cd
:10997400f304000023010000c503000027fe0000db
:1099840056090000b4030000de000000a00e000031
:10999400c6020000d80700003c00000010040000cc
:1099a400260200005afd0000b403000077fb00000b
:1099b4006b0300001ff900004401000047fc000095
:1099c400fbf600006803000010f900006b020000c1
:1099d4008cfa000050fe0000cefd0000dbf7000012
:1099e4004d0200007efe0000d802000010fe0000c0
:1099f400b2ff000011010000c4fe0000bfff000020
:109a0400da030000d004000083fc0000d7ff00004c
:109a14008af90000f7fd000053020000680000000e
:109a2400650600008dfe0000d6ff0000d401000092
:109a3400ee010000dc020000d1000000310400004f
:109a4400250200005d00000040ff00003402000019
:109a540058ff0000fa0000007e0300001cfc000018
:109a64000c02000063ff00002c030000b30200009e
:109a74006afc00004c0000001901000028010000ed
:109a8400c3f70000e5ff0000f1fa000050fd0000fc
:109a9400a802000089fb0000f4030000a6f7000000
:109aa400efff0000a6fc00001ffd0000aa05000057
:109ab4003afe0000bb090000ebf9000036ff00008d
:109ac400630300003cfa0000880200001dff000050
:109ad4008100000004fb000090ff00005802000019
:109ae40033010000b702000015ff00008a080000df
:109af400d3010000abfe0000bf020000abfe00007b
:109b04009b030000f3fd00004102000096020000e8
:109b14004ffe00008a0400006ffd0000e802000010
:109b24002cfe0000e40100001c050000d0f8000039
:109b340053fe0000f1f9000075fc000094fb0000e6
:109b4400f501000024ff0000d4fa0000e70400003f
:109b540003fc0000480400003a010000c0ff0000bc
:109b64007a05000067000000bffe0000a1fe0000af
:109b7400390300003f020000fd020000ebfd00007d
:109b84003bff00005fff000017ff000058ff0000cc
:109b9400e4fe00000c0000005cfa0000c2000000bb
:109ba400c1fb0000dbfa00007afc00008efb000021
:109bb4006bfe000049fc00007f030000ebfe000088
:109bc40054040000e4040000ba0000003a09000054
:109bd4002ffe0000730600000009000032fb0000a5
:109be400250400000c0300004b040000ba0400002c
:109bf400ebfe00002f0300002dfd000081fe00009d
:109c0400ac01000098fe0000f5020000defc00003c
:109c14007ffc0000a6fd0000d1f4000075fd0000eb
:109c240035fe00007ffa000069ff000088fb000099
:109c340080fc000000fe00001a0100006d0000001e
:109c4400c60100004d0100002401000015060000bb
:109c540062fe000090000000f6ff00009b00000080
:109c6400630000003b0000000a030000befe000089
:109c7400d103000000fe00001a0300009903000055
:109c8400b3000000db0400001cfd000085000000a0
:109c9400fcfd000017020000c801000037fe0000b0
:109ca4007d000000e6fa0000b6010000f1fe0000ad
:109cb4001dff00001f0400000bfe00002500000033
:109cc4009bfe000090fd000051fe000088fe000095
:109cd4000f010000c3fd00003bfe0000affe0000ca
:109ce4004f010000f1000000ce000000d00200008f
:109cf4001e00000075010000e2fd0000ec01000000
:109d0400cbfc0000eafd0000b005000021fd0000ce
:109d140010020000c4fd0000bbfd00000ffe0000a7
:109d24004ffd0000c9040000c7ff00003c02000012
:109d3400be0000002c010000a1ff000089fa000011
:109d44003d02000010040000f80200004a02000076
:109d54004b0000007bff00005ffd000014000000ca
:109d640040020000af010000f4020000e8fe000021
:109d740085ff000088fe0000cafe00007e0000008f
:109d840097fb0000ca000000d9fe00008dfd000012
:109d94000bfd000078fc00007401000039fd000098
:109da4001302000062020000db0500009c010000b9
:109db4007ffa00005f030000fdfb00006404000064
:109dc4000001000091fe0000b10500004bf9000005
:109dd400a501000088000000550300002ffe0000cc
:109de4000efd00000a030000c0f70000bbfc0000e9
:109df400e5fa0000ad020000a9fc00009efd000091
:109e0400320000005bfc000051050000a2fd0000d0
:109e1400ca0a0000360000001d020000820700008c
:109e24007afe0000dd0600005afe0000f505000081
:109e3400c1fd00000c010000d20300006a00000014
:109e440035030000b9fb00009a08000080fc000004
:109e54007201000074fe0000b9f900005401000012
:109e6400baf2000022040000abfc0000e9fc000090
:109e74009dfe0000a9f2000032fd000019f300006d
:109e84009cfe0000d9060000eb010000f80400006d
:109e9400ff04000024020000c9020000a500000025
:109ea4008dff0000310d000011fd00006c03000067
:109eb40012020000d6f90000640000009cf60000c5
:109ec4008e0b000035ff0000a8000000cc0000004d
:109ed400baf800002205000037f400003a0100003f
:109ee4009400000085fe000072010000f5fd0000f2
:109ef4008dff000022000000b60b0000bf0300002d
:109f0400aa080000f703000084ff0000c0fe000060
:109f14008af900007d040000a4ff0000640600002c
:109f2400fc0400001dff0000890000002df8000063
:109f340010010000b203000072fd000063f800008d
:109f4400cff3000053fc0000bbfe000018f9000032
:109f5400aef60000dffc0000f2fc0000b2f60000e8
:109f6400fbfd000089fb00009c0200009804000037
:109f74000fff0000450a00004500000061050000d5
:109f84004e0800004b040000700d00001e0100008c
:109f9400090a00006b0a0000c4fc00002eff000048
:109fa40037f5000067000000eb040000ee0200003b
:109fb400b9ff000080f000007d040000f4030000fd
:109fc400b40000008f05000070fd000097fe000043
:109fd400affa000074fe000010fd0000eb0000006a
:109fe400e1fa0000bc00000023090000c9fb0000e6
:109ff40001fd0000820000007401000059f7000018
:10a00400b2fa00006bfc00000204000060050000ce
:10a0140085fe0000e1fc0000b4f900008a0a00009b
:10a024005900000028000000e3fb000080f6000057
:10a03400d9fe0000f5fa00009e07000073fa000044
:10a044003ff90000790700002dfd0000150600000f
:10a05400800600007d040000050d0000a2f9000048
:10a06400af00000046fc00003afc0000681000004d
:10a074001e010000a103000043f900006d0500006b
:10a084003d070000b0f700001c0e0000e1020000d4
:10a094003bfc0000ecfe0000cafa000055fe000084
:10a0a400cffb0000dd010000b7060000fefc00004d
:10a0b4008af6000087f5000033ff0000f7f7000080
:10a0c40068f1000067fc0000e7f300000e040000e4
:10a0d400fc04000093f5000087fe000086000000e9
:10a0e40039050000350f0000710f000067050000fe
:10a0f400410600004c0200004bfe00002c0400004e
:10a10400690700005a04000037ff0000dbfc000070
:10a11400b6ff00001cf80000ffff0000611a0000f9
:10a1240061f6000062ea0000cef7000077f9000053
:10a1340089030000ddfc0000bc0200002ff40000d5
:10a14400d500000013080000e90000004f060000dd
:10a15400eaee0000f9f70000780e00004c08000059
:10a16400160600002a150000bcff000017000000be
:10a1740074030000a6fb000053020000dbfa000099
:10a18400410b000066f60000a1f7000009f600008c
:10a194000cff0000c50b0000c9ea00003efa0000f5
:10a1a40063f300006b05000098010000e6f900006d
:10a1b4006006000048e6000041fe0000db080000e5
:10a1c4003705000084070000120700005e1200003b
:10a1d4007f0d000022080000e2050000d405000005
:10a1e40089fc0000edf1000098f5000048f800003b
:10a1f400cced0000700900009e1200000ef3000078
:10a204002a00000078050000a5fa0000b8fc000050
:10a21400a60800005a020000e1fb000052050000fd
:10a2240097f40000660300008dfe0000fbf60000ba
:10a234002b110000b1fe000001fe0000790a0000ad
:10a24400421700003303000020f30000f8fe000072
:10a2540097ee0000280200006b0100002a060000af
:10a2640019fc0000a4ec0000f40d00003a06000004
:10a27400360a0000990000002df700008af700005c
:10a284007cf10000f7fb0000d1fd00004805000050
:10a294003fed000030f50000feff0000f4f5000083
:10a2a4007e160000bf110000f6020000f2f6000066
:10a2b400bdf00000011000008e0b000055060000e8
:10a2c4005f05000097ef000081fb0000f0fc000038
:10a2d400a2fd00000c0a000053060000a8060000be
:10a2e400770c00001d110000a8fe0000ec02000025
:10a2f40009070000e4f900006c030000c4f1000049
:10a30400faf70000f0030000abeb0000b9ef000027
:10a3140002f200004af900008f020000f00e000073
:10a324006c10000058ea0000eb090000c20a0000ab
:10a33400eef20000db12000087f600005cfc000077
:10a34400c2ff0000f9f70000ca080000440e000034
:10a354008d13000048fd00002a0d00006cee000083
:10a3640024ec000005070000d0f70000380b0000c3
:10a37400b7f50000c8f00000b0f1000008fb0000d1
:10a384003d02000058000000980a000088fc00000c
:10a394000f1b0000011300006bfa0000360c0000d4
:10a3a400b5fb00004ff90000fe01000008f40000b6
:10a3b400b80900002f060000b7ee000016050000e3
:10a3c400e90f0000160b0000770d00005a1300007f
:10a3d4002eec000032e5000083f30000bbf1000026
:10a3e4008f0b000016f700006df000004bef00002b
:10a3f40007eb000094fb00004c0a00004e0f000025
:10a404006c000000810d0000f5fb0000d4f5000095
:10a414005a0e0000c2090000b90b0000b8f9000090
:10a4240072f800009e0c00008eff0000b4020000d1
:10a43400e20c000009010000bb01000080fe0000e6
:10a44400d2fb00008ef8000035f100004bfb000049
:10a45400c5fe000062030000fd010000300300009f
:10a464007f030000def2000093000000130c0000e4
:10a474009b010000c20700008d11000014010000c0
:10a484008df5000077030000ac0500009d0d000071
:10a49400380a0000c1fa000032fc000047ed000059
:10a4a400b0f40000250c0000b509000013090000f9
:10a4b4004d05000098f10000e9ea0000e3f800000f
:10a4c40097f80000cb0400001bfe000017f000000a
:10a4d400c3f70000c7e4000079fa0000580900003f
:10a4e40097000000f8fc0000440200007e16000003
:10a4f400880a0000ca0e0000ccfb00000f00000018
:10a504009a120000abf90000ee0500009408000068
:10a51400f9f8000048060000b60a000025f2000021
:10a52400be070000a30b0000c6f2000017f00000f5
:10a5340024ea0000ae010000520c000037140000b1
:10a54400d506000093f30000c0f10000ecf2000017
:10a55400780c000034fa000009f0000020fe00002e
:10a5640066f60000770200004104000077ff000057
:10a5740078120000b213000035000000cdf6000090
:10a58400050900008c07000084080000b0140000d6
:10a5940020f2000043f9000003fb000004f2000075
:10a5a4001b04000017f00000fffc0000860f0000f1
:10a5b400b506000099f9000094f6000049f5000082
:10a5c40070e40000800200006f000000f0f300005f
:10a5d400a01900004e0f0000da1400002f0900003b
:10a5e40001f000000b1d0000a91c000028fb000066
:10a5f4005df20000a9f6000008eb0000bb000000bb
:10a60400b214000018f500000f0300001af4000053
:10a6140089f700007e0d000019f7000049fc0000d6
:10a6240046100000d2050000acdf0000c5f40000b5
:10a63400ade60000d0e60000fc0d000096ec000042
:10a6440085f100008e010000c00e00002f1e0000e6
:10a6540099040000cbf30000911300000f1d0000cb
:10a66400fa030000140d000084110000c2fa000077
:10a67400fbfe0000340900008ee7000083fd0000ab
:10a6840071f8000001f30000dc0e000029e3000073
:10a694004902000088150000fd020000e2f40000f9
:10a6a400a1eb000078f6000075f000009d15000095
:10a6b400ff0a00000f010000960b00003f0c000091
:10a6c4008d2000005a05000005fb0000221d00003b
:10a6d400fc18000008eb000005f30000b3ef0000d5
:10a6e40048e900000313000085fb0000e2f00000cd
:10a6f4009ef70000aae90000fb0e00007d10000098
:10a7040008ed0000b8fe0000bf0e0000b0fc000021
:10a7140014ed000073f1000059df00000ce80000a4
:10a724002a0900002ff00000ef0d00009b07000035
:10a7340089fc0000842b00009df30000d8f5000084
:10a7440051220000d4260000ec1100005ef6000047
:10a75400dffd0000cbeb0000a00b0000610c00004b
:10a7640005f600000bfc0000b3e8000025ff000024
:10a774006d020000f2e800000bfa0000af1b0000bd
:10a784007ff90000dff30000e0fa00000fec0000a6
:10a79400ac130000b60000000e0a00005e0d0000bd
:10a7a40095f5000050150000aa1a00006a01000087
:10a7b400bce60000a80b0000ce0700001afa000057
:10a7c4001e000000c5e90000b5fc00002fff0000da
:10a7d40007060000d2020000d9fe0000b3fd00000d
:10a7e4000f0b0000c7ff00007ddb00003a0f0000e4
:10a7f400d811000030fa00008bec00004fdf00009d
:10a804007fe400008ff70000fa170000be07000085
:10a81400d516000050fb0000ccfc0000b022000064
:10a8240070fc000030150000c51f0000950e0000ec
:10a83400cf0500001df10000d9ef000084000000e6
:10a844002b160000fff90000bef20000d8f3000050
:10a8540080e60000e10b0000c7f6000006e00000ff
:10a86400fe0a00007c0800001201000026fa000025
:10a874000ee0000048e50000ae0100009206000072
:10a88400bf0700007d1600001800000006fd000050
:10a894007a0d000088f80000150600007a260000f2
:10a8a4003c1600004200000098ee00001be6000089
:10a8b400b4060000a810000055f7000001000000d5
:10a8c400c7f0000012e70000100b0000a9f7000019
:10a8d400a4fd00005d09000028f800002afe000025
:10a8e4000eee000054ea000064fa0000891600002d
:10a8f400540900001a090000dc140000c4fc000024
:10a904009d1a0000dc130000f1010000a3140000f4
:10a9140031170000e7120000b20500004df60000f8
:10a9240060e900005c010000a60600004eee000095
:10a9340096fc00007fec00000ece00009ff50000a6
:10a9440071f80000a2f70000f7180000e101000010
:10a95400290600002bf5000014d70000aefc00000f
:10a96400b5150000c80f0000ff050000c8fe000078
:10a974009aed00003efd0000870b0000ed0300008f
:10a98400e20d0000be150000d00f0000a20200007e
:10a99400eef30000a9ec00008f100000e2fd0000bf
:10a9a4001fec0000c90c000070e80000caeb0000b6
:10a9b4001108000094f8000006fa0000270a0000bd
:10a9c400a9110000730b0000b7fb000054e1000064
:10a9d400fdfa0000001b0000b8ff00001c0f00007f
:10a9e400a40b0000cbe60000fa0700001a0f0000d9
:10a9f400ef020000cb1000006d190000390a0000be
:10aa040039fa000002f30000dbe80000c511000081
:10aa14006302000015ec00004aff00000fe3000091
:10aa2400b1ed0000a90a0000390b0000fefb000094
:10aa3400c2010000da070000edf90000dbee0000bf
:10aa4400fde70000af020000220c000094f80000b3
:10aa5400d4030000210a000041ec0000cc050000f2
:10aa64000719000036060000d71d0000081a000070
:10aa740058130000b4080000a2e7000098f9000091
:10aa840016130000010500003df3000007fa000062
:10aa940042ee00007edc00005e0600004a02000078
:10aaa40096ed000010080000a5fa00002001000047
:10aab400a7f40000f4e400004e040000c50a0000fe
:10aac4006ef90000f9f40000370a000098f3000062
:10aad40073ff00008a19000017ff0000f204000051
:10aae40007110000b81400005e06000047f40000df
:10aaf400e3f90000e8110000db02000059e1000066
:10ab0400faf5000001f1000039f00000bb0f00006d
:10ab1400010c00007eff000084f3000058fb0000dd
:10ab24007f040000c2f10000fdf900002c090000c0
:10ab3400c70f00005401000075f900002412000042
:10ab4400520b0000fa1900000f2b0000bc0c00008f
:10ab5400630a0000b20e000013040000e7050000c1
:10ab6400b0e80000bdee0000060d000063f6000032
:10ab74008deb00009bec0000fbf4000015e30000eb
:10ab840073f80000f209000057ec00005df80000c3
:10ab940089f200005e060000c9f40000ebf1000039
:10aba4004b1600005c070000cd04000008f800000c
:10abb40083010000270300003c000000eb0d0000af
:10abc400f9000000e8eb0000b7fd0000fd110000f3
:10abd4007c0a0000e60100008cf400004d0b00002c
:10abe40048fb00003df000002f040000b904000001
:10abf4002d07000002ff00002006000054f70000ab
:10ac0400b3f50000da090000851900003d070000d3
:10ac14002bf300001e070000bc0400000a00000023
:10ac24005bfe0000e40700009f05000049060000e9
:10ac3400af10000051fe0000d7ed000058f20000f4
:10ac4400a60400007b00000033f100004ef2000077
:10ac54003c02000041060000e5ec0000d9ea0000d7
:10ac64003c0f0000740900005bfe0000c7080000f0
:10ac7400b6f80000b1ee00000afd00000715000060
:10ac8400b60000003fef000005f7000011010000ce
:10ac9400b30b00006f0800004e040000a30700007f
:10aca40042080000b9f1000052fd000047f6000020
:10acb4009603000064260000d2180000dc060000a1
:10acc400a1fb0000e3170000400500000bfe00009c
:10acd40025f90000f5f70000e40300009de2000000
:10ace400e2fa0000aee7000009e7000049fe0000b8
:10acf400ff020000210d0000bce60000d6f60000b3
:10ad0400f402000024fe000017030000c607000040
:10ad1400830d00005102000092fc000060ef00006f
:10ad2400eff8000073060000ac1e00003c180000a1
:10ad34008ef5000011f800007cec0000e501000035
:10ad4400a7050000abf600009b07000012f8000006
:10ad54003ef8000025f2000096f0000094f2000096
:10ad6400a7030000b61a00004dfa00007ffc0000a3
:10ad7400e2f8000037090000ce1a00000d0f0000b1
:10ad8400f813000035020000dc0a00003e02000057
:10ad94007fff0000a9020000ed0c0000b92a0000aa
:10ada4009519000091ff000067ed000081f200009a
:10adb40010fa0000b80100007af9000069f60000fa
:10adc400a9f100006ce300002ae6000098d300001b
:10add400faed00002b1200001a1c00007608000097
:10ade4007cf40000e2f500000ffa0000551e00009c
:10adf400fa150000b90300000bfe0000baf80000c9
:10ae040021f700004eed000064f300004bfb00004e
:10ae1400281a00004b0f00002aea000016ee00007a
:10ae24007af300005b040000340a00009a0000007a
:10ae3400eb0a0000550a00001a010000eaf40000c1
:10ae44000de9000065fb00008a1300002e240000b9
:10ae5400ef0f00008cf5000089f80000e5f9000010
:10ae6400850c00009f0f00001a04000080fd000004
:10ae740028f80000f9f4000020f0000096ff00001c
:10ae8400210d0000651700003d110000e7f30000ec
:10ae940040ed0000f6fc0000cf0e0000270c00007f
:10aea400c6fb0000c0fc000059f200008bf000005b
:10aeb40029f60000d3e70000fb050000e50d0000c3
:10aec40072090000d516000054f000005ee800008e
:10aed40062f40000d7ff0000c00d000080030000f2
:10aee4006b05000035fe000009f5000077ef000057
:10aef4007df60000e710000045220000b8250000a0
:10af0400ce050000b2ed0000c7fa0000d015000025
:10af1400e0160000ee0900005f0e000005ee0000e0
:10af240040ee00009bf30000a9de00008bfa000055
:10af340093f70000f3f0000001fb000065ec000053
:10af4400ade8000041000000bb120000a1070000b2
:10af5400c001000007060000a2080000f10d000077
:10af6400affe000014e50000b20600007f170000e9
:10af7400eb0a000050160000acfd00009ffc00002e
:10af84009307000039f90000aef7000052020000f8
:10af940079f50000dcde0000e3f4000030e7000097
:10afa40073f200006c1500003cf80000eb00000098
:10afb400bbf90000f5f20000d216000007260000dd
:10afc400be17000002fa0000860f00004b030000c9
:10afd400010900000e250000b6fb00005e0d000014
:10afe4009e1400008afc000088020000160900007c
:10aff400fafb00002ef300007dfb0000eeee0000e3
:10b0040033fa0000f1f300008eed000079f4000043
:10b01400c4e400006bdd0000e5f70000a10d0000b2
:10b0240081f2000051040000df000000e5fa000096
:10b03400682300005d1e000027090000c50500000c
:10b044007d0200004beb0000eb0100000df5000059
:10b05400aceb0000af110000d9ee000039ed0000a8
:10b06400be060000670a000074070000be1200005c
:10b07400ca05000020e40000970300001d0500003d
:10b0840071fb00004f000000c8e50000d7ef00008e
:10b09400e812000014080000630400009f1a000076
:10b0a4005e0a0000eb020000090a00002cff000009
:10b0b40025020000060e0000e7fe000079fa0000f9
:10b0c400c3f5000027eb00000e100000260c000062
:10b0d4007cef0000fdfc00005a110000ac0a0000e7
:10b0e400c9030000be050000b3e5000043e9000009
:10b0f40045fa00005af800005cff00001ef800004a
:10b10400b6f00000b6fa00008ff4000072ee000002
:10b1140068190000c91c0000060a00003804000079
:10b124006af9000064ff000051030000c810000029
:10b13400590800004cf6000065f1000057000000bb
:10b144004c100000140b0000180c0000b81a00008a
:10b15400b4210000d3070000c80a000036fc000038
:10b16400b1e0000075eb00002ee80000acec00003c
:10b17400ebec0000f5ee000099f2000032ef000065
:10b18400efe300005af700008f210000061a0000c8
:10b19400bf100000ea0c00000e0a0000adf500002c
:10b1a40077070000fd1a000018e700005bf70000b5
:10b1b4003801000093ff0000cd1300003ff80000a9
:10b1c400e4070000cc1c0000fcf80000cbdb00000e
:10b1d400c2ec00003eef000067e80000f701000049
:10b1e40099ea0000e7dd0000fe010000e7f8000036
:10b1f40011fa00005509000025080000d2220000c1
:10b204009c2e0000271600007c0700004f1f000042
:10b214002d090000b7fd000039230000bdf800002f
:10b22400ffff0000f0150000c5fc00003508000019
:10b2340003f80000d7fe0000501a0000420300008b
:10b2440029d00000c5de0000d2f1000011da0000b0
:10b25400cb000000a2ff000052e4000005f1000052
:10b26400f7ea000032ef0000280700003011000068
:10b274006a150000432a00003c1900002300000066
:10b284001b1500004b05000027ef0000780e00009e
:10b2940054f8000075e9000085070000e8f7000095
:10b2a400e6f8000047ec0000cfe80000990a00002f
:10b2b400441000007bf0000020e70000ac02000016
:10b2c400f0e30000b9ff0000ed1c0000fced0000fd
:10b2d4003ef90000cffd0000bdfd0000ea0d0000b6
:10b2e400440d0000961200006d2d0000772200002e
:10b2f40027f10000a2010000780e0000b9f600005a
:10b30400cb07000038050000cee50000b8fd0000c2
:10b314008114000048020000f2f70000ecf5000080
:10b32400f9060000250d000068ef000051e8000058
:10b334001cf20000e2ef000010f80000d70000004b
:10b34400f9f20000e5ea00007e0500008d0400002b
:10b3540074ef000032fb0000270700004f200000bc
:10b36400df17000080f40000ee050000e30e00008b
:10b3740091070000520b000047110000a9040000cf
:10b384006af600007f0a0000640200007afc0000f4
:10b394003807000072090000070e0000b4f2000034
:10b3a400cbeb000054f6000035fd0000b4010000b2
:10b3b40029f7000075ea0000e0dd0000f1f100006b
:10b3c40097fc0000cbf3000037f40000c304000036
:10b3d40075180000a3180000dd160000e806000040
:10b3e400e006000042030000dbf90000130c00003b
:10b3f4008f0000009ff400001f0a000036070000c1
:10b4040094f7000028010000b4070000ae07000014
:10b4140025f70000f6dc0000f6db000036f2000041
:10b424001e09000022fd00004fed00007de4000035
:10b43400dbed0000b00b000049fe000048f90000fd
:10b44400dd12000000200000562700000821000043
:10b45400d70e0000d50b0000041a0000af06000050
:10b464007eff00006d0d00002a0300000e1800008e
:10b47400720d00001de800004fe800003ae90000ea
:10b4840093fb00008ffa0000cde200001fe80000eb
:10b49400e50000002d0900008cef00004fec0000d7
:10b4a4005eee00000cee0000280800009af8000090
:10b4b40042f60000cd180000b02200001123000065
:10b4c4006d0f0000e7010000980400003a1000002e
:10b4d400f804000030ee0000a8fa000044f3000075
:10b4e4007fff0000d90d000088f10000e5f10000a5
:10b4f4004ff20000a7ef000032fe0000def500006e
:10b5040072f60000480a0000d901000088ed00002e
:10b51400c3ea000031f4000028fd0000c20e000060
:10b52400e80a000044f70000b81600007821000083
:10b534009e1d000051230000fbf90000b9f000003b
:10b544003f050000f4070000350600004f07000027
:10b554007d03000018fc00005c03000060f00000a4
:10b56400b7e70000f4f80000c3fa000036ff00005b
:10b57400e9fa000056f200009bfd00006209000099
:10b58400beef0000e3e4000055f4000054f50000b1
:10b594004b1400004c170000acea00001ef9000038
:10b5a400231200009d090000eb130000d1030000ea
:10b5b4008bfa00008a0d0000410600002bfd0000fc
:10b5c400bbfc000026130000c2100000e00c0000c9
:10b5d40052ff00008be20000970900003e100000bb
:10b5e4009f020000dc01000052fd000028fb000067
:10b5f400b6f7000085f9000011e400001cf100001a
:10b6040060f1000053f70000040600006de700003d
:10b614003b020000e51e0000cf0700008cfd000087
:10b62400e803000065030000d70f00001e110000ae
:10b6340067fd0000edfd00008302000055090000d5
:10b6440018050000d4f9000023e70000f4ef00001f
:10b65400d30800008cf00000f60200009c090000f2
:10b6640088de00008df00000e3f700006af20000bd
:10b674009f000000a70400008008000083f8000079
:10b6840082ed000065fb0000fc1d00002b20000083
:10b69400e30700006e0f0000ef030000d900000074
:10b6a400c9160000ab110000710500008d0b0000ed
:10b6b400b00f0000210b0000d5080000c6f6000002
:10b6c40064f900007405000056ed00003eef000030
:10b6d40033fd000068e90000fdee00009501000064
:10b6e40047e60000e1e0000070fe00006002000098
:10b6f400770900003dfe0000c6f500008f1400002d
:10b70400301800009009000091090000350d000078
:10b714002bfe0000e9050000c91300005efc0000d8
:10b72400bd040000390b0000caf40000b3ed0000b2
:10b734006be2000011e90000b61600007f00000073
:10b7440069e30000dafb000026e100005efa000075
:10b754005b1900008afd00002af7000093f700003f
:10b76400bf020000c8f90000e80700006f0e0000e7
:10b77400070f0000cb1a00000dfc0000e1070000d9
:10b78400910d0000b5fe00001e0a0000f80b000039
:10b7940089f90000a9fb0000ac1800003f05000077
:10b7a4009afe00003ff2000041e300007510000023
:10b7b4002808000011f50000effc00008fe60000ef
:10b7c40063e90000b700000044f700009bf20000aa
:10b7d4004903000027f90000adfa00008f0a0000b9
:10b7e400a20600008c120000d915000077000000aa
:10b7f400b9f40000e1fb00002e0200006e0f00000f
:10b80400041d00008efd0000d7f00000c3010000fd
:10b8140065fd00007f0d0000ce0300009af10000da
:10b824009a120000a20300005ded00002bfd000051
:10b834004afa0000e307000003080000d3f5000003
:10b8440021f70000d1f10000d4ee000074010000e3
:10b8540026050000d7f000003d0200002f10000074
:10b8640023f800006bf60000b2010000fffb0000ab
:10b874005e0a0000961b0000f1040000df0b0000cc
:10b88400d20700002af1000081080000b8fa000085
:10b89400b9f300005c1e0000f30b0000f5df0000ac
:10b8a40034ed0000aff2000097f50000170500002a
:10b8b400d7f5000067ec0000faea0000b8f20000d7
:10b8c400ed0b000073140000bb040000630c0000c7
:10b8d400fb120000b4f0000015f50000170e000084
:10b8e4007f0a00003b1200000c1200003ffa000027
:10b8f400a00200000a0a0000c90500008017000029
:10b9040094ff000063fc0000821d00005f0500003e
:10b91400aeea000002f200003eee000019ed000065
:10b92400b6fc0000dcec000031e70000f2f400009b
:10b9340040ee00005f070000dd0e0000f1fa000099
:10b944001e1100005b14000069f3000029f20000de
:10b954009a0c0000c0100000431e0000e8250000ff
:10b9640035f70000b2f40000990300006ef3000004
:10b97400d10400003a04000001f90000c0070000ef
:10b9840030f60000e6da0000e6ea0000b1f8000054
:10b99400f1f70000d0ff0000cbf40000bce400008d
:10b9a40049f500006e0e0000e8130000ec130000df
:10b9b400b206000034060000bf0c00000cf80000c2
:10b9c400ecf800003a0800003811000044160000aa
:10b9d400310b0000d4fd00006ffb000093fc00005d
:10b9e40096ff0000d50200009d0200000c1100002b
:10b9f400291500003efe0000a1e8000036e4000026
:10ba0400cde800006cf400000a03000094f5000087
:10ba14005fe7000072ee000088fd00002b0b0000c1
:10ba2400490b0000e30e0000020d00009106000027
:10ba3400d4f80000a8f50000031600003d1700002c
:10ba4400ce0e00006a010000e8e800002cf70000b8
:10ba540054000000c60c00002e080000f002000094
:10ba64008509000091fc00006e04000067fd0000e1
:10ba740034fc0000e1f7000087fa0000b301000085
:10ba8400daf1000032fa0000eaf60000470d000087
:10ba94009c0d000015f7000035050000d1020000e0
:10baa40007fb0000b4ed00000bf0000016f70000e7
:10bab400160b00009a190000c3040000e3f800000c
:10bac40047f60000b2f900007a0c00000c200000d8
:10bad4002a0f0000c40c00003b030000ebe9000047
:10bae4005cf20000bced000075f2000012050000dd
:10baf40016ff0000badd0000f2da000059fa000077
:10bb0400b9100000d7100000e9ff0000d7010000c1
:10bb14003d050000d30b0000b607000074010000cf
:10bb240027020000fb090000751200002900000034
:10bb34009c000000d4ff0000570a0000b409000074
:10bb44002ef80000e1020000b6080000421c0000cc
:10bb540072080000cdf1000033f1000015f100007f
:10bb6400e60e000034f10000c3dd0000f9e400003b
:10bb74002be80000a11100008906000071fd0000ff
:10bb8400a5090000bdfa000011fb0000b6fe00008c
:10bb9400750a0000371400002a2000001312000068
:10bba400e5f10000fbfb00003d0200001916000057
:10bbb400391c00009bf8000084ef000082fa0000aa
:10bbc400f703000006f6000050ed00001dea000037
:10bbd400b4e700001ef10000fae10000bfef00002e
:10bbe40041fa00006bf9000088130000400a0000cd
:10bbf400ea0c0000c515000037090000e804000045
:10bc0400ae0200005f0400006f050000151a00007a
:10bc140083170000a903000062f80000ecec0000a8
:10bc2400140a0000bd0f0000f4f9000007fd000035
:10bc3400050200007102000045050000f700000045
:10bc44008ef200008ff70000dcf10000d9e500005f
:10bc540056f30000afef00005cf000000212000099
:10bc64005a02000051e700007503000004000000c0
:10bc7400f80b000049210000ff0400004700000009
:10bc8400dd150000cd0a000016f50000d401000007
:10bc94005ff100006a070000c5170000e3ea000036
:10bca40060f90000e3050000530a000044050000a9
:10bcb4006dfc0000fbf00000c4f4000089080000e3
:10bcc40094ee0000b3fa0000dcf6000096fb0000de
:10bcd400041f0000000c000094f700002bff00007c
:10bce400df090000eefa000040060000f7fc000047
:10bcf40027f50000a11000004df800004ff10000ee
:10bd040078fd000051ff00000c120000a11a000091
:10bd140069f700005cf3000042160000ca07000047
:10bd24006b0c0000c30400005ce7000009f5000090
:10bd340054f40000beeb0000f6f5000075f70000b7
:10bd440050e50000a0fa00006500000026e20000b3
:10bd54007304000022140000030000001a15000000
:10bd6400f3130000c102000036170000a00b00000e
:10bd7400cffd0000e305000017fe00007f05000072
:10bd84008c0c000026ff00008ce900003005000048
:10bd9400280700005bfd00002b150000e2f3000003
:10bda40007f200000ff800008af3000046fd0000cf
:10bdb400d4f300005ff20000bff50000710300003f
:10bdc400b0f30000d9ff00002e190000c2050000e6
:10bdd400380c000066070000090000005807000046
:10bde400e90a0000f9120000ea020000cf00000096
:10bdf4001a060000c60800009c05000085f3000038
:10be040025050000f8fe0000fdf80000a5f900007b
:10be1400e0e700001ded0000dee10000bff30000dc
:10be2400a4f80000b1ef0000aefb00006ff80000c2
:10be34007d06000034fc0000f305000078230000b8
:10be4400bd170000cf0f00009d0e0000410600004a
:10be5400cf0000009b070000ac0f00009405000019
:10be640023f9000002fc000004f7000022f60000a1
:10be74002ff800006bf700005f0500006b03000063
:10be84008af6000027ff0000250500009ff8000047
:10be940056fe000095ff00007dec000042f6000015
:10bea400d4ff000080f600001e03000094ff000091
:10beb400bbfe0000ad140000a601000079fd0000e7
:10bec400c41200005402000099f600006c15000032
:10bed400b909000040f100004e0300007ff40000a7
:10bee4008efb0000a9060000beff0000030e000048
:10bef4004f080000b3ec0000d9ec0000bc0f0000b8
:10bf0400b7f80000fdf90000b30d000038e80000a8
:10bf14006af700000a04000046fa00004309000022
:10bf240014130000b70600006c0600000f0900009f
:10bf3400fceb0000fe0700004c0a000040ef00008c
:10bf4400bb0a00007b0400009ff90000edfb000029
:10bf540028fd000059f5000055020000880e00007d
:10bf64008d0a0000db1b00007bfa0000cdec000012
:10bf74000b050000e103000001ed0000f3f60000f2
:10bf84001a0300009fe6000043f6000056e7000095
:10bf94008fef00002a08000005f70000d608000013
:10bfa400c6070000d60400004c0a00005c20000014
:10bfb40047120000b8fb00007b18000027030000b4
:10bfc40012fd0000d9080000edf900005fff000039
:10bfd4004400000086fc0000f8ff0000f6f20000b8
:10bfe400daec000043020000d201000077ee00000a
:10bff400c0ec00007d0000008dfa0000c8ee0000d7
:10c00400ca0500004afa000035090000980f000034
:10c01400e5f800003d1a0000560000008901000008
:10c02400c5200000f80a0000aa03000015f800006b
:10c034000f0a00000df6000002fd0000510d000083
:10c04400cef10000c0190000fbfd00009ff10000cc
:10c0540088fb0000cae20000a1f9000088fb000090
:10c06400d8fd00006ee3000015f600001305000083
:10c0740097e50000d1090000f4f90000b0fa0000cf
:10c0840087170000500c0000de0e0000981100001d
:10c0940065120000fe0d0000b91a00008bfb0000c1
:10c0a4004af50000cd0c000005f60000c4fd0000b8
:10c0b400b1f50000bef5000013fa00000f07000000
:10c0c400edfc000006e40000ec0c000031f300007d
:10c0d400b70000009f1400006ee3000026fb000080
:10c0e400ca090000fefb0000c6fc000040ff00007f
:10c0f40071f100002c0600002a0b0000a9f80000d2
:10c10400810c000017090000c30a0000acfc000009
:10c11400bdfd000043ec0000ddf800004613000004
:10c12400d2ef00009f19000028fe000035ff000038
:10c13400eb190000afe90000dffb0000a0fa0000eb
:10c144000e0900007efe00005f01000052fd0000a9
:10c154008ddc0000960e00009bf90000eaf7000059
:10c16400bf120000e7ed0000db0f000054170000d1
:10c17400bcea0000581100003816000019fc000049
:10c1840070030000f4fa0000e503000079f50000f4
:10c194007a0e00006f0500001ff200005813000023
:10c1a400e5ea0000581400002504000049e10000fd
:10c1b400561200001cf30000d3ff00008dff0000a6
:10c1c4008df6000072f200000aee000039fe000055
:10c1d40001f0000007fc00000ef7000032fa000036
:10c1e400700a00001cfb000033fd0000e81d000085
:10c1f400b8080000190400000a190000bef6000087
:10c20400240f000080110000aa0a0000f40f0000af
:10c21400a3ed000013fd00003801000046ff0000fc
:10c22400cafb00001fef0000b00100009dea0000ff
:10c2340081ef0000bf0200000fe6000005050000ca
:10c24400fc00000055f50000df01000082ee000054
:10c254001a130000870c0000a5fe0000080f000060
:10c264002dfe00005f170000ee130000a40a00007a
:10c27400f9090000ebe9000033130000f3090000a2
:10c28400ecf50000200900008bea00001108000012
:10c2940043fa000007f00000c90500005ff0000049
:10c2a40060010000dfeb0000fee300003cfa000048
:10c2b400dcf70000050a0000c1020000f0ee0000f7
:10c2c400bbfb00008d06000061130000f7080000ae
:10c2d4000e060000c5150000950300006e1b00004b
:10c2e4007213000007fa0000d10800001af50000dc
:10c2f40095020000fffc0000f9ed0000d40f0000df
:10c304004907000079f900008bed000088eb00007c
:10c314009c02000030f600006a040000b4f800003b
:10c3240076ed0000b00d0000b3f800000208000034
:10c33400cdf80000b8e90000220d0000ccf60000a2
:10c3440044040000860600005dff0000230d000089
:10c354008f0400005f11000032fc0000d2fa0000dc
:10c36400101300006ffb00009cf70000c1fc0000ec
:10c374002dfd0000361400004c0600003cf20000c5
:10c3840084fa000062ed000003050000e3090000e8
:10c394000cfc000034030000a6ed00004601000080
:10c3a40003f60000edf10000200700001dff00006f
:10c3b4008e120000210400008c0400000a0d00000d
:10c3c400910a000023140000750200002aee000008
:10c3d400b6f70000a00a0000460b0000990900000f
:10c3e40028ee00005b0300002c0c000062f9000042
:10c3f400ca06000068ea00001201000005f8000007
:10c404009cf900003306000055db00007b000000af
:10c4140020ef000048f500006b000000b1ee0000c2
:10c424008c1e000091fc0000fafd000040fe00009c
:10c4340028ef0000a9240000591600007f16000010
:10c44400100a000022ef0000790d0000d40500005e
:10c45400ac010000c9f8000097f90000d50c0000f9
:10c4640012f2000014fe00002af90000feeb0000a6
:10c47400f20b00009bf000003afe00005d0000009b
:10c48400f9e300007f110000d4f4000023ee000063
:10c494003d080000700600007e1e000050ff0000f2
:10c4a4000e08000050000000f7f800008a27000082
:10c4b400c0fe00008d0a0000c5070000c5e00000b2
:10c4c4000d1400004dfa0000dbf30000ca14000054
:10c4d400d9f900005b050000e6f60000a8ea0000b8
:10c4e4006cf700005ef3000058fc00000be800004d
:10c4f40086ec000022000000c7fa00006c13000064
:10c504006afc000037eb0000d41600005c04000055
:10c51400f20b000082100000b9f600004018000081
:10c52400f60e0000ac0e00009e11000078fd000025
:10c53400010000001efb0000810a000059f0000009
:10c544001dfb0000101a00003aed000029f2000063
:10c5540025e5000030e9000009130000e0020000b6
:10c56400260700007efc00003de6000087f5000081
:10c57400160e0000c302000064f000001d0000005d
:10c584009e0900000afc000067020000c20e0000c1
:10c594008cfb0000d91900005d00000044fd000080
:10c5a40006190000e6e90000eb0e0000bff80000e9
:10c5b40005eb0000a40600003b090000521d00002a
:10c5c4000ee700003beb00006ff0000012e70000f4
:10c5d400591300006d020000c2f800008efc000038
:10c5e40011e300001e0000008f0d0000fbfd0000a1
:10c5f400751800009a1300005e090000e6030000ad
:10c60400cf040000c2140000a70600009a02000034
:10c61400e3f7000012f4000088060000d1ff0000d8
:10c62400561500000c0000007ce10000cb0c00005b
:10c6340086fb00006c000000e3f700000aed000038
:10c64400bc010000f6ea00008908000092f5000031
:10c6540035fb000081f9000000ea000072100000c0
:10c66400eeee00008d0300004a1900007e01000078
:10c6740069f50000e6fd0000700a0000aa1a000037
:10c684000b1f0000e80700009906000096f0000068
:10c6940061ff000094fd0000ed070000b6fe0000fd
:10c6a40074ec00001b0c0000c3e5000062fe0000f7
:10c6b4000108000068f600007afd0000b2ea0000fc
:10c6c400e0ec00003efd0000dc030000c6fd0000bd
:10c6d40045090000cc000000ba0300003f07000039
:10c6e4004c1d0000e1ff0000f7fd00007c0d000080
:10c6f400e9eb0000871d0000affc00003c090000ce
:10c70400f7090000fae40000d1f900004afe000035
:10c71400361a00009ef90000980b0000c4fd0000ca
:10c7240037e70000a502000037f90000fbf2000023
:10c7340006f40000e6eb000079e90000830b00003a
:10c7440071f70000630f0000ff0f00006ff200009c
:10c75400aef9000035030000d8200000310b0000c2
:10c76400941d00000f08000082f30000e20f000097
:10c77400b3f80000f00a00002711000087e200006f
:10c784007b010000dd0a000048ea00008c0e000076
:10c7940065f70000e5ec00008bf0000041f50000b7
:10c7a40067030000effd0000ac0900005ff100002a
:10c7b4003c000000def40000acf000009a1200001f
:10c7c4000a02000043ed0000fb0600007b020000ab
:10c7d4001ffb0000212800003d000000b6010000fe
:10c7e4009eff000040ed0000d20e0000410e00004c
:10c7f4004105000074f800002e12000078f40000d7
:10c80400f3f9000089180000a9e80000db04000027
:10c8140086fc0000f7d20000d5fe000036030000bd
:10c82400d1ff00003e0600005bf3000041f700006a
:10c834001a0a0000891b0000eaff0000a911000089
:10c8440057150000baf300003f1800004908000023
:10c8540006e90000a80e0000d6f300001ee4000064
:10c86400f4160000e5f000000a0d00009508000031
:10c874003ae5000099f80000f1eb0000961400007e
:10c88400ddfe0000dc15000022f40000eedb0000f9
:10c8940094160000eee5000058fc0000580c00005f
:10c8a400c4f00000e2010000cf03000037f30000f1
:10c8b4008e1500008e060000f1fa000074060000d8
:10c8c4005bf80000060c00007d0a0000b41c0000a8
:10c8d40063f5000024050000990b000048f00000f7
:10c8e400051400009efb000057f4000035f800001a
:10c8f40035f40000cff80000d1190000f7f0000073
:10c904007af100001b0600005ae300004303000014
:10c91400a80400001614000045f100000304000000
:10c924007600000021e90000712d00002af50000c6
:10c9340075090000d00d000063db0000220c00002c
:10c94400ad070000d005000055020000a7fa000062
:10c9540090f400007bef0000be1e00003d020000ca
:10c96400dd0300002112000018ec0000630a00003f
:10c97400f6f200008cef000027030000c6f200006e
:10c984008fe900009efb00006208000073f80000bd
:10c99400d00b0000fdf200005dfe0000fb00000073
:10c9a4006f1600000f2300009d060000a81200006f
:10c9b4001ee300009c0e000029fc00001efd000088
:10c9c400f9210000edea0000ca01000073f1000043
:10c9d4001cfd00009a020000b4010000e5f500000f
:10c9e40093ec0000d6f10000d3ef0000ca11000060
:10c9f4006ff80000250c00003ef5000014ff000055
:10ca0400230100008cfd0000f9200000beeb0000b3
:10ca14004012000019eb000075f900002026000008
:10ca24002dfe00007815000054ec000033f60000e1
:10ca34009f000000df0000002712000088f70000bc
:10ca440065fe0000f6fe00006efc00000e01000012
:10ca5400f6f80000be02000067fc00005be800007e
:10ca64003af50000b2010000720d0000f30400006a
:10ca74008ff000006df60000c4f80000fc04000014
:10ca84009b2100006f1300001a05000067020000dc
:10ca940024ff0000f00b00006df90000c505000044
:10caa4009fff000075f600001bf80000d9ef00009e
:10cab400e90f00005dfe000029030000a4fe000051
:10cac40011e5000098020000cf0b0000620b00008b
:10cad400ec040000e3ee0000a4fa000037020000ba
:10cae400fffd0000040b00004ffb0000affd000041
:10caf400b3ea00009ef7000021130000f0fa0000e2
:10cb04004308000067fd000036fb00002cf5000020
:10cb1400e9fb0000cf1100004d1100003f000000b0
:10cb2400fbf500002c08000026fd000002110000a7
:10cb34003a0e000073fc00003ee90000d6f8000045
:10cb44001f11000091ff0000a00b0000f6f100008f
:10cb54005dfa000074ef000026f30000d50a00001f
:10cb6400b8f90000930600000103000082060000eb
:10cb74009df50000f3000000f9150000290d0000e8
:10cb8400e9ef0000b5f10000bb050000b5020000ac
:10cb9400081600009ef1000091f8000085f50000e1
:10cba4009afa0000261a00009ffd00000505000007
:10cbb40076fd0000d308000035f70000f1f0000016
:10cbc4009f09000020fa00004bfb0000b9ed0000b3
:10cbd40083f1000043f800001e0c0000e91200007d
:10cbe4004500000032f60000e5f50000a71500003e
:10cbf400f81100005e080000f6010000670500005f
:10cc040092050000eaf800007d0a0000bdfc000067
:10cc14000b040000af00000009f0000020fb00003e
:10cc240017f600001709000014050000f6f20000d2
:10cc3400aced0000c7fb0000e2020000620100004e
:10cc440081040000aef40000f5fb0000e7050000dd
:10cc54003d130000230100003b0800008501000093
:10cc6400f8f20000500d0000a8f300007c09000059
:10cc7400690300005dfc0000baf70000c4ef000087
:10cc8400fe040000acf50000d0190000e9ff00002c
:10cc94008bf2000020000000dff90000c10f00004b
:10cca4006708000039fb000090f00000cb0400008e
:10ccb400a0f40000ef0500004c060000dbf30000c8
:10ccc400060b0000e3fa0000110900001400000044
:10ccd400390f000039100000b8040000cb08000030
:10cce4004eed0000e9040000640500007af600003f
:10ccf400c6f9000067f3000091f3000087110000fb
:10cd04000f030000f4f30000b3fd000078f200000c
:10cd1400c90d0000bd01000040020000cf03000067
:10cd24009401000085fe0000d7ed00006c0a0000ad
:10cd340043f9000032060000010f000040eb000040
:10cd440017f80000abfd000078fd00009309000017
:10cd54008efb00008df500000cff00004405000070
:10cd640063fe0000c0fe0000b20e0000c8f6000022
:10cd74008d1000002c0f000006fa00004d11000079
:10cd8400380200004c020000e2f90000b4fb00008d
:10cd9400d2fd0000fd090000b3f6000036eb0000f0
:10cda4009eff0000eeef0000e3fc000047020000dd
:10cdb400d70e0000bdfb0000860900002f0a00000a
:10cdc40053f70000fa0c0000d1f10000ba02000091
:10cdd400460300009efc00003803000075090000b3
:10cde40080ff0000f6f90000a40900008ced0000ab
:10cdf4002bfe000099090000d30a0000d9010000ad
:10ce040074fe0000fffd00005aef00003afe00002f
:10ce140017f100007a020000fefe0000e7f20000b5
:10ce2400ec07000002010000c9fd00009ffd0000a6
:10ce3400a0080000a9fe0000480000009b080000b4
:10ce440020fe0000301000001c08000017ff000046
:10ce5400f505000032020000980000007107000090
:10ce6400280200004dea00008b04000006020000c6
:10ce740014f80000e407000008f3000024fc00009c
:10ce8400f3f60000e2ef0000adf9000049010000f4
:10ce9400310600009406000008150000a6010000f9
:10cea40006010000bb1100005700000006f8000056
:10ceb40051fe000098fa0000e80700005d09000038
:10cec40088f100007ff3000029f500007ff00000e6
:10ced400b9fa00001b10000041fc000038040000f7
:10cee400af1700006af40000dbfc000087000000bc
:10cef400b7f800006e010000c2fe000036f8000022
:10cf04005f0400004c0800007aff0000950e00004a
:10cf1400b6020000bef50000ca070000c6110000fa
:10cf2400bff70000c3000000ad0800000ff90000c7
:10cf3400220d000050fa000024f9000086fd0000d4
:10cf440028f60000c8ff000048070000b2fd0000fa
:10cf54004ff200006815000045fb00002cf20000b1
:10cf64005e04000009f400007c0700000efc0000d1
:10cf74006ff60000d7f90000660000007b0c00008b
:10cf84002007000007060000f1ec0000aeff0000df
:10cf9400e90b0000c9f30000aa01000042000000f0
:10cfa40026fd000017020000b5f90000d1f10000d1
:10cfb40035ff00001a09000098040000e81400007e
:10cfc400ea0900001f020000c5150000f80a00006d
:10cfd4007ef4000068f9000013000000ccf80000a3
:10cfe400ec030000cef00000eaed0000cb040000ea
:10cff4004cf0000034080000720a0000dff4000066
:10d0040061080000ac0400008a030000fcf7000083
:10d01400630200004306000098fe000019020000ad
:10d024003bee00000e0700006cfd0000f8fb000062
:10d034007210000060fa00002dfc0000740500006e
:10d04400f3100000d4fa0000a4f700003d01000032
:10d0540073fc000027030000b4f60000fefa000091
:10d06400b200000006ff0000f6040000ee0b000012
:10d07400a3f700004cfb0000ff0d000037fc00008c
:10d084003ef8000007fa0000c60500007208000020
:10d0940041ff0000fbf4000014010000230700001e
:10d0a40044ff0000bb130000b7ff00000df80000b0
:10d0b4000f0500000c080000e9fa000051eb000025
:10d0c400e6040000bcf80000d2fc00000ff50000ec
:10d0d40082e80000a8100000bdfb0000f70b000070
:10d0e40040140000d8f50000c40c000067080000dc
:10d0f400870a000098f7000053f40000d70c0000e2
:10d104009ffd00006cff000052ed0000e1f70000fd
:10d11400570a0000e2ee0000dc03000053070000a1
:10d124008cee0000310e0000e511000089f80000cb
:10d134005afa0000a9fa0000c6040000f100000039
:10d144003ff80000b9f6000061040000bf0b0000c6
:10d1540010fa000030100000fd020000daf00000b8
:10d16400651300006006000085f500002708000034
:10d17400a6040000e3020000110200006ff20000a8
:10d1840032fd0000540500002c0100003cfc0000ae
:10d19400a90800008afc00006cf400006d17000070
:10d1a40029f500006af1000048ff000028f00000a3
:10d1b4003204000042fc000021f60000b906000021
:10d1c400f608000093f7000004080000740600004d
:10d1d400aef50000470800001006000046fb000002
:10d1e400f1f800004e040000f1fc0000dd03000033
:10d1f4006ff800008eec0000900c0000fbff0000b4
:10d20400b0fd00002f0e0000a606000089f7000004
:10d21400080e0000280c00001af70000b1060000f8
:10d224001efb0000b20000007102000052f8000072
:10d2340004fe0000bb080000d3f7000069f50000fd
:10d244001e0e0000e9f00000db04000019140000c9
:10d254003ffb000083f90000bdfc0000360700001e
:10d264007dfa00007eff000008f700009c0000002b
:10d27400c608000033ee00009008000074060000a9
:10d28400d3f7000063070000c4080000c5f80000dd
:10d29400fdf900005d0500001dff00006d010000a8
:10d2a400bef30000f6fc0000290700002bfd00007f
:10d2b40003ff0000f00300008c080000adf800003c
:10d2c400160e0000af030000e2ee000009070000a4
:10d2d40051f8000062f9000031fc00007afd000002
:10d2e400d40700001107000013fc00004dfc0000ef
:10d2f4009910000042ff0000ed0300003d0e000005
:10d304005af700002ef500007b020000f6fd000035
:10d31400caf800004b0100001df90000dfff000007
:10d324005cfe0000bff80000870b0000d40c000076
:10d334001cfd0000200000007e0a0000f6fc000036
:10d3440044fd0000140500000dfc00002ef900004f
:10d35400fe03000048f800005dfe0000c1fe00006e
:10d3640029ef0000700900000afb0000aa00000079
:10d37400a00c0000bb010000c6ff0000abf50000dc
:10d38400d804000004fa0000150000007d06000027
:10d394004dfa00008dfc00002ef900002b01000066
:10d3a400f3090000e500000092010000c914000028
:10d3b40070000000a4fc00004c060000db06000026
:10d3c400f6010000f4f500004fff0000e9f9000049
:10d3d4002c02000005fb0000f8010000300d0000e5
:10d3e40047f90000d5020000dc0000003cf3000017
:10d3f40047f90000dd000000fcf600005fff0000bc
:10d40400d0fa0000fcfd000080060000fdf50000dd
:10d414003d05000079000000280500009705000084
:10d4240014020000a0060000c6f4000082010000ff
:10d434005c0500002b000000effc00000f0300005f
:10d444007104000014f7000090fb00009600000037
:10d454009e09000066040000a5f800003c020000dc
:10d46400d1010000aaf80000e2030000d20300008a
:10d47400ea0500002803000053fc00002906000010
:10d484003ef2000058f80000ef0300004dfc0000dd
:10d49400da03000079040000fe06000042070000e1
:10d4a400dffc000028f800001d0500005df9000005
:10d4b40024fd0000dc00000014f50000b0ff0000b3
:10d4c40075fb0000a009000018fd0000fcfb000033
:10d4d400e70a0000b4fc0000940300001cfc0000f8
:10d4e400670600001708000080f90000c1fb000077
:10d4f400d0020000cb01000058f70000940c00009b
:10d504001f03000081fc0000d107000029fa00007d
:10d514007dff0000b2f500004af500006400000041
:10d5240071fc0000a0fb00005cff00004708000045
:10d5340095fe0000e5010000ca070000fa0700009c
:10d5440019040000a8fc00001403000078fa00008d
:10d55400960400009a03000082030000b802000051
:10d56400d3f100000d08000061fb00001ff2000071
:10d574006d060000c9010000760100007c01000076
:10d58400a8fe000047040000abff000094fb00006d
:10d59400ce0400001dff000047fb00008c000000cb
:10d5a4002e05000020f500001bf500009805000082
:10d5b4001afe0000130400000a0100004c020000df
:10d5c4000004000007fc00001efd00005f030000d3
:10d5d40055ff00004af70000430400004efc000021
:10d5e40017fa0000ae020000df070000ce020000c0
:10d5f4009a000000a9050000b5ff0000020a00001f
:10d6040092fa000065020000e40700006bf40000d9
:10d61400ef070000d40100005cfe00009405000048
:10d6240026fd0000cb050000a400000057fa00000e
:10d634003702000043f90000fbfa0000c1f70000c4
:10d64400bcfa0000d2fd0000cdf10000d7040000b8
:10d65400d5000000b5ff00003304000061ff0000a6
:10d66400b40b000068040000dffc00001e01000091
:10d67400d3060000e9fc0000f90300005f04000089
:10d6840024f50000a000000073ff00009bf80000d8
:10d6940070fb0000420100009efe0000d60800005e
:10d6a400eefe0000caf50000c30a0000b1fc000051
:10d6b40092080000a7060000d8f60000aa050000a2
:10d6c40026fe0000df0500001efa000084f40000be
:10d6d400f004000045000000570a00003bfe000073
:10d6e40075fd0000210a000097fd0000a6fd000062
:10d6f40021ff00002bfc000033fc00002609000081
:10d704007cfa0000f1f30000b601000051fd0000b6
:10d71400ca090000e1fd0000f0fb000079020000ee
:10d724005cff0000ccff000050ff00004f01000030
:10d734007efb000070090000cb00000086020000a0
:10d7440087fa0000a1fa0000960e000003fd000015
:10d754007d01000088fd0000310400008bfd000005
:10d76400fbf7000098fe000053f2000013fb0000da
:10d7740059030000d708000011f900009e030000bf
:10d78400d0060000040500008e08000007f8000021
:10d794000b0a000052010000430000009d05000038
:10d7a40051fe00008dfd000053fb0000a0070000a7
:10d7b40065f700008bf2000066fd0000e603000040
:10d7c400240700009cfb0000fbfe00009f010000fa
:10d7d400ee0400003d030000e8fd000056060000d2
:10d7e40034fb0000710000004009000032f2000028
:10d7f400fbfa0000f40300003e00000073fd00008b
:10d8040046f6000026ff000097000000a601000075
:10d81400fafc000075fc0000fafe0000ef020000b4
:10d824006b070000b9fe00000cf8000006f80000c9
:10d83400b80e00007a050000deff00009a06000022
:10d84400ba010000ad08000009f8000078ff0000ec
:10d8540062ff0000720300005809000012fe00007d
:10d8640093040000bff80000860300002f080000a6
:10d87400f0ff000006fb000026f70000c0010000d6
:10d8840009fd0000ebfd0000b5f90000d4f600002e
:10d894001dfc000079fc0000b00100003fff000007
:10d8a4003b00000011080000290700006ffe000083
:10d8b4007efe00001004000022020000f7020000b7
:10d8c40062fb00003bfe0000e40300008dfe00004c
:10d8d400f204000081f7000060f6000080f8000008
:10d8e4008bfe0000ec0b00000bfb000082fe00002e
:10d8f40006fe0000f2020000ee05000044020000f3
:10d90400430a000052040000a0030000c5fc00000c
:10d91400960100003bfe0000ce020000fe0b00005a
:10d92400f7f7000069fa0000b9ff0000f6fe0000f6
:10d93400c60500004efe0000ddf500005c0000009e
:10d944007cfd000074fd000005040000dff8000009
:10d95400a1f90000e9010000ff020000a2fc0000a0
:10d96400fc0100004d0600003bfb000026fc00000b
:10d9740000fe000091fb0000110a00006707000090
:10d98400a1f80000e1ff000029010000ec02000002
:10d99400a20a000032040000a5f8000020000000e4
:10d9a400defc000019fe0000890700005dfa00009b
:10d9b400e5fd00007dfc00002ff80000e5f9000003
:10d9c4003f0700002b0a000084ff00005004000001
:10d9d40029fc00005dff0000550100003c0400002c
:10d9e40071020000410300001bff00009bfe0000c9
:10d9f400f50b00004bf400005a010000c7fd0000c5
:10da040074f3000076020000affe00004d07000032
:10da14007cfa0000d2fe000089fc00005e030000d6
:10da24008109000033fd0000ba0b00006ff700000d
:10da3400d9f800003602000068fb00000b05000066
:10da440039fd0000f9fc000071fa000049f90000fa
:10da54001b010000c0ff0000500b0000cbfd0000c4
:10da64005df20000d00b000090fc00007c00000080
:10da7400c70b0000f9f50000eeff0000ff010000f5
:10da8400c1010000d4060000db050000dcfc00003e
:10da940022ff000080030000d6f50000dd0a00002c
:10daa4001d0a0000d0f50000e5ff0000a4040000fa
:10dab40074fd00006a0400005905000034f70000fa
:10dac400a2fe00000bfc00001dfe0000f706000093
:10dad40043fc0000d4f30000c00000004dfc000033
:10dae40063f1000013100000d106000081fd000066
:10daf4001a020000fcf7000025010000cf0400001a
:10db04009f060000f50200000d0600004df3000022
:10db1400affc0000b90c000029f600007001000001
:10db240039fa000051fb000098fb0000f6fc0000ed
:10db34008c0b0000a1fb0000ca010000d7fa000012
:10db4400860200001f0b000001fc0000fd0b00001a
:10db5400b5030000c3f60000830100005606000070
:10db64008dfe00001e01000074fe0000c5f60000da
:10db7400420000000dfa0000bc080000a00b0000e9
:10db8400c9f5000013f9000058010000c3010000aa
:10db940000fb00000906000078020000c9f800003c
:10dba40059000000f2000000510300004000000092
:10dbb40019ff000062fd000097fb00008ef90000d1
:10dbc40036000000e20f00004e010000a2f7000042
:10dbd4005104000043ff0000030000007b09000023
:10dbe40042fc000041f9000069fd000027fc000030
:10dbf400350c000041fe000044f40000b9050000ab
:10dc040098f8000090f80000110200003b0b00009f
:10dc1400d308000022fc0000df0600008ef900009b
:10dc24007bfd0000bc0900005b01000078030000dc
:10dc340067fa0000dffe00005d090000b103000088
:10dc440020fa000052fe00006ffc0000e7f1000023
:10dc54000cfe0000e50400004c020000ebff000095
:10dc640064ff000012000000f4ff00008fff0000ba
:10dc7400c80600006609000062f2000023f90000f3
:10dc840086060000eafe00005a050000fa000000c3
:10dc940041fc0000d9f50000a0f500006a02000074
:10dca40076030000de02000086fb00001600000080
:10dcb4004801000090fa00005f0b0000910600008c
:10dcc4002ef9000054020000220000006d00000044
:10dcd400260400006c030000fb05000057ff000051
:10dce400b3f7000069fe0000c40d00005eff0000f1
:10dcf40037fc00004105000006000000ae030000f0
:10dd0400e40200005e0800003df3000012f700008a
:10dd1400f1fb000026f90000a20a0000b1fa00009d
:10dd2400cb080000e7f8000004f10000eafd000061
:10dd3400edfe0000c90b000062fc0000910500002c
:10dd4400c6f9000047fc000033070000b5020000dc
:10dd5400e80a000001f8000063010000d405000097
:10dd6400e7f8000061fe00001f0600008c000000c0
:10dd7400c2f9000032f90000f0fb00009c02000030
:10dd84007cfd0000d6ff000008fc000093000000aa
:10dd9400c704000008070000560e0000f5f3000059
:10dda400e4fa00008f08000060fb00001306000086
:10ddb40054060000bcfe0000e6fc00004efc00001f
:10ddc4002afd000076020000fe070000d8000000d3
:10ddd4004803000060f9000020f40000d9070000a7
:10dde40079080000efff00003ffc0000c8f90000c4
:10ddf40087f50000cbfe0000560400006bfe000017
:10de0400b202000028fc0000dffd0000b80300009f
:10de14003ffb000021000000650a000053fd0000e4
:10de24009afc0000d7080000edfa0000ee000000a4
:10de3400c5030000dcfa0000a3040000d7ff0000c3
:10de44005302000099070000e2fd00002af60000da
:10de5400e0f90000660400000a0500001701000054
:10de6400c0fe000082f90000cbf90000630200004c
:10de7400470200008b0700003d07000099fe0000e8
:10de8400c601000042f700009bfb0000540c000098
:10de940014ff000026fd0000b000000017f600008b
:10dea400cbfe00004e05000072020000bb01000022
:10deb40090020000f4ff0000ee0200006b06000078
:10dec4002ff7000060000000c70000009afc00006b
:10ded400dd0100001cfa0000eafe00007bf80000ef
:10dee40046f90000dcf800000b010000bb0700004d
:10def400fc0100009206000016f800003dfa000044
:10df0400f4010000c20700005f0300009c00000051
:10df140035ff0000ccf70000a8060000fcfd00005f
:10df2400920a00001c0800006dfd00005804000067
:10df3400d4fb0000a106000031f900009e08000097
:10df44003e030000bef50000420300007ef4000022
:10df540073040000bffd0000f7010000040200008c
:10df64007bf90000e602000006fe0000e205000066
:10df74007af5000003ff0000d401000093fd0000c7
:10df8400d7040000dbfc0000cf03000057f80000ba
:10df9400e4010000f1fe000099020000ec0b000017
:10dfa400c2f80000fc050000a0fa0000fff9000020
:10dfb4009c050000df0100005801000044f7000048
:10dfc4004afe000024f9000004010000ec070000f0
:10dfd400440100003201000025fa00007f03000024
:10dfe400abfe0000d402000009030000e2040000bc
:10dff400e1050000cbf40000ee0900002ffe000054
:10e00400f9f90000130100002df80000df050000fd
:10e0140093030000ac040000da00000009050000ce
:10e024007bf300004df800003d06000099f6000067
:10e0340097090000b1f80000d3fa0000c9fc000001
:10e0440013ff0000660a00009bfa00002509000087
:10e05400e6fa00003c010000bc02000016fc0000cf
:10e064009e04000077000000fb02000049f7000056
:10e07400d4040000ebf900009302000091060000b4
:10e0840036f700008d0d00005cfa00000e0300005e
:10e094002108000019f90000ceff0000a2f90000d9
:10e0a4003bfe00007c080000e505000017fe0000b0
:10e0b4007c0600005ffe0000d7fd0000c2fb0000ec
:10e0c40017fc00009708000036f90000470900001b
:10e0d40027fd000033f60000610c0000fbf6000091
:10e0e4006500000061ff00009ff3000088ff00004e
:10e0f40040fc0000d2fd00006dfd0000380200006d
:10e10400b6fb000042fd0000940b0000cdfd0000b2
:10e114006800000049ff00007d05000022060000a1
:10e1240013fb00009e01000017fd00002108000001
:10e134007efd0000cffe000014050000fffc00007f
:10e1440029060000f3fd000006010000b1fc0000f8
:10e15400f4fd0000a0ff000095fe0000390000005f
:10e16400fff900009502000063020000e3040000d0
:10e17400d00000006bfc0000a0050000860b00002e
:10e18400a1fe0000b1f800006aff000005000000d5
:10e19400010f000018ff00008bf6000026060000a7
:10e1a40059f700008afb00004200000034f7000029
:10e1b400bd01000057fd000094fd000007ff0000b2
:10e1c400bcf70000530200003c04000043070000b9
:10e1d4008cfd0000fcf50000720200004aff000004
:10e1e400c8020000bc070000d5f600008001000052
:10e1f40039120000dafb0000f9ff0000c1fd000045
:10e20400defb0000ac0c00003703000045010000f9
:10e21400bdff0000fff80000bff60000240300006b
:10e2240022fb0000e7ff00006c0800008ffc0000e8
:10e23400b803000067f200005bfe00003203000038
:10e244000f070000c405000084f20000ab060000c4
:10e254005ef8000065090000e808000056f80000b8
:10e26400f7080000e3fc00000a01000031f9000097
:10e274008dfe000028fa000056fe00000e0c00007f
:10e28400dcf400003107000034fb00000af9000050
:10e29400a50800001bf40000f100000007040000c2
:10e2a4005c0c0000b8020000b4ff00002102000072
:10e2b4007ff60000ee120000ba000000dc0300004c
:10e2c4001df80000e6eb0000180700006cf40000e5
:10e2d400fe07000022f90000a1ff00004206000032
:10e2e400b8ed0000c70700003efa00003d10000032
:10e2f400db120000d1f6000006ff000045f4000028
:10e304003100000079080000bbfd0000b1fc0000f2
:10e31400a5000000810b0000dd03000077fe000073
:10e32400a3fe00003bf700001f0900008302000069
:10e33400f2fe0000b703000034f500002cfb0000df
:10e3440072ff000054fd00006efc0000140e00007b
:10e354005303000006fc000037f40000c3f0000083
:10e36400660f00007a0c0000a80c00008cef00007f
:10e37400e0f6000003fa0000d7f8000029120000bc
:10e38400a0f10000f50c0000fb060000a8fd000051
:10e39400de0500000bf30000870a0000d2f5000040
:10e3a40050f400002105000052f800001dfa00009e
:10e3b40030020000bbfe0000c7fc00002df400008a
:10e3c4002d070000a5210000e209000087130000ca
:10e3d4009cfb00003afc0000201300002bf7000017
:10e3e400b30f00004fe900007be300003b05000091
:10e3f400b4f40000e8090000d7030000240500007d
:10e4040059f600005ef400003e080000bcff000066
:10e414002d0c0000560900007e070000bbf300002d
:10e42400dbe2000035e90000f7130000a01400004f
:10e4340027ed00004405000057f30000120e000011
:10e44400dd0e000015f20000e30500003cf30000bf
:10e454000a140000060300004cfa00001e05000028
:10e4640088ea0000860600008f0000009d06000078
:10e47400820d0000c9fb0000ed06000078000000da
:10e4840090f4000053f9000012fb0000fd0b0000a3
:10e494004f1000005cf00000cee200006bf80000ba
:10e4a4009a15000074040000ff05000095050000a3
:10e4b400f2f10000d00c0000c10300006102000072
:10e4c400b6010000a4ea000002f8000033020000d4
:10e4d40007f80000a0f800009c0b0000cc0a000024
:10e4e400510400009d020000f4f5000067f30000f1
:10e4f400f8160000651a0000970200005603000099
:10e50400f0f40000e10d0000c6060000cce50000b8
:10e51400b9f800008bf5000006ff0000620f000050
:10e524000f070000d1e90000cce20000f002000077
:10e5340093000000e9f90000fd0e000072120000d3
:10e54400710c00006f060000a8ee00005eff0000e2
:10e55400d40600000a0100002c1600006feb000036
:10e5640037e50000f3fc00004b050000c412000076
:10e5740059f2000093f80000d1f700001a040000db
:10e58400bd11000057f30000f90d000099ff0000d1
:10e59400d9050000dc14000072ee0000380c000005
:10e5a400830d0000e1f6000038f8000048fa00008e
:10e5b4000c000000c8ff000057fd0000b3f6000087
:10e5c40009f900002af80000960f00008f0c0000e3
:10e5d40000030000f2f7000008e80000e60e000067
:10e5e40099070000e2050000a4f9000093f0000080
:10e5f40088fe00004fe70000bbfa00004b04000057
:10e60400fe1a0000220d0000b4f2000039010000df
:10e614007df100000f0b0000590c000075fe000096
:10e62400080a0000e3070000090300007106000067
:10e6340096080000f0f8000051f20000dcf0000041
:10e6440065040000890200004ef700001cfa000077
:10e654008e0400005e160000eef7000088fd000046
:10e66400a60a0000b7ff00004afe000095f2000071
:10e674003e070000eb080000f201000018fc000057
:10e68400efeb0000eaed000065f300005a10000013
:10e694006a180000be090000610900003bf8000090
:10e6a400e1ee0000ba04000012fc0000a6e900003c
:10e6b400c3000000e60b0000110800007efe00000d
:10e6c400ab0100006d1300001e0c00005dfd000096
:10e6d40019ef0000d1fc0000cefe000068e9000044
:10e6e4001cf9000029f6000051fb0000c1fe0000e7
:10e6f40063f900004f0f00000af800008e000000cc
:10e7040085120000ff1200006110000073f8000081
:10e714005b09000070f70000ecf90000f8ff00004e
:10e7240041f600007e0f00009d0b0000f702000080
:10e7340046f200002afc0000cf020000d0100000c6
:10e744000009000074f400000409000012f5000040
:10e75400edf900003bff0000bd0900000ffc0000c4
:10e7640041e60000faf900008bef0000bcf5000060
:10e774000ef60000bf1700009419000036fa0000de
:10e784007b020000b807000083100000adf2000017
:10e79400b5f900001cfe000051f900001210000041
:10e7a400e7020000ebfd0000b7f5000012f50000e1
:10e7b4003208000085080000c3fc00007e0700004a
:10e7c400d8fb000095ef000030f900001bfa0000b0
:10e7d4008507000083fb00008e0b00004b07000040
:10e7e4002fee000034060000cd130000521a000082
:10e7f400a7f30000f4df0000b3000000e20500000e
:10e80400f9fe000040060000e2040000a7fb00003f
:10e8140062fa0000240200007b14000046fe00009f
:10e8240090f900000512000062fe00004fef0000a6
:10e83400a5eb0000e1f50000e90700005cf600002c
:10e8440035050000c30b000089fe0000051c000014
:10e85400d2fb0000d5f3000019eb000020f7000004
:10e86400a12700004ae70000a8f6000003fc00000e
:10e8740028f00000a30b000004ff00002c1d000082
:10e8840071fe000044f60000120b0000430000007b
:10e894003cfa000064f40000be1f0000eb17000007
:10e8a4009bec000080fc0000f3000000de0400008c
:10e8b400b8160000f2fa00009dfa00007bfa00008e
:10e8c400dcfb00009910000079ef00000aeb000067
:10e8d4000bf10000befc0000fcff00006ef4000021
:10e8e400c00500003bf80000860600001707000082
:10e8f4000af5000005060000300900005a1a00005d
:10e904002b070000d4f6000033020000470c00007f
:10e91400c3140000e7e7000011e10000e7f0000085
:10e9240043ff00006d0f000011fc000074fa0000aa
:10e934001ff90000e7f60000d7f700009807000071
:10e94400ebff00006ef700001d0f0000a9fc0000a3
:10e9540059f70000bef70000c90e0000fe230000b6
:10e9640085000000befb0000a4fd00004a0b00006f
:10e974007c130000120500005d010000e7f20000b6
:10e98400b80300008e0f00002afc000050fb0000ba
:10e994000efe0000e0fd0000af050000e8030000eb
:10e9a400defb000047f9000049e7000099ed000094
:10e9b400dcf100009fe7000004fc0000120d0000e1
:10e9c4004f1d00007ffb000028fa0000441a0000dd
:10e9d400720f0000b31d0000b7f700007aee0000cc
:10e9e400a5fd00009bfd0000790b000011ed000067
:10e9f400e2f10000aaf10000d5f700007404000061
:10ea0400cffb00004f020000890f0000750c0000ce
:10ea1400cffc00006afb000033e900007508000029
:10ea2400730b000015ff00009aff000085f2000040
:10ea3400571a0000880f0000a7020000a3ee000090
:10ea44008afb0000251d00008a0200000bfd000067
:10ea54005eeb0000d8f900001bff000070fd000011
:10ea6400ba050000aef700007a020000f9050000c4
:10ea7400e0060000eef200001bf80000cb0f0000df
:10ea8400810c0000a20000005bf100001df80000f2
:10ea940007f70000e1040000fefd00008df0000017
:10eaa400d4f30000fdf70000421e00006eff0000da
:10eab400a3f50000bb0f00003b0b00009611000003
:10eac400c4f7000038010000eefd00004afe00001b
:10ead4007906000071ef000006f80000d4f300008e
:10eae400710a0000ac12000075fc000089fb0000f4
:10eaf400e90b0000fa0c00003f0300004105000090
:10eb0400c8ef0000d301000045030000a303000088
:10eb14008a0200001ce6000090f800003c0000009f
:10eb2400920c000066f900007af90000141300004a
:10eb3400b1f80000cef1000033f700003901000005
:10eb4400cb0c0000131500009c080000800000009e
:10eb540084010000e0030000c31000000ff800006f
:10eb640087e6000091f10000e2020000eaf50000ef
:10eb740033ee00006df6000069e4000041fd000082
:10eb8400a405000018fd000096060000f9fb000033
:10eb94004b160000d90f0000daf300006a020000ef
:10eba4008b0b0000ef11000079f80000cafd000093
:10ebb40084130000bf070000181300001e080000a3
:10ebc400e4f2000095f7000051040000670d000016
:10ebd400240800003cf1000086f80000c1ff00009a
:10ebe40067f500003908000079fa000042f60000d9
:10ebf40088fb000046f60000b5f90000fcf20000b6
:10ec040036010000ad090000510c0000750200003f
:10ec1400e4fc0000000c000065030000eb010000b0
:10ec2400a700000094f700002e0b0000c70a0000a4
:10ec340049000000ecf90000e7f10000baf9000017
:10ec44007cff000062090000f4f0000029f20000db
:10ec5400e4010000cff600007bf6000090f900000c
:10ec640033020000fefa00006f0a000017f90000ea
:10ec74008d0600003a160000070600000b1c000079
:10ec8400c0f5000063f30000ac00000012140000a3
:10ec9400f30f0000eff80000d909000073f400003e
:10eca400e3fe0000adf9000003f50000aeff000034
:10ecb4008f0300007804000053fa0000bff6000040
:10ecc400b3f50000bc08000055fe000020fa000067
:10ecd400dbf900002c08000037010000b0f500004b
:10ece4001f030000a8ea0000d90200001d0e000066
:10ecf400ed03000083fe000042ec0000c1fd0000b3
:10ed04007e0c00007c080000630a0000c80a0000b2
:10ed14006d060000aaff0000e7ed0000cbfb000039
:10ed2400a80a0000290d0000dc0c0000ebf700002d
:10ed3400c8f2000072fa000031010000550b000017
:10ed440071fe0000cff600002808000020fb000040
:10ed5400b70a0000db00000003f80000fe0a000010
:10ed64008bf70000fe07000080f50000a6f6000007
:10ed7400c6ff0000ad040000b30a00006df10000fe
:10ed8400a50c0000980700000d020000e2f9000045
:10ed940062f60000520600006f1300002b130000ff
:10eda40037f6000032f300003bdc00004ef70000b1
:10edb4000c0800002bfb00003ff7000059f3000093
:10edc400f900000058e9000009ff0000eaf600001d
:10edd400f0050000a61c0000aff40000f9f70000e5
:10ede400ccef0000780700004f150000651100000b
:10edf400daff000099fb0000be1a00002d08000095
:10ee0400b80a00003900000004ff0000520f00009f
:10ee140090120000670b00009af100004bf800000c
:10ee240075f100006b040000080100003be50000e0
:10ee340052020000eb000000f0f10000fbf30000c0
:10ee44001efb0000b60d0000431c00009b0a0000de
:10ee5400f5ea000023f000000ffe0000c60a0000df
:10ee64007d1800007fff0000a8f0000057ff00009d
:10ee74005afe000030fc0000cdfa000013ff000031
:10ee8400fc0300000108000003fe000038ed000050
:10ee940011f5000021f90000db040000e204000089
:10eea400c6e70000a5f30000ff0e0000c300000049
:10eeb4004bfb00008eff0000770500006d1700007b
:10eec400b9140000fffb00000bf5000064fe000015
:10eed400e9000000e92000005f0f00009af3000041
:10eee4001e080000ddfb0000c1fb0000f7f9000074
:10eef4000cff0000c3090000540c0000ce04000005
:10ef0400b3ea00000fef000049f700000906000013
:10ef14006f0d0000e4ee0000a6e50000e10500002e
:10ef2400d0030000b7fa000053ff0000f7f200001e
:10ef34008a020000c6080000e4f8000009f300009b
:10ef440037ff000076030000d40900002d120000f2
:10ef540065f50000c90000003d12000064f60000e1
:10ef640023fb0000a900000073ff00002d1900001e
:10ef7400c70f000071f80000b7f900003bf900006a
:10ef840094020000b9130000440400000cef0000d8
:10ef94005cfe0000d9080000a2ff0000ac010000e4
:10efa400850b0000feff00007e0600001dfa000035
:10efb4003feb000003080000f0fb00001208000013
:10efc400cd0b0000beee000066f80000a9080000aa
:10efd40016050000fef60000fefd0000b2f9000078
:10efe40090030000650b000092f800006bf4000031
:10eff40019f20000a3ed0000f0fe000081050000fe
:10f0040067ed0000e7fd00000e040000b4f200000c
:10f0140090f80000530100008a0100003608000047
:10f02400ad060000d1f5000001040000f80700005f
:10f034008a0e0000c7100000390200004dfa0000db
:10f04400aa0900004c1000000ffa0000100f000085
:10f05400bb030000cc0700006f1200007cfc000022
:10f064006c010000cff70000c8fa000060fb00004c
:10f07400a7ff0000fced0000e5f90000090d000009
:10f084007df2000093fb0000a1f80000840400005e
:10f094001d0a000001070000def9000080f50000f1
:10f0a400450900009af900004b0c00001f00000005
:10f0b400b2ef00005703000039fd000085f800009e
:10f0c400e2fe00004d0c00008d050000cf0800009a
:10f0d4009300000058ee000043f900002ffa0000ee
:10f0e40091f600009901000010f4000096f400006d
:10f0f4008e120000fbfd000021fa0000270400002e
:10f10400b40400007e0e0000b20b0000a406000050
:10f114007df90000c90900003a050000c8ff00009d
:10f124007a0b000057f90000540200002f0600007b
:10f1340027f60000a5f6000052050000ca050000ed
:10f14400840800006d0b000057ed00009cf30000e4
:10f15400cdfe000073f500000fff000066f0000014
:10f16400e2f10000aaff00001dff000012fc0000f5
:10f17400c6f3000015040000fa020000880b00002a
:10f184000f060000dcf70000230e000072030000ed
:10f19400320400007b030000aefa000097f900007f
:10f1a4005b0700002b0400000af40000fe090000c5
:10f1b4003a070000a4160000710a0000cef7000010
:10f1c4000ffb000080fb00002607000078f9000018
:10f1d40037090000c7f50000f6fc00006b0d0000c5
:10f1e4001af50000fe00000019000000ce0800001f
:10f1f400c308000086030000eaf70000cd01000008
:10f20400ad0800003cfb0000b70300001df7000040
:10f2140024fb00003c020000950600002af40000d4
:10f2240084f60000e90400003dfa000079080000bb
:10f23400a0f0000038f10000abf9000090f60000e7
:10f2440031ff00001dfb00008dff0000cdf0000029
:10f254008c04000066fe00007fea0000ad0200009e
:10f2640090ff00007c0f0000140800001ef6000050
:10f274002d0b00002c0b00008f0a0000d6040000a8
:10f28400d8060000b70000006dfc00008f140000d9
:10f2940041040000c0fe0000760600001d060000c8
:10f2a400890a0000cbfd000093fb0000140200005b
:10f2b400f7030000fbf700005f0000004dfd0000b5
:10f2c4000ef30000ba0800003afd000012f400003a
:10f2d40082f900002e04000027140000e702000059
:10f2e40041f800001dfe0000eeff0000cbff00000f
:10f2f400e0fa0000f80100009cfa0000c4f40000e9
:10f30400ce06000019ff0000e1fa00007fff0000b4
:10f314000d03000006050000d2f70000ccf1000048
:10f324003dff00002c03000068f5000036000000db
:10f334009dfa00002cfb00002a090000c001000017
:10f34400cafb00001dfa0000ed06000030070000b3
:10f35400320d000028040000cd0300001c11000041
:10f3640051ff0000c40100003b080000a903000095
:10f3740094f90000330400008f02000038f6000006
:10f38400e00200006b01000028060000c5fe00003a
:10f39400b0f100006afe00008a040000cbf6000011
:10f3a40008f90000ccfc000021f00000b2f20000db
:10f3b40067f900006ffc0000f8f60000b7fe0000db
:10f3c400da060000e8060000530a0000c6fe00004a
:10f3d400a70800002701000047f20000c404000051
:10f3e400d7fb00007cfb0000f4060000ec040000e6
:10f3f4006102000082fb0000450b0000aa0e000021
:10f4040025080000a9060000ba0400001e0a000036
:10f41400dafd000077ff00004e050000f6fa000058
:10f42400a6f60000120200003e01000042ff0000a8
:10f4340050090000b5000000060a00000e03000099
:10f4440031fe0000960a000078ff0000fef800007c
:10f45400a2f5000028ff0000e1f9000036fc0000de
:10f464008a06000057f4000017f60000acfb000009
:10f4740076f5000029fe00001bfc0000b8f800002f
:10f48400df010000f8f3000075f50000ab01000097
:10f4940049ff0000c2f80000f4f300004efa000037
:10f4a4005af900000f040000fe080000e8050000ff
:10f4b400dc05000015020000280b0000a40c00006d
:10f4c4008bfb000085fa0000940a0000d6020000bd
:10f4d40035020000fe0900005b0500006602000022
:10f4e40083060000f2070000ecff00002e06000077
:10f4f4005d060000b606000088ff000018ef00005b
:10f50400e3fe0000bc07000018fb000093fe0000af
:10f514005c02000066fb00005500000004060000c9
:10f52400330700008603000047ff0000cffc000003
:10f53400dcfc00009df7000052f00000fa06000019
:10f544000d02000002f20000f6020000befd000001
:10f554001bfa0000d8fd000027fc000049fe000053
:10f56400e3f9000048ff000060fe0000d4fe000044
:10f5740039fc0000b3f70000360b000061fd000009
:10f58400d4fb0000430d0000ba010000d6000000c7
:10f594005f000000a70700005a0700005b05000099
:10f5a4003d020000160000000c050000eff9000009
:10f5b4007f090000330800003efa000030ff00001d
:10f5c400edfe000004fd0000cffb000081050000fb
:10f5d400c7ff000069fe00004afc00002ffc000089
:10f5e4008602000057f80000fdfa00004b010000fd
:10f5f40030fe00009def0000bbf90000e6010000b2
:10f6040065f70000bd030000fb0200005105000087
:10f61400fe070000220000007700000007fc000045
:10f624002df500005aff0000530b00002dfa0000d6
:10f6340075fd00004d030000a6ff00008d040000ce
:10f644000a0300007a0a000031ff0000610800008c
:10f65400ce060000ebfe00006408000060f8000025
:10f66400250d0000a505000033f50000d6ff0000bd
:10f6740083040000af08000048fd0000d00400002f
:10f684008d0200001f0900009e04000037fd0000e9
:10f6940091000000edf90000af040000bafe000084
:10f6a400c4fd0000b0f000008efa0000c6ff0000a8
:10f6b4008bec0000eafb00003bf6000042ff000078
:10f6c4005f010000bcf8000041000000e2fa000005
:10f6d400df00000019050000a3fd000000f2000097
:10f6e40087f10000b1020000e101000059f90000b7
:10f6f400d90300006e0300000e080000ca010000d8
:10f70400cdfc0000bf0600008bfd00007e0500005c
:10f714005705000062fe0000b3f90000aa020000d1
:10f72400710a0000f6fe00004905000015070000fc
:10f73400220800005d090000300a000072fe00008b
:10f74400d702000075010000e7fd000096110000db
:10f75400a9f80000eefa0000ee0500004b020000dc
:10f76400ac04000043ff0000c90800001cfe0000b8
:10f77400f7fb00008bf900006ef5000016fe000098
:10f7840085f800008a0000007fff000050ed0000b3
:10f7940097f50000da02000063fe0000dbfa0000c7
:10f7a400ccf7000037f8000055020000a201000069
:10f7b4005f000000e000000060fa00008204000026
:10f7c400170600007e0100009ffc0000f703000004
:10f7d4008a0d0000dafc0000f90400002106000094
:10f7e400eb060000e1070000a9ff00005fff000036
:10f7f40043fc0000a704000097010000f609000084
:10f80400e0f30000d2f20000ce080000a9f90000e5
:10f8140036070000fafe0000cb000000d90100000a
:10f82400befd0000130100002cf600004d03000093
:10f8340046f8000043fa000055fb0000e6f3000020
:10f844008f010000a7050000900100009ffb00004d
:10f854008704000027fe00004002000000000000b2
:10f8640080f900005a000000ccf5000050010000af
:10f87400b10200006fff0000adf9000035fd00008b
:10f884009706000022ff00000e0a0000e5020000b7
:10f89400ec0600002204000027000000b70a000064
:10f8a40032020000b1060000fd080000300900002b
:10f8b40097fb00003d010000dd0b00003306000053
:10f8c40027040000e90100005c03000080f8000048
:10f8d40077050000afff000012ff000035fc0000b8
:10f8e400a4f000008f07000039f70000d8f50000ed
:10f8f4007afe000099f80000b3f8000010f7000049
:10f9040000fe000070fe000095fe00008cfc00006c
:10f91400f7f800006ff6000080fe000028010000e8
:10f924003b000000f9f700000bf60000b6020000ef
:10f934000cfe0000620200005c070000d40200001c
:10f944002dfc0000f001000095030000a902000056
:10f954005b05000010fc00005d02000078fd000063
:10f964008afd000003060000bc060000b40200008b
:10f974001dff000010050000f4000000ca0900008b
:10f984001c070000c602000086020000b10000004f
:10f99400da070000aa0400002f08000079fd000027
:10f9a4006d040000cc050000eeff00000a0a000010
:10f9b4004ffd00006601000035f9000042f7000029
:10f9c400c9fb000055fc0000e6010000d4f600006d
:10f9d40077ff000087f20000a6f500008404000011
:10f9e400ccfa00003601000020fb000095fa00006c
:10f9f40045ff000008fd000031ff000071fc00001d
:10fa040049fc000035000000a3fe000029020000ac
:10fa1400f4fc00004b000000ef0a00002ef9000087
:10fa2400ee0200004208000001050000ee0a00009a
:10fa3400b2ff0000db0500005dff00009a0000003b
:10fa440024080000150100001700000062f5000002
:10fa5400a204000000060000a4f900002e08000023
:10fa6400fef90000f5ff0000cb020000e4f4000002
:10fa7400090400009dfa0000bbff00008eff000097
:10fa840036f30000a3fb0000bdff000025080000c2
:10fa940012fd000001f800007a010000a6fa00003f
:10faa400e1fc0000cb04000082fb0000b3ff000077
:10fab4002afc0000a7fb00002309000048fa00000c
:10fac400f7ff0000a202000024050000b2050000b8
:10fad40095fd0000500c00007f01000001010000b2
:10fae400c5fe000048f90000350c00002b0700009b
:10faf400fc040000d304000015fb0000e205000034
:10fb04003b0a0000ca070000d30500005e000000a5
:10fb140068040000c9fe00006e010000a20100009c
:10fb2400a9fa000016fd000034fc00002eff0000be
:10fb3400e3f8000036f40000def8000027020000bd
:10fb4400c1fb00005df40000b00000004fff0000a6
:10fb5400deff0000eef90000adf3000081fe0000be
:10fb640097fe0000aa010000110200006af70000dd
:10fb74000ff9000058fe00001f0300004c000000b5
:10fb8400c1fd000036020000f40000008103000003
:10fb940060ff000053010000df020000a701000025
:10fba4009e010000f4f90000a5fe0000d40100004d
:10fbb400490c00003a0b000083fe0000f002000034
:10fbc400f30300003a030000ca01000091fd0000a5
:10fbd40048020000f00500005d020000a4070000d8
:10fbe40053000000fbfd00003e0600008f040000ef
:10fbf400ea0500008f0200001a0400007e030000e2
:10fc04002efc0000a3f4000007fb0000bbfe000074
:10fc14001dfe0000dafe000033f6000001fa0000c9
:10fc240097f300002e02000020070000b1f9000045
:10fc3400200200002ff700002cff0000ddfd000073
:10fc44007ff700000b04000069fb0000460200007f
:10fc5400a9fe0000c9f90000510100000bfc0000de
:10fc6400430a000085ff0000d7fd0000dc0d000002
:10fc740078030000020b000010fe0000a5fd000048
:10fc8400d6070000cf000000e0080000ba01000021
:10fc9400e5fb0000cefc00003aff00000804000071
:10fca400b202000096f9000083010000e3ff0000a7
:10fcb4002af800002f000000a8fa00002207000024
:10fcc40020fb000060f6000012fb000079f3000046
:10fcd4009608000091010000430300006a0200003e
:10fce4002ffb00008b050000c4fc0000c1fc0000d9
:10fcf40062fd0000acfd00007c0000007bfd000004
:10fd0400c9fd0000d5f90000f6f80000df0400008a
:10fd14005706000081010000df03000039030000e2
:10fd2400670500005dfc000006ff000007050000f9
:10fd3400a4050000770b0000f50200002506000072
:10fd440032fb00004904000003100000840300009b
:10fd5400220b0000c5fe0000d90300003cff000098
:10fd64005bfa0000ec030000f9f9000093030000c3
:10fd7400fcf8000023fb00006ffa0000a6f200006c
:10fd84006e03000045fa000041fc0000cbfa0000bd
:10fd9400bcfb00008802000084f80000befc0000e8
:10fda40068f900007ffd000086fe000088fd000069
:10fdb400eafe0000a7f600008f010000f701000032
:10fdc400890500003b0400003efe000033030000f0
:10fdd4008efd00007dfe000060fe0000ff030000b9
:10fde40015ff00002ffc000043fc0000c1f50000db
:10fdf4001c010000ec050000f90b0000ac08000039
:10fe04004300000091010000bf0400009b040000b7
:10fe140007000000cb0400000e040000f8030000fb
:10fe24007405000029020000b8000000200400004e
:10fe34007c0800001e050000590300005401000066
:10fe4400c5fe00005afe0000a1f6000038f90000cb
:10fe5400fbff000053fc0000b7fe00001af800008e
:10fe6400c9f8000061f90000e1fd0000ef0800009e
:10fe7400d1fb00000cff0000b2f70000baf800004c
:10fe84006c010000d7f9000064040000a5fb000029
:10fe9400860000008dff000022fb0000dd0700004b
:10fea400f9fe0000cf070000cc050000a7fe00000b
:10feb400160500000f020000fe040000da03000033
:10fec40028fe00005bfd000096ff0000a0ff00007c
:10fed40017000000030000000402000002000000fc
:10fee40024030000fc08000050fd000023ff000074
:10fef400aaff0000eafa0000d7ff000066ff000036
:10ff04001eff0000c8fc000002f9000028f60000f3
:10ff14004bfe0000950100009d040000ca0500008e
:10ff2400a0fd000087ff0000f4fb00003a0400007d
:10ff3400f2fc0000bcfb00004d02000031f60000a2
:10ff440008020000d6f90000b20200005d040000bf
:10ff540057f9000063050000bffc0000980300008f
:10ff6400ba000000d9000000b4ff0000dafd000070
:10ff74009505000055020000f00900005f04000030
:10ff840029020000c00400003906000062080000d5
:10ff9400630d0000d003000020ff00007403000084
:10ffa4009af800007d02000006ff0000cbff00006d
:10ffb4000cfb000029f60000f3fa000087f90000aa
:10ffc400a904000002fa0000b6fe000075fe00005d
:10ffd400daf70000fffe0000c8010000ca010000bb
:10ffe40037fb000044fb0000e7f8000002fe0000bd
:10fff4006dfb000002ff0000f90000008b00000010
:020000040001f9
:10000400aa030000a4fc00009b03000097fe00006c
:10001400da0200004cff00002df900003304000058
:1000240097fe00003c030000ecfa00002ff80000eb
:10003400b9000000c2fd00001806000054030000cf
:10004400d70200001ffd000022000000850a000006
:100054000bff0000d5090000c5020000f6010000f6
:10006400640900008dfc0000d10a0000a108000012
:10007400b30900006d02000012f90000d101000074
:10008400fafc0000e10600006ffe0000b7f6000075
:10009400d9f9000036f600006eff0000f9fe0000fa
:1000a400c4f900001c00000013ff000068fe0000fb
:1000b400cd020000fef800009bfe0000640000007a
:1000c40064fa000093ff000014ff000036000000f3
:1000d4002e01000046fd0000f6f500006fff000051
:1000e40087020000de030000e1030000cdf80000f9
:1000f40033fe0000910000007a060000880300002f
:10010400f3050000de04000046f80000ef050000df
:100114004a000000c1fd0000f308000001010000d6
:10012400a7ff00006c000000befd0000d904000021
:10013400af0600002aff0000c9fe000027ff0000f0
:10014400a900000078fe000022020000b2020000b4
:1001540052f70000c900000092fe000006fe0000f5
:10016400980100001ff70000d301000068fb0000a5
:10017400abfc00002503000035f9000092fc0000f0
:10018400eaf80000efff000022fe00009a020000df
:100194002608000049fd0000e90000006bf700009c
:1001a40064000000a6090000e3ff0000070300004c
:1001b400310200000cfb000056fe00003505000073
:1001c4004404000082060000d80100005406000028
:1001d4007500000091000000c4060000b501000095
:1001e4000d0c0000d5f90000f60200002604000002
:1001f400acf900007307000006f600005efc000086
:1002040031fa0000a1fe0000c6010000dbf6000088
:1002140073fc0000cbf70000cb050000c300000016
:1002240078fe00007704000066fb000000fc00007c
:1002340028fe0000c5ff00006eff000082030000de
:10024400bbfe00006cfe00000dfe0000adfd0000d2
:100254008e0200003504000078fd0000ccf7000099
:1002640051ff00008ffa0000660100005f060000e5
:10027400befe00007bfd000037fe0000b0fe000063
:100284007601000089000000e7030000ab080000cd
:10029400fffd0000df07000084020000c606000026
:1002a400b003000064f60000de08000076fd0000e4
:1002b4000f090000ae08000039fe000026fd000012
:1002c40086f60000f303000030fd0000e1040000a6
:1002d400940200004df9000092f90000e8f60000d5
:1002e40042020000820200002efd00000501000011
:1002f400e504000042fb0000cefe00005d050000a6
:10030400a7010000120000005afc000005fc0000d8
:1003140070ff0000f10000002afb00005afc0000fe
:1003240051f80000fefa0000030200000e03000072
:1003340070020000ddfc0000adfe000039f8000092
:1003440099030000160300007f030000e50300008a
:100354003df70000850c000061030000dd03000090
:100364008c080000ff07000072ff00008af70000fd
:10037400420d000090fe0000a80a000098fb000057
:10038400a0f700003c0600006cf4000018fd00001b
:1003940037fb0000d005000026f6000051020000e3
:1003a4005dfd000075f8000065100000aff6000068
:1003b400eb01000077f7000051070000d4030000b0
:1003c400b3f500007b030000b5ed0000ff0500005d
:1003d4001bf9000052ff00008913000080f900009f
:1003e40044fa0000d90200000800000020020000c6
:1003f4001205000025fd00008c0d0000caf4000069
:1004040078f80000f00600005bf90000b214000068
:1004140046fb0000960800009403000017fa000051
:10042400dc160000efec0000b00700006b000000d9
:1004340028f500009e0e000044e90000590a00005f
:100444002900000000ee00000907000063fe000020
:10045400ba070000aff800004400000022020000c8
:10046400e0f8000021fc00009cfc00007506000080
:10047400db0200007afa000029f600004a0a0000b4
:10048400b0fd00006d0b000074080000b8f6000019
:10049400910b0000e0f800006005000097fb0000ed
:1004a40019fd00008ffa00001af8000002fd000098
:1004b40085f10000e90d0000f2f600005e05000081
:1004c40069010000b0f800004f060000fcfc0000c9
:1004d400cf140000f6fd00007e050000dc010000e2
:1004e40020060000970d0000ecec000025ff000042
:1004f40083fb0000c7060000ca090000ce03000009
:100504002105000012f700002f0500001df5000072
:1005140084fb0000a5030000d1ff0000c10a000015
:1005240009eb000043f000001afe000050fa00003e
:10053400c20700008f050000df0200002702000050
:10054400af010000b6020000e6060000e7f9000073
:10055400fcfa00003b0b000022fe000055fa0000ec
:100564002bf7000091fc0000a30000007d010000b7
:100574003c06000042fc00006904000015fc000079
:1005840015fe0000de020000acf60000d7020000f9
:10059400290100007bfb000076f90000360400000e
:1005a4001505000088050000051200006101000027
:1005b400f601000018fd0000b0fe00001e1000004f
:1005c400f1030000b3fb0000cdfb0000c6020000f5
:1005d400d2f8000049f3000078010000dd020000b9
:1005e400370600009efd0000fdf9000050fa0000ef
:1005f4006dfe00001f0400008e030000ec040000e8
:10060400eef5000077ff0000dffc00003df2000083
:1006140029f40000adfb00005b0c0000a403000003
:100624000605000076fc00005cfd0000b6fd00003d
:10063400930600009f0c0000e7f80000b3060000da
:1006440033000000befd000054f500009af90000dc
:100654003e0d0000ef0a000034070000e9fe000030
:1006640078090000d3fe00002a040000ac08000052
:1006740073fe000060f5000093f300000f0100001a
:1006840098f6000059fd0000900000006e0c000078
:100694005c07000092f4000045ff00006cfd0000c0
:1006a400e2f80000980000003f0b0000ccfa0000c4
:1006b40062f4000070fd00009b01000009fa0000d4
:1006c40036fe00005a060000d1020000560d00005c
:1006d400cbfb0000adfd0000d4fa0000b701000020
:1006e400cb1100004ef8000024f70000cdf200000a
:1006f400f0060000fa08000015f00000c90500002b
:100704009a060000ebfb0000b90c0000e7fc0000b7
:10071400a8f70000600e0000c80b000012170000cc
:10072400b0fa000084f9000081ff0000aff100007e
:100734009801000061ea0000000a0000580a000065
:1007440009000000cc0300008ce2000070ff0000f0
:10075400700500004702000088fe000074f40000e9
:1007640082ff000075020000ae0000008cfb000058
:10077400c00200009f040000b2ff00004209000014
:10078400b10b00002f060000b40f00009d04000010
:10079400d5ff0000eafe0000cff20000e5f3000000
:1007a4003cf3000060040000080100007b0200002c
:1007b400db07000061f50000a2ff0000a5ef0000c8
:1007c4000eec0000400c000012fc00003605000096
:1007d400a503000085e4000021fc0000f3000000f4
:1007e400690a00008a100000200400003f0a00008b
:1007f400280d00005d13000077ff0000ebff0000f0
:10080400730b00000701000027fa0000f1f9000053
:10081400c0f700001b060000860d0000a8ee0000d3
:10082400f003000061f6000067ff0000dd11000026
:100834003ddf000020ff000056020000f00c000025
:10084400990300005fee0000ae0a0000c4ed000052
:100854009c07000046f400005df00000ae0f0000ad
:100864001af100001d130000350000006cf20000b6
:10087400870f000042fc0000d4fa00006e01000063
:10088400eb00000080030000f00b0000d004000027
:10089400bb0400000cfc000042fb00004bfc000009
:1008a400bdfb0000ce0d00008ef10000db11000046
:1008b400a7010000f6ea00004a0f0000eee0000085
:1008c400ebfe0000c8fe00008f000000411700008e
:1008d40089fe000036110000070400002c0d000002
:1008e40043ff0000dbfb000054fb000082fb000020
:1008f400d6110000e3f300005cfd000079ff000066
:10090400960600005ef7000043ee0000b0f8000019
:100914002cf5000038140000aefb0000d2fa0000f1
:100924007ffb00003bfc00007402000089eb000028
:1009340089fb0000ebfb0000880a000059fb000063
:1009440064f800001f0b00001a000000b317000039
:10095400ad0000008cfb0000ca0900008603000003
:10096400861600008a0d0000840400005809000067
:10097400830800002df7000059f400002df2000058
:1009840049f300008dff00001dfc0000a5010000dc
:100994003df90000c10200007ef600000af60000e6
:1009a400dbf80000e9f50000a71e00009af900003a
:1009b4006cf50000b90500000af300007e0d00008c
:1009c400c116000088070000960a00006dff0000b1
:1009d4001eee0000c5070000c5fe000000ff000079
:1009e40015f900009bf400000af70000cff10000a5
:1009f400c00d00005af00000f40d00005e0c000071
:100a0400e0f30000dd0d000039eb000041fc0000c4
:100a1400c7010000e2f200006bfc0000d7040000f4
:100a24008b070000360200003203000038fb000090
:100a3400750500005f18000082150000f00b00002f
:100a440027030000a8f00000110f00002b0b00008a
:100a5400b0fa0000000f000037fc000074f9000039
:100a640076e900006aee000048f10000a1090000e8
:100a7400290a00007fe00000a5fc00001ee400003d
:100a8400170300001f1c00002ef400001a0d0000c4
:100a9400aa05000064f4000079f400006a01000073
:100aa40095010000b70700005a130000dff90000a9
:100ab4009d05000026090000f6fc0000320c000031
:100ac4004eff0000b8fc0000ce1200006a0b0000cc
:100ad40096ee0000e0f600002ff5000019ec00008f
:100ae400191a0000a3fd00000efa0000630f0000b5
:100af400f2e6000037fb000040fd0000e0fc0000cf
:100b040016030000d5fc00000cec0000b8eb00005c
:100b140023100000ed0a00001d1a00000a15000051
:100b2400c9fa0000f50a0000010c0000edf900000c
:100b3400ea110000310b0000d3f80000810300002b
:100b440071df000098fe0000f2fe0000e5ef0000f7
:100b540091fc0000abf400005d070000fbea00001c
:100b6400f10000004aea000005f000000221000044
:100b74002ffa00008609000047fb0000a5f70000db
:100b840015070000200200005fff000001150000af
:100b9400071d0000c5f80000a60d000085f4000044
:100ba40092f40000870f0000461200006616000051
:100bb40034ff0000e5fc000094f40000b8030000da
:100bc4001fe60000e7f00000de0a0000f5e3000085
:100bd4000efb0000eaf30000fdf5000090070000a2
:100be400c9080000aa040000a4f6000034030000b1
:100bf400c1ef0000da040000420e00007df900009d
:100c0400771f0000cf070000b7fa0000b0150000fe
:100c14003a06000018040000050600004300000026
:100c24003d05000050fb0000a5e400007afa000036
:100c340039f9000078f10000b6f7000004f700006d
:100c4400c4fc0000b5e90000590e00004f0200008a
:100c54002d0200005f15000060ed0000250000007b
:100c640013ea00007bf20000a70e0000b60d00009e
:100c7400a317000094150000160a000088f2000073
:100c840085060000e8ff0000700900008a0d0000de
:100c9400da0b0000251e00002df6000084f9000088
:100ca400b1f7000056fb0000f9fa000063ee000003
:100cb4004503000079e500008ef80000f6fc000012
:100cc40084ee00006e030000f9f100005c030000f4
:100cd4007ff90000ddef0000fc000000300e000092
:100ce40098180000030300009f080000fbf30000b5
:100cf400d4fd0000140b000001ff0000e20f00000f
:100d040008020000c71300001f090000ce01000004
:100d140068f9000091ef0000fd070000e1f0000019
:100d24000bfc0000b3f40000b3f900007d050000e3
:100d340069fa0000990200001ffe00004905000046
:100d440011f700009cf80000a4e900006af9000013
:100d54005d1500000d100000ae17000016f900002c
:100d6400a7f800000dff0000ec060000020e0000d2
:100d7400591700003a1a00001d010000400100004c
:100d8400bfec0000ccf000004bfb0000fcf80000be
:100d94000ffc0000f7f900003ff80000a6f1000086
:100da4000f040000b8ea00001aef00001e0400005f
:100db400edef00009b09000095fb000071fb0000b3
:100dc400430d00004a0000000e0d0000d90f000082
:100dd400f30c0000e2f700006c010000ad04000019
:100de400dafe0000a41a0000ee0c00001209000054
:100df400320200004cfa0000bdfa00001e0300009d
:100e0400bd030000aafb000030040000b6df0000b0
:100e140084f10000e302000050f10000d90000005a
:100e24004bfa0000fdec0000bef90000140b0000ba
:100e340071fe0000801300007003000030fb00000e
:100e4400ec070000b6f1000020010000b30a000026
:100e5400c11a00002705000025100000f10d000054
:100e640048ff00003f15000076ed0000aaee0000e8
:100e74009ef600006bfd0000300100000900000038
:100e84002be70000d9eb00004e02000056e60000fc
:100e9400df0d0000bc03000023fd0000a7020000da
:100ea400e0ee0000f7f300009f0300000f130000c2
:100eb40047fb00000e12000093f500006df90000de
:100ec4008d240000570b0000e40d0000560b0000b9
:100ed4005800000004fb00004c0e0000ebfc000076
:100ee400d60000002a0f00001bec0000c401000023
:100ef40092000000f3f200005eff00001ef5000007
:100f0400fde2000054f20000100200001df3000096
:100f14000d0b000054000000bcf20000860f00001e
:100f2400b8fb00003a030000130f000038f600007d
:100f3400cffb0000600e00008c0600004709000093
:100f4400d1120000aaf70000cdfc0000af0600009b
:100f5400fd0400000c0a00004509000000fd00002b
:100f6400c3f300003cf40000d2dc000032050000b2
:100f74005900000085eb00009b0a00004df20000c0
:100f84000e030000db120000f9010000d8f4000099
:100f94006fff0000fff9000022fe0000ae11000008
:100fa4008bf60000750f00009f1500005bfe00002b
:100fb40050ff00002e1200006c0b000039050000e9
:100fc400220e00002be70000ae000000dcfc000055
:100fd40086f300006f0c000074ec00006af9000056
:100fe4004801000025f5000089f2000070000000af
:100ff4002f04000001ec00009005000045f90000fa
:1010040012f600007d1100002df000006c030000ba
:10101400080a0000f3000000181800004f0b00003d
:1010240074fb0000f4f500004f080000b3fd00005d
:1010340078040000a20e000025080000410d000005
:10104400ddf300007cfb0000dc030000a9010000cc
:101054007aef000080fd0000eaf4000026eb0000b7
:10106400f010000030f300006601000008fc0000ee
:101074007dfb00005a06000078fa00007d0900009c
:10108400f5070000760c0000b2ef00005b060000dc
:101094002505000044fa00001d050000d9fe0000eb
:1010a4009e0b000013050000d116000030fe000066
:1010b400a407000031f900007bf20000ec130000eb
:1010c400e5e60000b6f900001d0100000ff0000085
:1010d40066ed0000d4f40000a20000000703000045
:1010e400d1080000dfee0000cbf5000027f500007a
:1010f4000df8000061140000dd0900008505000002
:10110400480d0000750a000053030000400600006b
:101114004d1300001c0500005b0b00005803000089
:10112400a8fb00001310000053ec0000ba010000fb
:101134001802000072f200009407000006fb000091
:101144000b000000f9e5000059f4000025f500004b
:10115400a0f600001c0400003af20000720e000029
:1011640081f5000070fa000008140000070b00006d
:101174007b040000d4fc0000fbfb00001ff1000016
:101184008b0a00002c090000d60d0000340d00006d
:10119400f6fa00000c0e0000440300003cfe0000c0
:1011a400c1030000b6070000baf30000d8f3000042
:1011b400d3fa000004e9000047fd0000ecf200004f
:1011c4009df80000f5ff00000afd0000580a000029
:1011d4001c0700009d010000a9f60000cd150000c9
:1011e40028050000a3ff0000a20b00008df50000fd
:1011f400be050000bafd00008a0f0000970b000036
:10120400e70b0000e20100000df2000036fe0000d2
:1012140099df0000c50d000037050000f4fb000055
:1012240042090000f7ed000012010000b1f20000d5
:10123400f70500000bfa0000a8fc00001a040000e7
:101244009bf40000ae11000048ef000096fc000083
:101254005006000064f500008b020000a9ff0000a6
:1012640046070000bf00000020070000150300002f
:101274009404000070070000d8fd0000080e000070
:10128400c4ff00005cf900009e0b0000a6090000ea
:10129400cc060000beff00009cf10000caee000076
:1012a400c8f00000d7f700009ffe0000f6fe000023
:1012b4005c00000053fd00008f08000023000000c4
:1012c40082020000f112000039f70000a1ff0000c3
:1012d400ccfe0000e0f4000053080000000400000d
:1012e4008f07000014070000040000001ffc00002a
:1012f400fb080000cb07000031fc0000dd07000004
:1013040034ff00003ffe00005d010000c1f7000053
:1013140068f00000d2f20000d2f700002bfe0000bb
:10132400da040000adfa0000c9fb000034fc000040
:101334000cee0000ebf30000f2010000dc00000002
:10134400890f0000a80a0000390000001e0e0000ea
:10135400dc0c0000b5110000fa0c00002d060000a2
:10136400c7fc0000e50700003b0500004ef7000045
:10137400760c0000d2f3000038fb000010fb0000e4
:1013840083ed0000dffb0000ecf1000010fe000024
:10139400d1f20000a7fc000097fa00004e04000000
:1013a4007a100000aeee00004f0a00004800000072
:1013b4000a0500006e0c0000d8fc00005d0500006a
:1013c4006cfa000007050000eff90000280a00008d
:1013d4007e0300009ef90000210a0000b0f6000020
:1013e4004b0b0000560a00002aff00008e0000008c
:1013f4000efa00006af100007df5000046fb0000d3
:101404008cf50000d3020000e9f80000f9fc0000ac
:1014140063fe0000cc000000050800003d0400004d
:10142400ec0800001efb0000951100008707000077
:10143400ecfb0000d50b00007af80000a1050000c9
:10144400a30b0000570100000500000090fd000000
:10145400a7f6000006fd000040f9000015f40000a6
:10146400130a00007100000057f800004cfa000055
:101474007ffe0000e5fe0000f20000000e03000005
:1014840085fa0000e50000000bfd0000d703000012
:10149400e8010000dbf90000a9010000bc02000023
:1014a400fafa000071f90000180600002a00000092
:1014b4006bff0000b6030000effe0000a30800006d
:1014c400ef08000030ff0000370b0000dd020000d1
:1014d400c5fd0000720c0000f0fa000001f50000e8
:1014e400fcfd0000dbfa000095f500008dfc000017
:1014f4004bf80000d0fd0000470100009df40000ff
:1015040060030000f7080000e6090000af020000d5
:10151400d208000036fa00007cf30000b40c00008e
:1015240097fa000073080000b4080000ca01000024
:10153400b50a0000caf60000a0ff0000460a000039
:10154400e5fc0000bef80000060700009d02000054
:101554001bf90000f4fc000078f9000063f50000ba
:10156400b8f60000c5fa0000dbfd000087fe0000ad
:1015740017f60000aefe0000c804000040f20000b0
:10158400fb010000070d00007ffb0000fe000000cf
:10159400120700003e0900000f0d0000a60d000018
:1015a40065040000080600009b0100002dfd0000fa
:1015b40008100000e5f600004efb00001b070000c9
:1015c4004cfc00006bf8000050f2000083060000a1
:1015d40010f1000022f60000caf40000e0f600005a
:1015e400370b00008ef60000af0f0000430300002d
:1015f400b602000060080000fdff0000d6020000f3
:1016040047f300004e0a000004fe0000ba04000084
:1016140087000000cefb00003c0b000004f000003b
:10162400d9010000e3030000e3040000f107000017
:10163400cf050000bcfe0000a2f10000a1fe0000e6
:10164400c4f3000069fd00006df7000073f70000ab
:101654007c060000d5fe000006fe000045060000e2
:10166400750d0000cdfa000048080000eb010000f1
:10167400afff00006a0b0000d7fd000072090000f4
:10168400bf0200007d04000013010000e40200001a
:1016940050fe000013f400000606000076f7000078
:1016a40075f90000150500002efd000096f80000f5
:1016b4008bf800001ef8000098fe00000bff0000ed
:1016c4005ef900009b05000034fc0000e702000006
:1016d4001f0c00000d02000067ff0000d3fd000096
:1016e400de040000fef8000047020000fe050000d2
:1016f4004c0200009509000090f1000043fe000038
:10170400dc040000b8fa0000cb0900005f0600000a
:10171400eb0300000e0700000a0200004dfb00006e
:10172400c8fa000066f8000092f9000096fb000079
:101734002ffa000049fa0000bf0000007802000000
:101744008af400003a0600005a080000be040000b3
:10175400fa0c000045fc0000f9fe00000e01000038
:10176400b30300009802000028020000d1fb00002f
:1017740017fa0000eb0200000cf90000220600003a
:101784001b0800008a030000d1fb0000e2fb0000fc
:1017940082000000cafb000004020000fff7000002
:1017a400310300008cfb000096fa00009b0200004d
:1017b40022f900007503000013fb000032ff000053
:1017c40043fd0000b40000005f070000b6fd000008
:1017d4008c0300004bfe000053060000430a000087
:1017e400d5fd0000a303000013000000b3fe0000b9
:1017f400e3090000a00200005300000064000000a0
:101804004cfa00007ffa0000d3f9000099fd0000b3
:101814006a0400004a020000f0f6000086f20000ac
:10182400c4f90000e40400007b000000c0040000d0
:10183400be040000140100000b0a0000c9fd0000f2
:101844002a0700003b030000a5fa0000e50400009d
:101854000efa00001eff000071fe000086fe00006c
:10186400f90100003bf900004f020000b30500003d
:10187400d7ff0000dd030000a3f90000aaf900006f
:10188400ddff000045fe00007f080000ccf50000ed
:10189400bdf90000ecfb000017f60000650700002e
:1018a400cefb00008c0f0000f004000090fb000051
:1018b400ad0a000091fe00001b0c000080fe000039
:1018c40037040000510200003df90000390b00000c
:1018d400fffb0000b006000016000000eef100005f
:1018e40060ff000080f6000053ff00003a0600008d
:1018f4007bfa00006bf90000d8fd0000de02000056
:1019040045fc0000b8fe000050fc000049f900004e
:10191400640500008f0200005a020000b8050000b0
:101924003606000003ff0000dc030000e9fb0000b2
:10193400e2ff00006e110000def700007efb0000f5
:101944008ef700007af900006507000062ff0000ce
:1019540083010000e8fe000085020000c5000000cd
:10196400af0300001ffe000005010000e5ff0000ba
:1019740083f900001cfd000010f80000ea000000dc
:10198400f2fd00003b0000001afd00008d02000083
:10199400170c000052090000f30700007bfe000052
:1019a400c1fd0000eefe0000ce0a0000a7fd00000d
:1019b400ad0200004a060000caf000004200000028
:1019c40022f80000c8fd0000f20700002cf7000018
:1019d40045fc000007fe0000520100004500000025
:1019e400e8ff0000ee020000a6f800003b00000043
:1019f40083fb000097fd0000b8060000cefd000048
:101a04006f00000054fb0000f802000068000000b2
:101a140026060000e502000073f90000160b000022
:101a24007bf90000e20600006405000051f70000a5
:101a34008206000072fb0000f00300009a0300001d
:101a440099fd0000ca050000f9fd000092fc0000a9
:101a540084fa000055fd00009d070000d1f9000044
:101a64008ef80000d3f6000065fd000012070000a8
:101a74009ffd0000010b0000a000000057030000c0
:101a840055040000940100004f070000a9fc000069
:101a9400220a00000af8000009fe0000bbff000053
:101aa40060f5000097070000eef500008b000000d1
:101ab4007d020000a5fd0000a30600007bfb0000e2
:101ac400f100000003fa0000f6fc00005f020000d1
:101ad40065fb00004e00000048fa0000c7fc00004f
:101ae40080fd000099fe0000eb050000f9070000ee
:101af4007201000060010000ad05000083fd0000dc
:101b04002c080000e50100008c0500001105000010
:101b140032fa00004a060000f9fe0000c0ff00008f
:101b24007cfc000073010000e3fc0000bcfb00002f
:101b340041000000a9f8000059ff0000caf70000a6
:101b4400a3fe000054ff00006500000084fd0000b7
:101b540074010000f202000075f80000470a00005a
:101b6400c2fe0000b00400002107000044fd000094
:101b74009e040000defb000037050000fbfd0000b2
:101b84009efa0000adf9000064f700002c0c000080
:101b9400bafc00004a0300006307000034f60000aa
